:020000040800F2
:1000000000000120352300084B1600084D1600089B
:100010004F16000851160008531600080000000093
:10002000000000000000000000000000551600085D
:100030005716000800000000591600085B1600085B
:1000400085230008852300085D1600088523000825
:1000500085230008852300088523000885230008E0
:1000600085230008852300088523000885230008D0
:1000700085230008852300088523000885230008C0
:1000800085230008852300088523000885230008B0
:100090000000000085230008852300088523000850
:1000A0008523000885230008852300088523000890
:1000B0008523000885230008852300088523000880
:1000C0008523000885230008852300088523000870
:1000D0008523000885230008852300088523000860
:1000E0008523000885230008691600088523000879
:1000F00085230008000000000000000085230008A0
:10010000852300088523000875160008852300084C
:10011000852300088523000885230008852300081F
:10012000852300088523000885230008852300080F
:08013000852300088523000867
:1001380010B5054C237833B9044B13B10448AFF319
:1001480000800123237010BD08010020000000007A
:1001580078EA000808B5034B1BB103490348AFF31D
:10016800008008BD000000000C01002078EA0008AB
:10017800034613F8012B002AFBD1181A01387047DF
:1001880081F0004102E000BF83F0004330B54FEA40
:1001980041044FEA430594EA050F08BF90EA020FAD
:1001A8001FBF54EA000C55EA020C7FEA645C7FEA40
:1001B800655C00F0E2804FEA5454D4EB5555B8BF63
:1001C8006D420CDD2C4480EA020281EA030382EAD4
:1001D800000083EA010180EA020281EA0303362D66
:1001E80088BF30BD11F0004F4FEA01314FF4801C39
:1001F8004CEA113102D0404261EB410113F0004F4B
:100208004FEA03334CEA133302D0524263EB430301
:1002180094EA050F00F0A780A4F10104D5F1200E9F
:100228000DDB02FA0EFC22FA05F2801841F10001FA
:1002380003FA0EF2801843FA05F359410EE0A5F1CE
:1002480020050EF1200E012A03FA0EFC28BF4CF0FF
:10025800020C43FA05F3C01851EBE37101F00045B5
:1002680007D54FF0000EDCF1000C7EEB00006EEBC2
:100278000101B1F5801F1BD3B1F5001F0CD349084C
:100288005FEA30004FEA3C0C04F101044FEA4452A3
:1002980012F5800F80F09A80BCF1004F08BF5FEA2A
:1002A800500C50F1000041EB045141EA050130BD0A
:1002B8005FEA4C0C404141EB0101013C28BFB1F51C
:1002C800801FE9D291F0000F04BF01460020B1FA67
:1002D80081F308BF2033A3F10B03B3F120020CDA3A
:1002E8000C3208DD02F1140CC2F10C0201FA0CF018
:1002F80021FA02F10CE002F11402D8BFC2F1200C7D
:1003080001FA02F120FA0CFCDCBF41EA0C01904032
:10031800E41AA2BF01EB0451294330BD6FEA04047B
:100328001F3C1CDA0C340EDC04F11404C4F1200266
:1003380020FA04F001FA02F340EA030021FA04F378
:1003480045EA030130BDC4F10C04C4F1200220FACF
:1003580002F001FA04F340EA0300294630BD21FA0D
:1003680004F0294630BD94F0000F83F4801306BFD3
:1003780081F480110134013D4EE77FEA645C18BFC7
:100388007FEA655C29D094EA050F08BF90EA020F5E
:1003980005D054EA000C04BF1946104630BD91EA56
:1003A800030F1EBF0021002030BD5FEA545C05D159
:1003B8004000494128BF41F0004130BD14F5800498
:1003C8003CBF01F5801130BD01F0004545F0FE410C
:1003D80041F470014FF0000030BD7FEA645C1ABF41
:1003E800194610467FEA655C1CBF0B46024650EA78
:1003F800013406BF52EA033591EA030F41F40021A4
:1004080030BD00BF90F0000F04BF0021704730B529
:100418004FF4806404F132044FF000054FF00001FE
:1004280050E700BF90F0000F04BF0021704730B5BF
:100438004FF4806404F1320410F0004548BF404294
:100448004FF000013EE700BF42004FEAE2014FEAE9
:1004580031014FEA02701FBF12F07F4393F07F4FC4
:1004680081F06051704732F07F4208BF704793F0C7
:100478007F4F04BF41F40021704730B54FF46074DA
:1004880001F0004521F000411CE700BF50EA0102DD
:1004980008BF704730B54FF000050AE050EA010286
:1004A80008BF704730B511F0004502D5404261EBF6
:1004B80041014FF4806404F132045FEA915C3FF437
:1004C800D8AE4FF003025FEADC0C18BF03325FEAD4
:1004D800DC0C18BF033202EBDC02C2F1200300FA85
:1004E80003FC20FA02F001FA03FE40EA0E0021FAAA
:1004F80002F11444BDE600BF4FF0FF3C06E000BF28
:100508004FF0010C02E000BF4FF0010C4DF804CD94
:100518004FEA410C7FEA6C5C4FEA430C18BF7FEA54
:100528006C5C1BD001B050EA410C0CBF52EA430C82
:1005380091EA030F02BF90EA020F0020704710F102
:10054800000F91EA030F58BF994208BF90422CBF91
:10055800D8176FEAE37040F0010070474FEA410C8A
:100568007FEA6C5C02D150EA013C07D14FEA430CA8
:100578007FEA6C5CD6D152EA033CD3D05DF8040B19
:10058800704700BF8446104662468C46194663464B
:1005980000E000BF01B5FFF7B7FF002848BF10F122
:1005A800000F01BD4DF808EDFFF7F4FF0CBF012067
:1005B80000205DF808FB00BF4DF808EDFFF7EAFFE3
:1005C80034BF012000205DF808FB00BF4DF808ED9E
:1005D800FFF7E0FF94BF012000205DF808FB00BF93
:1005E8004DF808EDFFF7CEFF94BF012000205DF81D
:1005F80008FB00BF4DF808EDFFF7C4FF34BF01202A
:1006080000205DF808FB00BF4FEA410212F5001216
:1006180015D211D56FF47873B3EB625212D94FEA41
:10062800C12343F0004343EA505311F0004F23FA2B
:1006380002F018BF404270474FF00000704750EA80
:10064800013005D111F0004008BF6FF0004070473D
:100658004FF00000704700BF80F0004002E000BF8C
:1006680081F0004142001FBF5FEA410392EA030F95
:100678007FEA226C7FEA236C6AD04FEA1262D2EBDF
:100688001363C1BFD218414048404140B8BF5B42E4
:10069800192B88BF704710F0004F40F4000020F07D
:1006A8007F4018BF404211F0004F41F4000121F093
:1006B8007F4118BF494292EA030F3FD0A2F10102DD
:1006C80041FA03FC10EB0C00C3F1200301FA03F11B
:1006D80000F0004302D5494260EB4000B0F5000F3E
:1006E80013D3B0F1807F06D340084FEA310102F1FD
:1006F8000102FE2A51D2B1F1004F40EBC25008BFAF
:1007080020F0010040EA03007047490040EB000078
:10071800013A28BFB0F5000FEDD2B0FA80FCACF179
:10072800080CB2EB0C0200FA0CF0AABF00EBC250A6
:1007380052421843BCBFD0401843704792F0000F94
:1007480081F4000106BF80F400000132013BB5E7E7
:100758004FEA41037FEA226C18BF7FEA236C21D05D
:1007680092EA030F04D092F0000F08BF08467047C2
:1007780090EA010F1CBF0020704712F07F4F04D190
:10078800400028BF40F00040704712F100723CBFA3
:1007980000F50000704700F0004343F0FE4040F4CD
:1007A800000070477FEA226216BF08467FEA23638B
:1007B8000146420206BF5FEA412390EA010F40F476
:1007C800800070474FF0000304E000BF10F00043C2
:1007D80048BF40425FEA000C08BF704743F09643A9
:1007E80001464FF000001CE050EA010208BF7047C4
:1007F8004FF000030AE000BF50EA010208BF70474B
:1008080011F0004302D5404261EB41015FEA010C5F
:1008180002BF84460146002043F0B64308BFA3F157
:100828008053A3F50003BCFA8CF2083AA3EBC25339
:1008380010DB01FA02FC634400FA02FCC2F1200258
:10084800BCF1004F20FA02F243EB020008BF20F08F
:100858000100704702F1200201FA02FCC2F12002F5
:1008680050EA4C0021FA02F243EB020008BF20EAEA
:10087800DC7070474FF0FF0C1CEAD0521EBF1CEA18
:10088800D15392EA0C0F93EA0C0F6FD01A4480EA06
:10089800010C400218BF5FEA41211ED04FF00063EF
:1008A80043EA501043EA5111A0FB01310CF000401B
:1008B800B1F5000F3EBF490041EAD3715B0040EA41
:1008C800010062F17F02FD2A1DD8B3F1004F40EB11
:1008D800C25008BF20F00100704790F0000F0CF0E4
:1008E800004C08BF49024CEA502040EA51207F3AA8
:1008F800C2BFD2F1FF0340EAC250704740F4000083
:100908004FF00003013A5DDC12F1190FDCBF00F073
:1009180000407047C2F10002410021FA02F1C2F121
:10092800200200FA02FC5FEA310040F1000053EABD
:100938004C0308BF20EADC70704792F0000F00F00B
:10094800004C02BF400010F4000F013AF9D040EA11
:100958000C0093F0000F01F0004C02BF490011F4A5
:10096800000F013BF9D041EA0C018FE70CEAD153A3
:1009780092EA0C0F18BF93EA0C0F0AD030F0004C23
:1009880018BF31F0004CD8D180EA010000F00040D7
:10099800704790F0000F17BF90F0004F084691F095
:1009A800000F91F0004F14D092EA0C0F01D14202CF
:1009B8000FD193EA0C0F03D14B0218BF084608D198
:1009C80080EA010000F0004040F0FE4040F40000E2
:1009D800704740F0FE4040F4400070474FF0FF0C75
:1009E8001CEAD0521EBF1CEAD15392EA0C0F93EABC
:1009F8000C0F69D0A2EB030280EA010C49024FEA0E
:100A0800402037D04FF0805343EA111143EA1013C6
:100A18000CF000408B4238BF5B0042F17D024FF47E
:100A2800000C8B4224BF5B1A40EA0C00B3EB510F59
:100A380024BFA3EB510340EA5C00B3EB910F24BF42
:100A4800A3EB910340EA9C00B3EBD10F24BFA3EBC7
:100A5800D10340EADC001B0118BF5FEA1C1CE0D18F
:100A6800FD2A3FF650AF8B4240EBC25008BF20F042
:100A7800010070470CF0004C4CEA50207F32C2BF96
:100A8800D2F1FF0340EAC250704740F400004FF033
:100A98000003013A37E792F0000F00F0004C02BF64
:100AA800400010F4000F013AF9D040EA0C0093F02E
:100AB800000F01F0004C02BF490011F4000F013B88
:100AC800F9D041EA0C0195E70CEAD15392EA0C0FF0
:100AD80008D142027FF47DAF93EA0C0F7FF470AF28
:100AE800084676E793EA0C0F04D14B023FF44CAF6B
:100AF80008466EE730F0004C18BF31F0004CCAD100
:100B080030F000427FF45CAF31F000437FF43CAF3B
:100B18005FE700BF4FEA4002B2F1FE4F0FD34FF03C
:100B28009E03B3EB12620DD94FEA002343F0004352
:100B380010F0004F23FA02F018BF404270474FF000
:100B48000000704712F1610F01D1420205D110F087
:100B5800004008BF6FF0004070474FF0000070473A
:100B680042000ED2B2F1FE4F0BD34FF09E03B3EB0F
:100B7800126209D44FEA002343F0004323FA02F03B
:100B880070474FF00000704712F1610F01D1420227
:100B980002D14FF0FF3070474FF00000704700BFA0
:100BA80053B94AB9002908BF00281CBF4FF0FF31CC
:100BB8004FF0FF3000F06AB9ADF1080C6DE904CED2
:100BC80000F006F8DDF804E0DDE9022304B0704720
:100BD8002DE9F047089D0C46002B4ED194468C45D4
:100BE8008646B2FA82F262D94AB1C2F12003914034
:100BF80020FA03F30CFA02FC194300FA02FE4FEA4A
:100C08001C471FFA8CF6B1FBF7F44FEA1E4307FBAB
:100C1800141143EA014304FB06F199420AD91CEB7B
:100C2800030304F1FF3080F01281994240F20F81F2
:100C3800023C6344591A1FFA8EF3B1FBF7F007FB25
:100C4800101143EA014300FB06F69E420AD91CEB49
:100C5800030300F1FF3180F0FC809E4240F2F980EE
:100C6800634402389B1B40EA044000211DB1D34075
:100C78000022C5E90032BDE8F0878B4205D90DB1E5
:100C8800C5E9000100210846F5E7B3FA83F1002918
:100C980046D1A34202D39042C0F0F080861A64EB9A
:100CA80003030120002DE6D0C5E90063E3E7002A2D
:100CB80040F09080A1EB0C044FEA1C481FFA8CF717
:100CC8000121B4FBF8F64FEA1E4308FB164443EA39
:100CD800044307FB06F0984208D91CEB030306F10E
:100CE800FF3402D2984200F2CD8026461C1A1FFA21
:100CF8008EF3B4FBF8F008FB104443EA044300FB0E
:100D080007F79F4208D91CEB030300F1FF3402D216
:100D18009F4200F2B0802046DB1B40EA0640A5E770
:100D2800C1F120068B4022FA06F71F4320FA06FC81
:100D380004FA01F343EA0C03F44000FA01F8380C12
:100D48004FEA1349B4FBF0FE1FFA87FC00FB1E4470
:100D580049EA04440EFB0CF9A14502FA01F20AD94A
:100D68003C190EF1FF3A80F08480A14540F2818061
:100D7800AEF1020E3C44A4EB09041FFA83F9B4FB5C
:100D8800F0F300FB134449EA044403FB0CFCA445BC
:100D980007D93C1903F1FF3067D2A44565D9023B56
:100DA8003C4443EA0E40A0FB0293A4EB0C049C4293
:100DB800CE469C4651D34ED055B1B8EB0E0364EBEA
:100DC8000C0404FA06F6CB401E43CC40C5E9006487
:100DD800002150E7C2F1200320FA03F10CFA02FCCB
:100DE80024FA03F394400C434FEA1C4800FA02FE2D
:100DF8001FFA8CF7B3FBF8F008FB1031230C43EA19
:100E0800014300FB07F1994208D91CEB030300F1E9
:100E1800FF362CD299422AD9023863445B1AA4B20D
:100E2800B3FBF8F108FB113344EA034401FB07F371
:100E3800A34208D91CEB040401F1FF3613D2A342E4
:100E480011D902396444E41A41EA004139E70446F9
:100E5800F0E6084606E7C845AED2B9EB020E63EBEA
:100E6800070C0138A8E73146EDE7034699E7304615
:100E7800D4E7D6467FE7634402384DE70646234663
:100E880008460FE7023E634430E700BF704700BFE3
:100E98001348144A08B54FF00043C0E90023042260
:100EA800426101220023C2614FF480510722C0E948
:100EB8000233C0E90933C0E90C1203610383837666
:100EC80080F8203080F82C30826380F83C30C3648E
:100ED80001F090FA18B1BDE8084000F0FFBA08BD6B
:100EE80024010020002401400268084B9A4282B085
:100EF8000AD14FF0B0431A6E42F400721A661B6EA4
:100F080003F400730193019B02B070470024014071
:100F18000268054B9A4201BF4FF0B042136E23F4AA
:100F280000731366704700BF0024014030B585B0D8
:100F380000240546CDE901440394FFF7A9FF1448AE
:100F480001F0ECFD08B100F0C9FA1148039401A9B9
:100F5800CDE9015401F0ACFB08B100F0BFFA0C4830
:100F680001F006FD08B100F0B9FA4FF0FF3108486A
:100F780001F040FB064801F0B3FD054801F094FB81
:100F88000446034801F056FD204605B030BD00BFB9
:100F980024010020014B024A1A60704724010020F6
:100FA8000024014008B50948FFF7C0FF68B1084BA5
:100FB800B3F8AA304FF6FF72934216BF40F6E442E8
:100FC800044B5343B3FBF0F398B208BD002000B4C0
:100FD8000075FF1FD8084C0013B50023ADF8063084
:100FE800FFF7E0FF04461948FFF7A0FF184BB3F8D6
:100FF800C820B3F8A8108A4204FB00F018D040F6C5
:10100800E443B0FBF3F364205B1A4343521A93FBA7
:10101800F2F31E331BB2ADF80630BDF806305BB2F2
:101028001B02ADF80630BDF8060000B202B010BDD4
:101038004FF47A7240F6FF73B0FBF3F35343A3F512
:101048003923A3F50C6340F6C412E0E7001000B0A2
:101058000075FF1F4FF0B04307B59A6C42F00402C9
:101068009A649A6C02F004020192019A9A6C42F016
:1010780001029A649B6C03F0010300930022022191
:101088000F20009B01F0E8FD0F2003B05DF804EB92
:1010980001F014BE08B501F095FF10B16FF004001F
:1010A80008BD064B9A6942F040429A614CF2FA3206
:1010B8001A6101F099FF0028F2D0EFE700400058CC
:1010C800F0B585B000230D4600930646A8B3FFF798
:1010D800E1FF044670BB01F075FF88BB1A481B4A44
:1010E80002230193D0F8E01506F1784302EA812142
:1010F800B3FBF1F701FB1733DB0A0293D0F8E005E5
:1011080005F178410139314402EA8022B1FBF2F05D
:1011180002FB1011C3EBD1230133694601A80393E5
:1011280001F0E2FF20B1022814BF6FF0010401248E
:1011380001F05AFF204605B0F0BD6FF00504F9E74D
:101148006FF00404F6E700BF0070FF1F00FCFF0308
:10115800014B186000207047880100202DE9F04FEE
:10116800B0F1006F89B006460F469046C0F0C080C7
:10117800DFF89091644DD9F8E03505EA832303F14F
:101188000063013B984200F2B380002900F0B3806D
:1011980040EA02035B0740F0AE80FFF77BFF04469E
:1011A80090BB01F00FFF002840F0A880D9F8E015A7
:1011B800009705EA812106F17842B2FBF1F301FBC1
:1011C800132208F17843013B3344B3FBF1F001FBF0
:1011D8001033DB0A01334FEAD22AA3EBD222012AC9
:1011E800039388BFC6F30A050AF58037C6F10803DA
:1011F8008CBFC5F500654546FF02B3460693039BC1
:101208009A4505D301F0F0FE204609B0BDE8F08FFD
:10121800A6F10803069A1A4495421CD8009B049527
:101228000193CDF814B04FF00009059B09EB0301B9
:10123800049B99453DD3009BAB442B44A8EB050583
:10124800B5F5006F009328BF4FF400650AF1010A55
:1012580007F50067D3E753F8081F5A68B2F1FF3F54
:1012680008BFB1F1FF3FD5D0284B186810B96FF00F
:101278000504C7E727B14FF4006239460CF01EFF9A
:10128800DFF888900099D9F80030CBF30A001844A9
:10129800AAB20CF013FF4FF400613846FFF710FFB5
:1012A80000BBD9F8003001934FF40063059704930D
:1012B800B9E7019B07914B4402930120D3E900232E
:1012C80001F0CCFE88B90799019BD1E9000259F8D1
:1012D8000310029B5B689A4208BF884205D109F156
:1012E8000809A2E76FF001048CE76FF0030489E7AF
:1012F8004FF0FF3488E76FF0050485E76FF00404CA
:1013080082E700BF0070FF1F00FCFF038801002078
:10131800B1F1006F70B510D30B4BD3F8E0650B4BF0
:1013280003EA862303F10063013B994205D838B1EB
:1013380092B20CF0C3FE002070BD4FF0FF30FBE707
:101348006FF00500F8E700BF0070FF1F00FCFF0307
:10135800B0F1006F10B40DD3084BD3F8E045084B3B
:1013680003EA842303F10063013B984202D810BCCE
:10137800FFF7A6BE4FF0FF3010BC70470070FF1F8C
:1013880000FCFF034FF0B04382B0DA6C0243DA642A
:10139800DB6C03400193019B02B0704770B50220DB
:1013A80086B000251F4ECDE90455FFF7EBFF04205A
:1013B800FFF7E8FF0120FFF7E5FF01A94FF6FF72ED
:1013C800032330464FF0B044CDE90123039501F0E3
:1013D800D9FE01A9144801F0D5FE01A94FF09040AB
:1013E80001F0D0FEE36C23F00103E364E36C23F027
:1013F8000203E364E36C23F00403E3640220FFF7D1
:10140800C1FF10210123CDE90113CDE9030501A98D
:10141800304601F0B7FEE36C23F00203E36406B044
:1014280070BD00BF000400480008004800B59BB02C
:101438004822002108A80DF06DFA1822002102A800
:101448000DF068FA01F0CCFF4FF0B0420120D2F85D
:10145800903023F01803C2F89030D2F8003423F407
:10146800C06343F40073C2F80034D2F8003403F4C4
:10147800C0630193019B2423089381230B930023CA
:10148800CDE91003B02208A8CDE9122302F020F913
:1014980008B172B6FEE74F23CDE90230CDE904006A
:1014A800CDE90600022102A802F0ACFB08B172B631
:1014B800FEE71BB05DF804FB08B500F061FFFFF71D
:1014C800B5FFFFF76BFF044803F0BAFA00F030FCF1
:1014D80000F035FCFCE700BF3C02002072B6FEE7D6
:1014E80000B58DB02C22002101A80DF013FA174881
:1014F800174B03601F2383604FF080420023C0E92D
:101508000433C0E9072383614FF48073436202F018
:101518001FFE08B1FFF7E2FF0C4802F045FF08B1D3
:10152800FFF7DCFF4FF000530022079307480892AB
:101538004FF4807301A9029206920B9302F068FEA1
:1015480008B1FFF7CBFF0DB05DF804FB8C0100205C
:101558000028004010B5044690B03822002102A8A7
:101568000DF0D8F92268194B9A422CD14FF48033E8
:10157800029302A84FF480730F9302F067FC08B13E
:10158800FFF7ACFF4FF0B0430220D3F8902042F4AD
:101598000042C3F890209A6D42F480629A659B6D70
:1015A800002203F4806311460193019B01F054FB70
:1015B800022001F083FB00222A20114601F04CFB97
:1015C8002A2001F07BFB10B010BD00BF00280040AE
:1015D8007047000008B50F4803F032FA00F066FBC8
:1015E8004FF6FF714FF0904001F078FE0A484FF631
:1015F800FF7101F073FE09484FF6FF7101F06EFEAE
:1016080000F0D4FE064B0120C3F88800BDE808406E
:1016180001F03EBF3C0200200004004800080048DA
:101628000004005800F0C9BE08B500F0BFFEBDE8D0
:1016380008400121002001F0DBBE704700F0BDBE6C
:101648007047FEE7FEE7FEE7FEE7FEE770477047F4
:1016580070477047014802F0CDBE00BF8C010020E2
:10166800014802F0FBBC00BF8C010020014803F0D8
:10167800EAB800BFC4010020054808B50823036084
:1016880002F0FEFE18B1BDE80840FFF727BF08BD0D
:10169800C40100204FF0B04307B55A6E42F0010272
:1016A8005A665B6E002203F0010301931146322053
:1016B800019B01F0D1FA322003B05DF804EB01F090
:1016C800FDBA00000CB407B5054A05AB102101931B
:1016D8000CF0FEFF03B05DF804EB02B0704700BFEA
:1016E8001CEB000830B585B0044602A80D460CF086
:1016F8001BFEBDF90C30064A00931021029B2046C0
:10170800FFF7E0FF2046FEF733FD288005B030BD27
:101718001CEB00084FF0B04210B5936823F4004367
:1017280093600CF089FE0D4B01241C700CF056FBE5
:101738000B480CF06DFB0B4B4FF400421A61002074
:101748000CF06CFBFFF726FC00F0B4F80CF060FC22
:1017580021462046BDE810400CF07ABCD00100209C
:10176800ED160008004000580CF088BC08B5FFF7DB
:1017780019FC40F6B83398420CD8B0F5E16F0BD39A
:10178800FE23A0F5E16058434FF49663B0FBF3F0F5
:10179800C0B208BDFE20FCE70020FAE77FB5684626
:1017A80000F06CF80198FFF7B5F900B207B05DF8E2
:1017B80004FB0000194A38B5D2F88035591C044694
:1017C80019D100F001FE054600F00AFE054400F0BC
:1017D80001FE2B0EE3712B0CA3712B0A6371030E10
:1017E800E370C0F30742C0F307232571C0B2A270AB
:1017F8006370207038BD190AC3718171190C1B0EF2
:1018080041710371D2F88435C370D2F88405C0F3EE
:101818000722C0F30743000EE9E700BF0070FF1F6F
:1018280038B5094BD3F8803503600133054609D133
:1018380000F0CAFD044600F0CDFD444000F0D0FDA4
:1018480044402C6038BD00BF0070FF1F01210220FA
:101858000CF0E8BB002102200CF0E4BB002070472C
:10186800024B187808B100F05DB87047D00100202D
:1018780082B00190019802B000F0F0B810B50446AB
:10188800FFF7AAFB074BA36040F30F20FEF79EFF6C
:10189800054B064A2360064B6060C4E90323002019
:1018A80010BD00BF0000484200007A440D093E0008
:1018B800AB03050000207047014B1868704700BF54
:1018C800D40100200320704708B501464FF47A720E
:1018D80000238002890DFFF763F908BD4FF47A737E
:1018E800A0FB0303800A40EA83507047034B9868C3
:1018F8009A689042FBD1C043704700BF002800405F
:1019080008B5FFF7F3FF014B186008BDD4010020AC
:1019180008B5FFF7EBFF024B1B68C01A08BD00BFF4
:10192800D4010020024B187808B1FFF7DFBF7047D9
:10193800D801002010B5074B074C0122DA654FF497
:101948008071204602F050FB4FF0FF3323630020E4
:1019580010BD00BF002800408C0100200246002175
:10196800014802F058BD00BF8C0100200246012149
:10197800014802F050BD00BF8C01002010B58CB0AA
:101988002C220021044601A80CF0C4FFFFF7D2FF67
:101998000C4B0D481B681C440023089306934FF01A
:1019A8000053E443079301224FF4807301A9029482
:1019B8000B9302F02DFC08B1FFF790FD00200CB04E
:1019C80010BD00BFD40100208C01002038B50546A9
:1019D800FFF78CFF02210446074802F023FDC4F3F9
:1019E80009024FF47A71A2FB0121920AA30A2A8004
:1019F80043EA805038BD00BF8C0100200148002117
:101A080002F010BD8C0100200148012102F00ABD3E
:101A18008C010020F8B50F4D2E78CEB90E4C4FF042
:101A2800FF372763FFF75CFDFFF784FF4FF48071F2
:101A3800204602F0D9FA2046276302F097FC324686
:101A48002046022102F0E7FCFFF75AFF01232B7022
:101A58000020F8BDD80100208C010020014610B5F7
:101A68004FF47A7200238002890DFFF799F8014636
:101A7800FFF73CFF0446FFF739FF031B8B4200D3F7
:101A880010BD00BFF7E70CF0DFBD000010B5064C35
:101A98000221204602F0C6FC0221421C2046BDE875
:101AA800104002F0B8BC00BF8C0100201348144A53
:101AB80008B54FF4E133C0E9002300230C22C0E944
:101AC8000233C0E90523C0E90733C0E909330361DC
:101AD80003F0D1FC08B1FFF701FD0848002103F02D
:101AE8003FFE08B1FFF7FAFC044803F019FE18B1ED
:101AF800BDE80840FFF7F2BC08BD00BF3C0200206B
:101B08000044004070B596B006461422002103A890
:101B18000CF000FF3822002108A80CF0FBFE326808
:101B28002C4B9A4254D10223089308A82A4B0A93B3
:101B380002F08CF908B1FFF7D1FC4FF0B043002553
:101B48009A6D42F400329A659A6D02F4003202925C
:101B5800029ADA6C42F00102DA64DB6C03F00103EA
:101B680001930422019B0223CDE9032303240723C5
:101B780003A94FF09040CDE90554079301F002FB0B
:101B8800082303A94FF09040CDE90334CDE905556A
:101B9800124C01F0F7FA124925621423C4E9001324
:101BA8001023C4E9023520468023C4E90435C4E97A
:101BB800065501F0E3F808B1FFF790FC2520F4671B
:101BC80000220221A66201F047F8252001F076F8EC
:101BD80016B070BD0044004004000C00DC01002079
:101BE8005800024002680C4B9A4210B5044612D1C4
:101BF8004FF0B0420C21936D23F4003393654FF0FE
:101C0800904001F06BFBE06F01F02AF9BDE810404D
:101C1800252001F061B810BD0044004008B50A460F
:101C28000146024802F02CFF002008BD3C020020BB
:101C380013B5114B114C18604FF40013009302AB0D
:101C480013E90600204603F00FFD2368DA69D10383
:101C5800FCD4DA695202FCD59A68084842F480023A
:101C68009A6003F047FD06490448012203F0B8FCD6
:101C7800002002B010BD00BFD00200203C020020AE
:101C8800D802002008B5074B1860FFF7E3F9FFF703
:101C98000DFF054AD2F8803043F00063C2F8803067
:101CA800002008BDD40200200008005808B54FF0F5
:101CB800B04308489A6B42F400329A639A6B22F454
:101CC80000329A63FFF78EFF0F2001F005F800201D
:101CD80008BD00BF3C0200200268044B9A4203D1B1
:101CE800034B00201B681847704700BF00440040A2
:101CF800D402002002680B4B9A4210B504460FD15B
:101D0800094B1B682BB1D0F8902012B90748012164
:101D1800984720460549BDE81040012203F060BC01
:101D280010BD00BF00440040D0020020D8020020AF
:101D380008B5FFF7EFFCBDE8084000F0F1B94FF037
:101D4800FF300CF0FFB9704770477047014BD870EF
:101D5800704700BF0C000020014B1874704700BF8B
:101D68000C00002008B5022000210CF0B3F9BDE8F2
:101D7800084001480CF016BC300400200021012066
:101D88000CF0A8B910B542F21073084C002818BF1F
:101D98000346074823600CF0B7FB216804480CF0A1
:101DA8003BFCBDE8104002480CF0FCBB08000020DA
:101DB8003004002008B50E4B1B78022B03D10021FC
:101DC80008200CF087F90B4800224FF4004101F07D
:101DD800F9FA084800224FF4007101F0F3FABDE85F
:101DE8000840044800224FF4006101F0EBBA00BF3C
:101DF8007000002000040048024800224FF400410F
:101E080001F0E0BA00040048024800224FF40071D3
:101E180001F0D8BA000400480A460149FFF778BA29
:101E280000F0030838B5154801224FF4004101F0CD
:101E3800C9FA124801224FF4007101F0C3FA0F48A1
:101E480001224FF4006101F0BDFA0D480CF05CFB73
:101E580004F0E6F860B90B4C0B480125257003F037
:101E680073FF2078294603F0C7FC05480CF09AFB5D
:101E7800BDE8384005480CF095BB00BF0004004899
:101E880030040020700000200C00002018040020FE
:101E980004F064B92DE9F04387B0FFF767FCFFF75A
:101EA80081F8064603F0A2FD054690B10024444897
:101EB8000CF02AFB434B42481B689C42214638BF22
:101EC80019460CF0A9FB3E480CF06CFB07B0BDE8C6
:101ED800F0833D4C6846FFF7D1FC0223029823703B
:101EE8003A49FEF7C7FCFEF73BFE87B20198FEF7BA
:101EF80011FE37490FFA80F80098FEF7BBFC33490A
:101F0800FEF76CFDFEF72CFE324A636812781A70F1
:101F18006368C0F307225A7063689870636883F82F
:101F280003806368DFF8B0803A0A1A7163685F71EA
:101F380098F80030082B01D0012B29D862680023BB
:101F480093716268D3716268137253726423B6FB2B
:101F5800F3F60B2396726370204C637A63B103F037
:101F680031FD012808D120460CF0CEFA1C48002289
:101F78004FF4006101F026FA98F803101248002285
:101F880003F04AFD063091D103F016FD04468EE7B2
:101F9800DDE90376D4F80490FFF7E8FB89F806003A
:101FA80063683A14DA7163683A121A7232149A72D0
:101FB80032125F72DA721E735D739D730F23CAE764
:101FC800300400200800002000000020000020410C
:101FD8000000C842240300200C000020DC0200207E
:101FE8000004004802484FF4006101F0F0B900BF56
:101FF8000004004808B504F01CF880B903F0E2FCBE
:1020080001280CD1BFF34F8F0549064BCA6802F46B
:10201800E0621343CB60BFF34F8F00BFFDE708BDFD
:1020280000ED00E00400FA0508B560B1037853B18B
:10203800054801224FF4007101F0C4F9BDE80840D9
:1020480002480CF0AFBA08BD000400480C03002099
:1020580010B568B190F9064054B906480CF054FA26
:1020680022460548BDE810404FF4006101F0AAB9C6
:1020780010BD00BFDC0200200004004838B504464B
:102088000D4681B3184801224FF4004101F09AF936
:1020980016480CF087FA2B782BB324B363682278A0
:1020A8000BB3022A0ED0032A1DD16278012A1AD155
:1020B8001878012802D0022800D0A0B9BDE838401D
:1020C80003F074BD6278012A0DD11B78084903F02A
:1020D80001030B7003B91A46BDE8384002484FF4B3
:1020E800006101F06FB938BD00040048F402002017
:1020F8002403002038B504460D4607484FF4006114
:10210800FFF726F930B92A4621460348BDE838408A
:10211800FFF724B838BD00BF00F00308704700007F
:102128001FB5002403A92046039403F067FF03A901
:10213800012003F063FF2C4B2C48009422464FF4F7
:10214800FA710CF083F92A4B2A48009422464FF47E
:10215800FA710CF07BF9284B2848009401224FF4BF
:10216800FA710CF073F92046FEF7F2FF08B1FFF799
:10217800B5F9234B009400224FF4FA6121480CF082
:1021880065F9214A002101200CF060F81F4A00215E
:1021980002200CF05BF81E4A002104200CF056F8CF
:1021A8001C4A002108200CF051F800F043F81A49A5
:1021B8001A4803F0D9FE1A4803F0C6FD0F480CF080
:1021C800F1F9184B0021187803F016FB1649009412
:1021D800164B0968164800220CF038F914480CF020
:1021E800E1F904B010BD00BF111E00080C03002067
:1021F800011E0008F4020020ED1F0008DC02002088
:10220800BD1D000818040020555B00089D1E00082D
:10221800991E00082D1E000800000301240000205C
:102228000C00002070000020080000206D1D000830
:1022380030040020034B0022C3E902220122C3E933
:1022480000227047480400200048704748040020D6
:102258004FF0B04382B0DA6C0243DA64DB6C0340BF
:102268000193019B02B070472DE9F04186B000242C
:102278000220154D0594FFF7EBFF0420FFF7E8FF58
:10228800124F03944FF4807601230DEB0001CDE942
:1022980001632846032304934FF4005800F072FFAB
:1022A80001A93846CDF8048000F06CFF224641466B
:1022B800384601F087F828462246314601F082F870
:1022C800204606B0BDE8F081000400480008004838
:1022D800032810B50ED8012810D868B902460B4853
:1022E8004FF4807101F06EF8002209484FF4005154
:1022F80001F068F8002010BD0122F0E70022034831
:102308004FF4807101F05EF80122EEE70004004806
:1023180000080048022070470020704701207047DD
:10232800002814BF16200F20704700000D4885466E
:1023380000F025F80C480D490D4A002302E0D45856
:10234800C4500433C4188C42F9D30A4A0A4C0023F7
:1023580001E013600432A242FBD30CF0E3FAFFF76A
:10236800ABF8FEE700000120000000200801002073
:1023780044F6000808010020B8210020FEE7704755
:1023880010B5032000F056FC01F092F9064B1860D6
:102398000F20FFF763FA044618B9FFF751F92046F2
:1023A80010BD0124FBE700BF740000204FF0E022BD
:1023B800136923F00203136170474FF0E022136999
:1023C80043F0020313617047014BD3F8900570473F
:1023D8000070FF1F014BD3F8940570470070FF1F72
:1023E800014BD3F8980570470070FF1F8068C0F351
:1023F80080007047F7B5002301930446002800F0D9
:10240800E980856D25B9FEF76FFDE56584F85450C0
:1024180023689A68D00040F1A1809A68D10000F141
:10242800B480A26D42F01002A265E26D42F0010292
:10243800E26501251846FFF7D9FFA26D02F01002E8
:10244800024340F0C980A26D206922F4817242F0F3
:102458000202A2659A68D2075DD4226BA67E94F820
:102468002CC0003A18BF01221703D4E902120A430C
:10247800217E42EA8132617E42EAC13242EA463234
:10248800002842EA4C02B4BF20F000414FF400118A
:102498003A430A4394F82010012903D1002E76D13B
:1024A80042F48032616A21B1A66A01F4E0713143D5
:1024B8000A43D968E66C21F4FE3121F4FF71114317
:1024C800D96094F83C206168012A01F0404C4CEA3C
:1024D800060609D1D4E910273A433243A66C3243A1
:1024E80042EA0C0242F001061F693E4A3A40324372
:1024F8001A6121F00042B2F1804F0CD0B1F1004FC7
:1025080009D0394ED6F8082701F4701122F4701258
:102518000A43C6F808275A69666BA16B22F00702BE
:1025280032435A615A6922F0700242EA01125A6132
:10253800002835D19A6A62F00F029A625B6903F04B
:1025480007039E423CD10023E365A36D23F00303F8
:1025580043F00103A365284603B0F0BD9A682349F8
:1025680022F0104222F0170242F080529A60204A6C
:102578001268B2FBF1F2013252000192019A002A6C
:102588003FF44BAF019A013AF7E7002552E7A16DF6
:1025980041F02001A165E16D41F00101E16581E7AC
:1025A800B0F5001FCAD19A6AE269013A92006FF049
:1025B8000F0102F01C0201FA02F2216E0A43BCE785
:1025C800A36D23F0120343F01003A365E36D43F0FA
:1025D8000103E3650125BEE7A36D43F01003A3657E
:1025E800F8E700BF02FCFF1F00200140400D030078
:1025F80074000020F8B54569082D04460E460AD037
:102608000368DB68D80705D5A36D43F02003A365ED
:102618000120F8BD0425FFF723F9074623681A6847
:102628002A4220D0A26D42F40072A265DA6812F440
:10263800406F14D1A27E92B91A6812070FD51846B6
:10264800FFF7D4FE20BB5A6822F00C025A60A26D34
:1026580022F4807222F0010242F00102A265227E79
:10266800FAB10020D5E7711CD9D0FFF7F9F8C01BE3
:10267800B04201D8002ED1D123681B682B40CDD1A0
:10268800A26D84F8543042F00402A2650320C0E72A
:10269800A26D42F02002A265E26D42F00102E265FD
:1026A800DDE70C221A60DCE70368186C704700004D
:1026B800F7B50023019390F85430012B044600F03D
:1026C800C08005680269012380F854302846FFF766
:1026D8008DFE002840F0AF80D1E90030022822F0BA
:1026E80004027ED0B2F1004FC3F3110E35D1AA6AAD
:1026F80042EA0E02AA628A68686902EA032222F0A4
:102708007C4222F0FF0220EA03210A43002B6A617F
:102718001DDA4D4A4D4DD2F80817AB4201F0E07072
:1027280043D10D0213D4D2F8083723F0E0730343E2
:1027380043F40003C2F80837454B1A68454BB2FB0F
:10274800F3F20C2302FB03330193019B53BB0020DC
:10275800002384F8543003B0F0BD226E00F01F0748
:102768004FF00F0C0CFA07FC6FEA0C0622EA0C0C6F
:10277800BEF1000F11D1C3F38462BA4042EA0C02E1
:1027880022668008E26901309042B4D8A86AC3F38F
:102798008362BA4006403243ACE793FAA3F2B2FA36
:1027A80082F2EAE7019B013BCEE72B4DAB420BD10E
:1027B800C901CCD4D2F8083723F0E073034343F0BF
:1027C8008073C2F80837C2E7244DAB42BFD14B0231
:1027D800BDD4D2F8083723F0E073034343F48003F1
:1027E800EFE7B2F1004F01BFAA6AC3F311018A43B0
:1027F800AA62002BABDA154813498342D1F808279F
:1028080009D1D1F8083702F0A07223F0E0731A4317
:10281800C1F808279BE71048834204D1D1F808374C
:1028280002F44002F1E70D48834290D1D1F808370D
:1028380002F0C072E9E7A26D42F02002A2651846D4
:1028480086E7022087E700BF00200140001000B0A3
:1028580074000020400D0300004000B8002000B4C0
:10286800026838B504461046FFF7C0FD08B90020D5
:1028780038BD9368990707D4936823F0004323F081
:10288800170343F010039360FEF7EAFF0546236839
:102898009B685B07EBD5FEF7E3FF401B0228F6D9E0
:1028A80023689B685A07F2D5A36D43F01003A3650C
:1028B800E36D43F00103E3650120D9E773B5002315
:1028C800026801939368DD07044602D5002002B030
:1028D80070BD9168214B194209D0A36D43F01003D4
:1028E800A365E36D43F00103E3650120EFE7936817
:1028F80023F0004323F0170343F001039360184BC0
:10290800D3F8083718021CD4637E012BDED0FEF7FB
:10291800A7FF144E054622681368DB07D6D49368D0
:10292800D9075FBF9368334043F001039360FEF714
:1029380097FF401B0228EED923681B68DA07EAD400
:10294800CBE7094B094A1B68B3FBF2F30133019348
:10295800019B002BD8D0019B013BF8E717000080B2
:1029680000200140E8FFFF7F74000020400D0300B5
:1029780038B504460068FFF739FD054620BB94F8D2
:102988005430012B20D0012384F854302046FFF71F
:1029980095FFB0B9A36D226823F4706323F0010397
:1029A80043F48073A3651C23E065136084F8540026
:1029B800936823F0004323F0170343F00403936064
:1029C80038BD84F85450FBE70220F9E7026838B5AF
:1029D800936891680446C80701D4002038BD990758
:1029E800FBD4936803F00503012B19D1936823F0F6
:1029F800004323F0170343F002039360032313609B
:102A0800FEF72EFF054623689B68DB07E5D5FEF732
:102A180027FF401B0228F6D923689B68DA07F2D5FE
:102A2800A36D43F01003A365E36D43F00103E36571
:102A38000120D3E770B5044600284BD0836D43F0DE
:102A480002038365FFF70CFF054668B92046FFF7C8
:102A5800BDFF054608B90123A3652268936823F0E2
:102A6800104323F01703936023685A6822F46772AF
:102A780022F003025A6040F29F321A60D968164A5F
:102A88000A40DA601A6922F040421A615A6922F053
:102A980007025A611A6A02F0F0221A625A6A02F0B0
:102AA800F0225A62DA6A02F0F022DA629A6A0B4A73
:102AB80000269E62D2F8083723F0FE73C2F8083762
:102AC8002046FEF725FAE6652666A66584F8546072
:102AD800284670BD0125FBE700023E830020014027
:102AE80010B590F85430012B044615D0012380F816
:102AF8005430FFF7B5FE58B92046FFF767FF38B9DD
:102B0800A36D23F4807323F0010343F00103A3654D
:102B1800002384F8543010BD0220FCE7F7B50023E9
:102B2800019390F85430012B04467FD0012380F89C
:102B38005430FFF74BFF23689A6812F001020546EC
:102B480007D0A36D43F01003A365002384F8543025
:102B58002DE0A16D364F21F4817141F00201A1658C
:102B6800DE68D96826F4FF4626F07C0621F4004189
:102B7800360421F00301360CD960082099683940E1
:102B880041F0004199609968002913DA01990131EF
:102B980001910199B1F52E3FF5D3A36D23F01203EE
:102BA80043F01003A365002384F854300125284618
:102BB80003B0F0BDD3F8B410013801F07F010A4426
:102BC800DCD199681A48014041F001019960D3F8B5
:102BD800B41021F07F0141EAD202C3F8B4209A6808
:102BE800024042F002029A60FEF73AFE0746236866
:102BF8009A68D20708D4DA683243DA60A36D23F002
:102C0800030343F001039FE7FEF72AFEC01B0228D7
:102C1800EDD923689B68D907E9D5A36D43F0100364
:102C2800A365E36D43F00103E365BFE70225BEE753
:102C3800E8FFFF7F0749CA6822F4E0620302120432
:102C480003F4E063120C134343F0BF6343F400330F
:102C5800CB60704700ED00E0164B30B5DC68C4F37C
:102C68000224C4F10703251D042B28BF0423062DC5
:102C78004FF0FF358CBF033C002405FA03F321EA2B
:102C88000303A54022EA0502A340002843EA020301
:102C9800ACBF00F16040084A4FEA0313B8BF00F028
:102CA8000F00DBB2AABF00F56140135480F800336F
:102CB80030BD00BF00ED00E014ED00E0002807DBA8
:102CC800044A4109012300F01F00834042F82130E3
:102CD800704700BF00E100E000280CDB430906490B
:102CE80000F01F0020330122824041F82320BFF367
:102CF8004F8FBFF36F8F704700E100E070B5D0E9E8
:102D080013456560446D14B1D0E916456560D0E996
:102D1800105404F01C060124B4406C60046863601D
:102D28008368102B0BBFA260A160E160E26070BDF8
:102D38000268416CD3B210B5083B1424B3FBF4F31A
:102D48000B4CA24288BF0B4A21F0030199BF01F145
:102D5800804202F50232521807338264064AC2647E
:102D680003F01F03012202FA03F3036510BD00BF3D
:102D7800070402401C0802408008024038B50028B9
:102D88005CD002682E4B9A424FF014014AD82D4B62
:102D98001344B3FBF1F32C499B00C0E91013022341
:102DA80080F825301368056923F4FF4323F0700386
:102DB8001360D0E9024323432B43456911682B4331
:102DC80085692B43C5692B43056A2B430B43136065
:102DD800FFF7AEFFB4F5804F04BF0023436043689C
:102DE800816C03F07F020A60D0E91314013B032BC6
:102DF8004C601ED8154B1649816513449B00012170
:102E0800013A01FA02F200214365C2651960114BCB
:102E18005A6400230122C36380F8243080F82520F7
:102E2800184638BD0C4B1344B3FBF1F30B499B0018
:102E3800B3E70023C0E91533C365EAE70120F0E7EB
:102E480007040240F8FFFDBF000002403F82001067
:102E58004009024000090240F8FBFDBF000402409F
:102E680038B5002841D00268136823F001031360C5
:102E78001F4B9A424FF0140130D81E4B1344B3FB3A
:102E8800F1F31D499B00C0E91013012403F01C0352
:102E980004FA03F3002515604B60FFF749FF836CC4
:102EA80041681D60D0E913325A604A1E032A06D8C9
:102EB800124B0B449B0094401D60114B5C64002333
:102EC800C363C0E91533C0E90B33C0E90D33C365EB
:102ED80080F8253080F82430184638BD094B134453
:102EE800B3FBF1F308499B00CDE70120F5E700BFEC
:102EF80007040240F8FFFDBF000002403F820010B7
:102F080000090240F8FBFDBF0004024070B590F8CC
:102F18002450012D04463BD090F825600125AE428F
:102F280080F824504FF000062CD1022580F8255057
:102F38000568C6632E6826F001062E60FFF7DEFEE0
:102F4800036BBBB12B6843F00E032B60A36C1A68AC
:102F5800D20342BF1A6842F480721A60636D1BB1D3
:102F68001A6842F480721A602B6843F001032B60E0
:102F7800002070BD2B6823F004032B602B6843F0FE
:102F88000A03E2E78023C36380F824602846F0E759
:102F98000220EEE70A4A536943F4802330B55361AF
:102FA800EFF3108472B60023CD58C5500433B3F53F
:102FB800807FF9D11369DB03FCD484F3108830BD1A
:102FC80000400058064B5A69002ABFBF054A9A605C
:102FD80002F188329A60BABF5869C00F0020704762
:102FE8000040005823016745044B5A6942F00042EB
:102FF8005A615869C043C00F704700BF004000586D
:1030080070B50546FEF72CFC124E04463369D90309
:1030180013D43369DA0744BF012232614CF2FA3221
:10302800134011D10B4E306910F480200BD0FEF7FD
:1030380017FC001BA842F6D304E0FEF711FC001BA6
:10304800A842E3D3032070BD024A1361024A01205B
:103058005360F8E700400058580400202DE9F0417B
:10306800184D98462B78012B06460C46174626D055
:1030780001232B704FF47A7000236B60FFF7C0FFB9
:10308800A0B9012E16D1104A536943F001035361C8
:103098002760BFF36F8FC4F804804FF47A70FFF78E
:1030A800AFFF094A536923EA0603536100232B70D3
:1030B800BDE8F08139462046FFF76CFFEDE70220B6
:1030C800F6E700BF5804002000400058054A53693D
:1030D80023F47E7343EAC00040F4803040F00200DD
:1030E80050617047004000582DE9F041234F3B786C
:1030F800012B054688463FD001233B704FF47A7078
:1031080000237B60FFF77CFF044688B92B68042BFB
:1031180013D11B4A536943F4803343F004035361CA
:103128004FF47A70FFF76CFF0446154B1A681B685A
:1031380000233B702046BDE8F0814FF0FF33C8F80C
:1031480000306E68D5E901321344B3420AD93046DB
:10315800FFF7BCFF4FF47A70FFF752FF50B1C8F881
:1031680000600446064A536923F47E7323F0020381
:103178005361DAE70136E5E70224DBE7580400206B
:10318800004000582DE9F04F524C00234FF00F0932
:103198000A6832FA03F501D1BDE8F08F012505FA76
:1031A80003F818EA020200F08E804E68032706F042
:1031B80003054FEA430E07FA0EFC6F1E012F6FEA54
:1031C8000C0C32D8876807EA0C0ACF6807FA0EF7A2
:1031D80047EA0A078760476827EA0808C6F300171E
:1031E8009F4047EA08074760C76807EA0C088F68E6
:1031F80007FA0EF747EA0807022DC76017D14FEA0A
:10320800D30800EB880803F0070AD8F820704FEAC3
:103218008A0A09FA0AFB27EA0B0B0F6907FA0AF769
:1032280047EA0B07C8F8207001E0032DDCD10768D6
:1032380005FA0EF507EA0C073D4316F4403F056012
:1032480041D023F0030707F1804707F5803703F0E3
:10325800030CBD684FEA8C0C4FF0070E0EFA0CFEFB
:10326800B0F1904F25EA0E0E2FD01B4DA8422ED05C
:1032780005F58065A84214BF0725022505FA0CF557
:1032880045EA0E05BD602568D74316F4801F0CBFBC
:103298003D4015432560656816F4001F0CBF3D408E
:1032A80015436560D4F8805016F4803F0CBF3D404C
:1032B8001543C4F88050D4F88450B60354BF3D4039
:1032C8001543C4F88450013362E70025D6E7012589
:1032D800D4E700BF0008005800040048374A2DE929
:1032E800F04F00234FF0010A4FF0070B4FF00F0982
:1032F80031FA03F401D1BDE8F08F0AFA03FC1CEAA5
:10330800010654D023F0030404F1804404F580340A
:1033180003F00307A568BF000BFA07F8B0F1904F58
:1033280008EA050E45D0264DA84244D005F580652B
:10333800A8420CBF02250725BD40754517D1D2F814
:10334800805025EA0605C2F88050D2F8845025EA54
:103358000605C2F88450156825EA06051560556803
:1033680025EA06055560A56825EA0805A5600568EB
:1033780003265C0006FA04F423FA06F6254300EB5C
:103388008606056003F00705376AAD0009FA05F5FA
:1033980027EA05073762856825EA040585604568D8
:1033A80025EA0C054560C56825EA0404C4600133B4
:1033B8009EE70025C0E70125BEE700BF00080058CA
:1033C800000400480AB1816170478162704743690F
:1033D80001EA030221EA030141EA024181617047DF
:1033E800024A136843F4807313607047000400585E
:1033F8000D4B10B55B690C4628B99A0507D500F046
:1034080027F820B110BD9B0501D400F019F8074A30
:103418001369012C23F00403136101D130BFF1E7D4
:1034280040BF20BF20BFEDE70004005800ED00E0DA
:10343800024B186800F4C060704700BF00040058D1
:10344800024A136843F4804313607047000400582D
:103458000C4A136823F4804313600B4B1B6832211A
:103468004B430A49B3FBF1F35169890500D533B9D8
:10347800536913F4007F14BF032000207047013BF9
:10348800F2E700BF000400587400002040420F001B
:103498000B4A136823F0070343F002031360094B38
:1034A8001A69012842F004021A6105D130BF1A696D
:1034B80022F004021A61704740BF20BF20BFF6E720
:1034C8000004005800ED00E04FF0B0431868C0F366
:1034D800404070474FF0B0431868C0F34000704751
:1034E8004FF0B042536823F47F4343EA002353600C
:1034F80070474FF0B0431868C0F340607047000051
:103508007FB54FF0B0432C4AD3F80831C0F303100D
:1035180003F00F0352F82040284A52F82330B4FB36
:10352800F3F4FFF785FF264B054693E80700B5F54A
:10353800007F04AB03E9070010D0224B9C4218D34C
:1035480003F5B70303F67F539C4229D903F5741397
:1035580003F510639C4225D802230BE01A4B9C42CA
:1035680007D91A4B9C421BD903F5370303F5D853E7
:10357800F0E7002304AA02EB830353F80C4C144D24
:103588002B6823F0070323432B60FEF769F90646EF
:103598002B6803F007039C4206D1002004B070BDDD
:1035A8000123E7E70024EAE7FEF75AF9801B02281F
:1035B800EED90320F2E700BF78EB0008D8EB00084B
:1035C80090EA0008C0CF6A00BFEA21013F933402A5
:1035D800004000584FF0B04310B59A68D96812F00F
:1035E8000C0205D00C2A4AD101F00303012B51D15A
:1035F8004FF0B0412B480B6813F0080306D00B6856
:1036080013F0080337D1D1F8941007E00C682407A9
:1036180056BFD1F894300968C3F3032350F8233018
:10362800002A0CBF184600204FF0B0418A6802F00B
:103638000C020C2A1ED1CA6802F00302022A2ED0FC
:10364800032A06D10B68184A13F4801F174B18BFBA
:1036580013464FF0B042D068D168D268C0F3062054
:103668005843C1F302130133B0FBF3F0530F013396
:10367800B0FBF3F010BD0B68C3F30313CEE7042AC5
:1036880005D0082A06D11B6813F4801305D0064814
:103698000023C9E700231846C6E70448C4E7024BDD
:1036A800D7E700BF78EB00080024F4000048E801E1
:1036B80008B5FFF78FFF4FF0B043044A9B68C3F388
:1036C800031352F82330B0FBF3F008BDD8EB000821
:1036D8002DE9F0410446002853D04FF0B0439D68CF
:1036E800DE6803689B0605F00C0506F0030668D53E
:1036F800026A1DB10C2D46D1012E44D1002A40D0BA
:103708004FF0B043A16A1A68170756BFD3F8943030
:103718001B681B0903F0F00399421FD90846FFF7FD
:10372800EFFE00282DD14FF0B042136843F0080394
:1037380013601368A16A23F0F0030B431360606AF7
:10374800FFF7CEFEFFF7B4FFAB4B1860AB4B186822
:10375800FEF784F8002834D0BDE8F0814FF0B0427D
:10376800136843F008031360136823F0F0030B4356
:103778001360606AFFF7B4FE0846FFF7C1FE002831
:10378800E0D00120E8E74FF0B043002A54D01A688F
:1037980042F001021A60FEF763F80746FFF79AFE47
:1037A800002842D04FF0B042136843F0080313607A
:1037B8001368A16A23F0F0030B431360606AFFF7F4
:1037C8008FFE2368D80748D42368990700F18C80B6
:1037D80023681E0740F1FA80A3694FF0B046002B1A
:1037E80000F0E180D6F89430E16903F010029142CC
:1037F80000F0C48003F00302022AC2D0D80740F1C7
:10380800B380D6F8943023F00103C6F89430FEF75D
:1038180027F80746D6F89430990740F1A580FEF7B7
:103828001FF8C31B112BF5D904E0FEF719F8C01BCC
:103838000228B3D903208FE71A6822F001021A6020
:10384800FEF70EF80746FFF745FE0028B9D0FEF749
:1038580007F8C01B0228F6D9ECE7082D03D00C2D79
:1038680005D1032E03D16368002BADD189E74FF052
:10387800B043A1681A6822F480120A431A60626889
:10388800B2F5803F10D11A6842F480321A60FDF711
:10389800E7FF0746FFF718FE002895D1FDF7E0FF80
:1038A800C01B6428F6D9C5E7B2F5041F04D11A680D
:1038B80042F400121A60E6E7196821F480311960B1
:1038C800196821F400111960002AE0D1FDF7C8FF3A
:1038D8000746FFF7F9FD00283FF476AFFDF7C0FF74
:1038E800C01B6428F5D9A5E7042D236903D00C2D46
:1038F8000ED1022E0CD1002B3FF443AF4FF0B04253
:103908006169536823F0FE4343EA016353605FE74C
:103918004FF0B046BBB1336843F480733360FDF7B2
:103928009FFF074633685A0505D4FDF799FFC31B67
:10393800022BF7D97EE77368626923F0FE4343EAF6
:103948000263736044E7336823F480733360FDF7E0
:1039580087FF074633685B057FF53AAFFDF780FFC1
:10396800C31B022BF6D965E74FF0B042E169D2F8E4
:10397800943023F010030B43C2F894304FF0B04753
:10398800D7F8943043F00103C7F89430FDF768FF87
:103998000646D7F894309A0718D4FDF761FF831BC1
:1039A800112BF6D946E7D6F8943023F00103C6F870
:1039B8009430FDF755FF0746D6F894309B0705D598
:1039C800FDF74EFFC31B112BF6D933E723685807C1
:1039D80054D50B4F3B68D90514D4FFF701FDFDF70B
:1039E8003FFF06463B68DA050CD4FDF739FF831B19
:1039F800022BF7D91EE700BF7400002078000020D2
:103A080000040058E3684FF0B046002B58D023F06C
:103A18008003052B02BFD6F8903043F00403C6F8A4
:103A280090304FF0B046FDF71BFFD6F8903043F0CA
:103A380001030746C6F8903041F28838D6F890302E
:103A48009B0705D4FDF70CFFC31B4345F6D9F1E6E8
:103A5800E36823F00403812B1BD1FDF701FFD6F89F
:103A6800903043F08003C6F8903007464FF0B046D8
:103A780041F28838D6F89030180504D5E36A002B4F
:103A88004AD1002068E6FDF7EBFEC01B4045F1D99E
:103A9800D0E6FDF7E5FED6F8903023F08003C6F8AF
:103AA800903007464FF0B04641F28838D6F890304B
:103AB8001905E3D5FDF7D4FEC01B4045F6D9B9E694
:103AC800FDF7CEFED6F8903023F080030746C6F8FF
:103AD800903041F28838D6F890301A0516D4FDF7A0
:103AE800BFFED6F8903023F00103C6F890300746A1
:103AF8004FF0B04841F28836D8F890309B07BDD5D2
:103B0800FDF7AEFEC31BB342F6D993E6FDF7A8FE58
:103B1800C01B4045DFD98DE60C2D4ED0022B4FF04F
:103B2800B0431A6822F080721A6033D1FDF798FE0C
:103B38000546FFF7DEFC38BBD4E90C314FF0B04244
:103B48000B43D0682D4901400B43E16B0B43216CBB
:103B58000B43616C0B43A16B43EA0123D3601368E9
:103B680043F080731360D36843F08053D360FDF74C
:103B780077FE0446FFF7BDFC002882D1FDF770FEF2
:103B8800001B0A28F6D955E6FDF76AFE401B0A28ED
:103B9800CFD94FE6FDF764FE0446FFF7AAFC30B91B
:103BA8004FF0B042164BD1680B40D36069E7FDF780
:103BB80057FE001B0A28F0D93CE6012B3FF4E1AD83
:103BC8004FF0B043D868236B00F003029A427FF4A9
:103BD800D8AD626B00F0700393427FF4D2ADA26B54
:103BE80000F4FE43B3EB022F7FF4CBAD636C00F01F
:103BF8006040C01A18BF0120AEE500BF8C80C1111B
:103C0800FCFFFEEE2DE9F0410D46044610B90120F7
:103C1800BDE8F081684E336803F007038B4216D382
:103C280023689A0727D54FF0B047A268BB6823F0EE
:103C3800F0031343BB60FDF713FE0646BB68DB03C6
:103C480019D4FDF70DFE831B022BF7D911E0336859
:103C580023F007030B433360FDF702FE0746336882
:103C680003F00703AB42DBD0FDF7FAFDC01B0228C7
:103C7800F5D90320CCE72368580617D54FF0B0478D
:103C88006269D7F8083123F00F0343EA1213C7F823
:103C98000831FDF7E5FD0646D7F80831D90305D404
:103CA800FDF7DEFD831B022BF6D9E2E723685A07EE
:103CB80013D54FF0B047E268BB6823F4E0631343C1
:103CC800BB60FDF7CDFD0646BB689B0305D4FDF739
:103CD800C7FD831B022BF7D9CBE72368180714D538
:103CE8004FF0B0472269BB6823F4605343EAC2032C
:103CF800BB60FDF7B5FD0646BB68590305D4FDF763
:103D0800AFFD831B022BF7D9B3E72368DA070FD47B
:103D1800294C236803F00703AB4239D8FFF7C8FCE6
:103D2800264B1860264BBDE8F0411868FDF796BD94
:103D38006268022A1DD1FFF7C7FB00283FF467AF6E
:103D48004FF0B04641F28838B36823F003031343B9
:103D5800B360FDF785FD0746B368626803F00C039E
:103D6800B3EB820FD4D0FDF77BFDC01B4045F3D9E0
:103D78007FE7032A02D1FFF7BCFBDEE712B9FFF7A2
:103D8800A9FBDAE74FF0B0431B685B05D8D43EE7E0
:103D9800236823F007032B432360FDF761FD0646E4
:103DA800236803F00703AB42B8D0FDF759FD801B29
:103DB8000228F5D95DE700BF0040005874000020D4
:103DC8007800002008B5FFF773FC4FF0B043044AB1
:103DD8009B68C3F3022352F82330D84008BD00BFC4
:103DE800B8EB000808B5FFF763FC4FF0B043044A8E
:103DF8009B68C3F3C22352F82330D84008BD00BFE4
:103E0800B8EB00084FF0B043D3F89000C0F340007F
:103E180070474FF0B0410209D1F8883002F47F2290
:103E2800000123EA020300F47F200343C1F888302D
:103E380070474FF0B041020CD1F88830120423EAE1
:103E4800020343EA0040C1F8880070470368DA03B8
:103E580070B5044639D5FFF7C3FAFDF701FD614E89
:103E680005463368DB0532D54FF0B043616BD3F8B4
:103E7800902002F4407291421DD0D3F89010D3F8EC
:103E8800902042F48032C3F89020D3F8902021F497
:103E9800407022F480328D07C3F89020C3F8900058
:103EA80009D5FDF7DDFC41F288360546FFF7AAFF84
:103EB800012840F090804FF0B042616BD2F890300A
:103EC80023F440730B43C2F89030002605E0FDF759
:103ED800C7FC401B0228C4D903262568E8070AD571
:103EE8004FF0B0416268D1F8883023EA124392B2A9
:103EF8001343C1F88830A9070AD54FF0B041A2682A
:103F0800D1F8883023EA124392B21343C1F88830BB
:103F1800AA0609D54FF0B0422169D2F8883023F4B7
:103F280040630B43C2F88830AB0502D5206AFFF71F
:103F380080FF680502D5606AFFF77BFF290502D577
:103F4800A06AFFF776FF6A0602D56069FFF761FF8E
:103F58002B0602D5A069FFF75CFFE80502D5E069EA
:103F6800FFF757FFE90610D54FF0B042E168D2F8E5
:103F7800883023F440730B43C2F88830B1F5807F52
:103F880002BFD36843F08073D3602A040ED54FF084
:103F9800B042216BD2F8883023F040430B43C2F87B
:103FA800883019B9D36843F08073D3606B0410D597
:103FB8004FF0B042E16AD2F8883023F040530B4307
:103FC800B1F1005FC2F8883003D1D36843F480337D
:103FD800D360304670BDFDF743FC401BB0427FF60E
:103FE80065AF79E70004005830B590F82C30012B04
:103FF80002464FF0020022D0174B82F82D00CA2447
:10400800012582F82C505C6253245C62B1F5807FF4
:10401800146B996914D121F488519961596C24F071
:10402800010421F0004159641463DD650A4BFF2146
:1040380059620020012382F82D3082F82C0030BD0F
:1040480021F408519961D96C24F0020421F000414F
:10405800D9641463D865E9E70028004070B50B4EB1
:10406800036B756D1D40EA07044603D50123F3650C
:10407800FDF709FDAB0704D50223F365204600F0E0
:10408800C9F9012384F82D3070BD00BF0028004015
:1040980038B50A4CE36823F02003E360FDF7E0FB42
:1040A8000546E3689B0601D5002038BDFDF7D8FB1F
:1040B800401BB0F57A7FF4D90320F6E700280040CA
:1040C800F8B5114DEC6814F0400406461AD1EB68B7
:1040D80043F08003EB60FDF7C3FB23460746EC681B
:1040E80014F0400401D1032B01D11846F8BDFDF7A7
:1040F800B7FBC01BB0F57A7F234684BF032386F83D
:104108002D30ECE70023F0E70028004038B50F4CCD
:10411800E36823F08003E360A3699B06054606D4A1
:10412800FFF7B6FF10B1032085F82D0038BDA3694D
:1041380023F02003A361FFF7ABFF10B1032085F83C
:104148002D00A36943F02003A361EFE70028004096
:1041580038B5044600284BD090F82D3003F0FF0204
:104168001BB980F82C20FDF7F5F90223214D84F8BE
:104178002D30EB68DB0636D4CA236B6253236B629F
:104188002046FFF79DFF10B1FF236B6238BDAB6976
:1041980023F08E6323F04003AB6121696368AA6949
:1041A8000B431343A2691343AB61D4E9022343EAE7
:1041B80002432B61D4E90931EA680B4322F4F8522F
:1041C8001343EB602046FFF7A1FF0028DCD1D4E9B8
:1041D8000713AA690B4322F0604213436269134331
:1041E800AB61FF236B62012384F82D300020CDE7FB
:1041F8000120CBE7002800400023092803D840EA23
:104208000310C0B270470A380133C0B2F5E70000A6
:104218002DE9F04790F82C30012B05464FF00200AD
:1042280069D0012385F82C304E4B85F82D00DE68C7
:1042380006F44076B6F5807F78D04C69087891F816
:10424800019091F802A091F82470002A55D19B6939
:1042580013F0400308BFCB70FFF7CEFF80464846F7
:10426800FFF7CAFF02465046FFF7C6FF81463846A9
:10427800FFF7C2FF0B6ACF78234343EA875343EA29
:10428800090343EA084343EA022343EA0063354A41
:10429800CA205062532050628C6A8869B4F5807FC6
:1042A800946945D124F4885494610124D465B6F501
:1042B800807F09BFCB6913640343536418BF5064FC
:1042C800284B4A681A672A6B42F001022A639A69E6
:1042D80042F488529A61244AD2F8803043F4003379
:1042E800C2F880301F4BFF225A620020012385F854
:1042F8002D3085F82C00BDE8F087B4F1803F07D059
:10430800B4F5000F04D09B6913F0400308BFCB70CD
:104318000B6ACA781C4344EA0A0444EA004343EAA5
:10432800092343EA825343EA0763B0E70023AEE771
:1043380024F4085494610224D465B6F5807F09BF3B
:10434800CB6993640343D36418BFD064054B4A68B0
:104358005A672A6B42F002022A639A6942F40852A9
:10436800B8E700BF002800400008005890F82C204B
:10437800012A03464FF0020012D00A4A83F82D00A2
:10438800CA21516253215162916941F02001916122
:10439800FF2151620020012283F82D2083F82C0090
:1043A800704700BF0028004090F82C20012A0346DF
:1043B8004FF0020019D00D4A83F82D00CA2151622E
:1043C8005321516291690A4841F080019161D0F806
:1043D800801041F48021C0F88010FF215162002034
:1043E800012283F82D2083F82C0070470028004014
:1043F80000080058064B5A6D520610B5044603D5FE
:104408004022DA65FDF742FB012384F82D3010BD08
:10441800002800407047890001F1804101F53141D1
:104428000A607047890001F1804101F5314108684F
:1044380070470000034AD2F8903043F40043C2F8B2
:104448009030704700040058034AD2F8903023F4A3
:104458000043C2F89030704700040058074B1A68B0
:1044680022F040021A6040F441704FF4B8521860CC
:104478005A601A6842F040021A60704700000158FA
:1044880037B5054600284ED0837903F0FF046BB199
:10449800032C0BD0254B4FF400629A612868FFF774
:1044A800DDFF002401232B71AC602FE000236B712A
:1044B8002846FDF7EFF81E4AD2F8903043F48053AF
:1044C800C2F89030002CE5D102234FF0B042AB7116
:1044D800D2F8943023F40043C2F89430154B1B688B
:1044E8001C214B43DB0C64214B430193019B93B983
:1044F8000124AC60FFF79EFF0C4B9A6842F40062FF
:104508009A604FF400629A61002CC7D00123AB7106
:10451800204603B030BD019B013B0193D2F8943093
:104528005B04E3D4E6E70124F2E700BF0004005887
:10453800000800587400002037B5174D2B68024654
:104548001C204343DB0C6420434314480193019B24
:1045580093B901209060114C21732B681C214B43A7
:10456800DB0C64214B430193019B6BB901209060E4
:104578000A4BDB6803B030BD019B013B01938368A4
:104588009C07E4D50020E6E7019B013B0193A36863
:10459800DB07E9D5ECE700BF7400002000000158F4
:1045A80037B5184D2B6802461C204343DB0C6420AA
:1045B800434315480193019BA3B901209060124C15
:1045C800FF2323732B681C256B43DB0C64256B438B
:1045D8000193019B73B9012090600B4BDB680B7052
:1045E80003B030BD019B013B019383689C07E2D572
:1045F8000020E4E7019B013B0193A368DB07E8D5B2
:10460800EBE700BF74000020000001580E4B0F4973
:104618001B681822534382B01B0D64225343019335
:104628004B69019AC3F3800322B9022383600120F6
:1046380002B07047019A013A01924A69920701D57E
:10464800002BEDD10020F3E774000020000400588F
:1046580007B50379012B0FD10A4B1B681822534366
:104668001B0C0193FFF7F0FE019B013B0193019B9B
:10467800002BF9D1FFF7DEFE03B05DF804EBFFF77E
:10468800C5BF00BF74000020F8B51E468379012B12
:10469800154604460F46DAB22DD14379012B2AD0AC
:1046A800022342718371FFF7D3FF0D212046FFF7E4
:1046B800CBFEFFF741FF390A2046FFF73DFFF9B26D
:1046C8002046FFF739FF2E44B5420ED12046FFF7AA
:1046D800B1FEFFF79BFFA06801230038A3714FF0DC
:1046E800000318BF01206371F8BD15F8011B2046AF
:1046F800FFF722FFE8E70220F6E7F8B51E468379C0
:10470800012B154604460F46DAB22FD14379012B07
:104718002CD04271FFF79CFF1D212046FFF794FE25
:10472800FFF70AFF390A2046FFF706FFF9B22046CD
:10473800FFF702FF00212046FFF7FEFE2E44B54298
:104748000ED12046FFF776FEFFF760FFA068012331
:104758000038A3714FF0000318BF01206371F8BD42
:1047680029462046FFF71CFF0135E8E70220F6E757
:10477800F8B51F468379012B154604460E46DAB272
:104788002CD14379012B29D04271FFF761FF06F044
:10479800EF03A3F18402534253412371314620466B
:1047A800FFF752FEFFF7C8FE2F44AF4210D1FFF7C4
:1047B80041FE842E02D02046FFF728FFA06801237F
:1047C8000038A3714FF0000318BF01206371F8BDD2
:1047D80015F8011B2046FFF7AFFEE6E70220F6E7D3
:1047E800F8B51E468379012B154604460F46DAB202
:1047F80027D14379012B24D04271FFF729FF39468D
:104808002046FFF721FEFFF797FE00212046FFF71D
:1048180093FE2E44B5420ED12046FFF70BFEFFF75C
:10482800F5FEA06801230038A3714FF0000318BFFC
:1048380001206371F8BD29462046FFF7B1FE013516
:10484800E8E70220F6E737B50023ADF8043001AAFF
:10485800022312210546FFF7C3FFBDF804400223D7
:1048680064BA01AAA4B219462846FFF781FFE207F5
:1048780002D5284609F0B4F9A30702D5284609F05D
:10488800B5F9600702D5284609F0DAF9210702D5FB
:10489800284609F0DBF9E20602D5284609F0DCF9DA
:1048A800A30602D5284609F0C5F9600602D52846B0
:1048B80009F0A2F9210606D514F4807118BF012168
:1048C800284609F09FF9A20502D5284609F0AAF959
:1048D800630402D5284609F0C5F903B030BDF8B520
:1048E8001E468379012B154604460F46DAB227D1B6
:1048F8004379012B24D04271FFF7AAFE0E212046EE
:10490800FFF7A2FDFFF718FE39462046FFF714FE11
:104918002E44B5420ED12046FFF78CFDFFF776FEF8
:10492800A06801230038A3714FF0000318BF0120CD
:104938006371F8BD15F8011B2046FFF7FDFDE8E798
:104948000220F6E7F8B51E468379012B1546044682
:104958000F46DAB22BD14379012B28D04271FFF7E9
:1049680077FE1E212046FFF76FFDFFF7E5FD39466C
:104978002046FFF7E1FD00212046FFF7DDFD2E442C
:10498800B5420ED12046FFF755FDFFF73FFEA06860
:1049980001230038A3714FF0000318BF0120637191
:1049A800F8BD29462046FFF7FBFD0135E8E7022060
:1049B800F6E7026852E8003F23F0C00342E80031FE
:1049C80002680029F5D102F1080353E8003F23F4F7
:1049D800000302F1080C4CE800310029F3D1202330
:1049E800C0F888307047000010B5026852E8003FF0
:1049F80023F4907342E8003102680029F5D10F4C86
:104A080002F1080353E8003F234002F1080C4CE888
:104A180000310029F4D1C36E012B07D152E8003FC1
:104A280023F0100342E800310029F7D12023C0F811
:104A38008C300023C366436710BD00BFFEFFFFEF45
:104A480038B50546C8B12423C0F8883003681A6809
:104A5800002422F001021A601C605C609C60FDF773
:104A6800C1F8C5F8904085F88440C5F888402046CC
:104A7800C5F88C40EC662C6738BD0120FCE70000C7
:104A8800F8B504461346D4F88850202D32D1F1B138
:104A9800EAB1E06FA4F85620A4F854200026212299
:104AA800C4F890602165C4F88820226888B1124F44
:104AB800C762124F0763124F2832C0E90D76FEF71E
:104AC80025FA30B11023C4F89030C4F8885001207A
:104AD800F8BD236840221A62226802F1080353E8ED
:104AE800003F43F0800302F1080141E8003000284C
:104AF800F3D1EDE70220EBE70D4B0008554B00081A
:104B0800614B000808B50346806A1B681B6813F0F0
:104B1800200317D1A0F85630026802F1080353E8C1
:104B2800003F23F08003083242E800310268002980
:104B3800F2D152E8003F43F0400342E80031002937
:104B4800F7D108BDFDF7C8F8FBE7704708B5806ADC
:104B5800FFF7FBFF08BD7047806A38B50468D0F8D6
:104B68008830D0F88C50A268120606D5212B04D1C3
:104B78000023A0F85630FFF71CFFA3685B0606D594
:104B8800222D04D10023A0F85E30FFF72DFFD0F8C6
:104B9800903043F01003C0F89030FFF7DCFF38BDC9
:104BA80070470000D0F88C20B0F86010222A08B5B1
:104BB800036855D15B6A826D0B401370836D0133B6
:104BC8008365B0F85E30013B9BB2A0F85E30B0F868
:104BD8005E309BB2002B42D1026852E8003F23F4BA
:104BE800907342E8003103680029F5D103F1080207
:104BF80052E8002F22F0010203F1080C4CE80021D2
:104C08000029F3D12022C0F88C20184A416793422A
:104C1800016705D1C26E012A0ED0FDF76BF81EE0C0
:104C28005A681102F6D553E8002F22F0806243E853
:104C380000210029F7D1EDE70022C26653E8002FD2
:104C480022F0100243E800210029F7D1DA69B0F810
:104C58005C10D20644BF10221A62FFF7A1FF08BDFC
:104C68009A6942F008029A61F9E700BF00800040A3
:104C7800D0F88C20B0F86010222A08B5036852D109
:104C88005A6A1140826D22F8021B8265B0F85E20D4
:104C9800013A92B2A0F85E20B0F85E2092B2002AE3
:104CA80040D153E8002F22F4907243E800210029F4
:104CB800F7D103F1080252E8002F22F0010203F1B4
:104CC800080C4CE800210029F3D12022C0F88C20E0
:104CD800174A41679342016705D1C26E012A0ED077
:104CE800FDF708F81EE05A681102F6D553E8002FC0
:104CF80022F0806243E800210029F7D1EDE7002285
:104D0800C26653E8002F22F0100243E80021002970
:104D1800F7D1DA69B0F85C10D20644BF10221A62E3
:104D2800FFF73EFF08BD9A6942F008029A61F9E769
:104D3800008000402DE9F84F0368B0F86060D3F8B0
:104D48001CB01F689D68D0F88C20222A044640F0C9
:104D5800B980B0F8683043B1DFF87491DFF874A116
:104D68004FF000081BF0200F20D1B4F85E309BB242
:104D7800D3B1B4F868209A4216D9226802F1080320
:104D880053E8003F23F08053083242E8003122689C
:104D98000029F2D1504B636752E8003F43F02003EB
:104DA80042E800310029F7D1BDE8F88F2368A26DE9
:104DB8005B6A33401370A36D0133A365B4F85E30AA
:104DC800013B9BB2A4F85E302368D3F81CB01BF0FB
:104DD800070F2ED01BF0010F09D0F90507D50122C6
:104DE8001A62D4F8902042F00102C4F890201BF017
:104DF800020F09D0EA0707D502221A62D4F89020D8
:104E080042F00402C4F890201BF0040F09D0E80710
:104E180007D504221A62D4F8903043F00203C4F88C
:104E28009030D4F8903023B12046FFF794FEC4F8B0
:104E38009080B4F85E309BB2002B93D1226852E880
:104E4800003F23F4807342E8003123680029F5D13C
:104E580003F1080252E8002F02EA090203F10800F0
:104E680040E800210029F3D120225345C4F88C20C2
:104E7800616721670AD05A68110207D553E8002FE5
:104E880022F0806243E800210029F7D1E26E012A6E
:104E980014D10022E26653E8002F22F0100243E802
:104EA80000210029F7D1DA69B4F85C10D20644BFB2
:104EB80010221A622046FFF773FE53E72046FCF7DC
:104EC80019FF4FE79A6942F008029A616CE700BF40
:104ED800FEFFFFEF00800040AD4B00082DE9F84FC2
:104EE8000368B0F86060D3F81CB01F689D68D0F8FC
:104EF8008C20222A044640F0B780B0F8683043B1CD
:104F0800DFF87091DFF870A14FF000081BF0200F58
:104F180020D1B4F85E309BB2D3B1B4F868209A427D
:104F280016D9226802F1080353E8003F23F08053A2
:104F3800083242E8003122680029F2D14F4B6367FA
:104F480052E8003F43F0200342E800310029F7D13E
:104F5800BDE8F88F2368A26D596A314022F8021B18
:104F6800A265B4F85E20013A92B2A4F85E20D3F8A4
:104F78001CB01BF0070F2ED01BF0010F09D0F9054C
:104F880007D501221A62D4F8902042F00102C4F831
:104F980090201BF0020F09D0EA0707D502221A62F7
:104FA800D4F8902042F00402C4F890201BF0040FBB
:104FB80009D0E80707D504221A62D4F8903043F0E4
:104FC8000203C4F89030D4F8903023B12046FFF79C
:104FD800C2FDC4F89080B4F85E309BB2002B95D126
:104FE800226852E8003F23F4807342E800312368C6
:104FF8000029F5D103F1080252E8002F02EA09025C
:1050080003F1080040E800210029F3D1202253458C
:10501800C4F88C20616721670AD05A68110207D545
:1050280053E8002F22F0806243E800210029F7D1DD
:10503800E26E012A14D10022E26653E8002F22F022
:10504800100243E800210029F7D1DA69B4F85C10AE
:10505800D20644BF10221A622046FFF7A1FD55E789
:105068002046FCF747FE51E79A6942F008029A6128
:105078006EE700BFFEFFFFEF00800040794C00089C
:1050880038B5044603682169A2681D68C0690A43E7
:1050980061690A437749024329400A431A605A68FA
:1050A800E16822F440520A435A60734AA169934264
:1050B8001CBF226A11439A6822F06E4222F43062C1
:1050C8000A439A60DA6A616A22F00F020A43DA62D6
:1050D8006A4A934219D14FF0B043694AD3F88830ED
:1050E80003F0030343F44033934200F0B480B3F178
:1050F800031F24D0013A934240F0B580B0F5004F29
:1051080040F08F80FEF766FA6EE05E4A93421CD14B
:105118004FF0B0435C49D3F8883003F00C0343F4F4
:1051280040228A4200F0978006D8002B7CD0574B4B
:105138009A42E3D0012026E0B2F10C1FFAD1B0F573
:10514800004F53D04FF4004075E04B4A9342F1D1E1
:105158004FF0B043D3F8883003F44063B3F5006FE1
:1051680018D006D85BB1B3F5806FE3D1FEF732FAF9
:1051780007E0B3F5406FDDD14FF400400BE0FEF7D8
:1051880021FE40B900204FF00113A3660023C4E9B3
:105198001D3338BD3E4865683E4B626A05EB4501E4
:1051A80033F81220B0FBF2F39942C3D8B3EB053FB2
:1051B800C0D800231946FBF7F3FC090241EA106145
:1051C8006B080002C0182A464FF0000341F10001A5
:1051D800FBF7E6FC304BA0F540729A42AAD8236848
:1051E800D860CFE7FEF7EEFD0028CBD06168294BE9
:1051F800626A33F81220B0FBF2F24B0803EB420369
:105208004FF6EF72B3FBF1F3A3F11001914291D87D
:1052180023F00F02216892B2C3F342031343CB6019
:10522800B0E7FEF7D7F904E0B0F5004FDAD0FEF7A3
:10523800C9FD0028A6D06368616A164A32F81120B1
:10524800B0FBF2F000EB5300B0FBF3F04FF6EF7356
:10525800A0F11002C1E7B0F5004F0D48EBD1C5E74A
:10526800FEF7C0FDC0E7B0F5004FF9D0FEF7BAFD74
:10527800DFE700BFF369FFCF00800040003801403E
:10528800020003000044004008000C0004000C0069
:105298000024F40018EC0008FFFC0F00836ADA070A
:1052A80010B506D50168C46A4A6822F40032224360
:1052B8004A609C0706D50168046B4A6822F480326C
:1052C80022434A60590706D50168446B4A6822F4AC
:1052D800802222434A601A0706D50168846B4A680F
:1052E80022F4004222434A60DC0606D50168C46BFA
:1052F8008A6822F4805222438A60990606D501689A
:10530800046C8A6822F4005222438A605A060FD538
:105318000168446C4A6822F480122243B4F5801F65
:105328004A6005D14A68846C22F4C00222434A606C
:105338001B0606D50268C16C536823F400230B438F
:10534800536010BD2DE9F843DDF8209005460F465F
:10535800164698462A68D36937EA03030CBF012327
:105368000023B34201D0002029E0B9F1FF3FF2D079
:10537800FCF776FAA0EB080048452C6802D8B9F18A
:10538800000F1ED154E8003F23F4D07344E80032E4
:10539800002AF7D104F1080353E8003F23F0010382
:1053A80004F1080141E80032002AF3D12023C5F8AE
:1053B8008830C5F88C30002385F884300320BDE898
:1053C800F88323685A07C5D5E3691B05C2D54FF48E
:1053D8000063236254E8003F23F4D07344E80032AA
:1053E800002AF7D104F1080353E8003F23F0010332
:1053F80004F1080141E80032002AF3D12023C5F85E
:105408008830C5F88C30C5F89030D4E773B50446B9
:105418000026C0F89060FCF723FA23681B681A0777
:10542800054619D423681B685B070AD56FF07E43CD
:10543800009300222B464FF480012046FFF782FF9D
:10544800B0B900202023C4F8883084F88400C4F858
:105458008C30E06620670CE06FF07E4300933246A4
:1054680003464FF400112046FFF76CFF0028D9D0FF
:10547800032002B070BD10B5044650B3D0F8883090
:105488001BB980F88430FCF73DFB22682423C4F85C
:105498008830136823F0010313602046FFF7F0FDFE
:1054A800012816D0A36A13B12046FFF7F7FE236838
:1054B8005A6822F490425A609A6822F02A029A6046
:1054C8001A6842F0010220461A60BDE81040FFF752
:1054D8009DBF012010BD000030B581658168A0F82E
:1054E8005C200023B1F5805FA0F85E20436735D1CA
:1054F8000369002B40F2FF1318BFFF23A0F86030A8
:105508000023C0F890302223C0F88C30016801F1E4
:10551800080353E8003F43F00103083141E8003431
:105528000368002CF2D1456E84680169B5F1005F0B
:1055380032D1B0F8685095422ED8B4F5805F244A2D
:1055480003D1244C002908BF22464267B1B153E871
:10555800002F42F4807243E80021F7E729B9036974
:10556800002B14BF7F23FF23C8E7B1F1805FC5D1AB
:105578000369002B14BF3F237F23BFE703F1080211
:1055880052E8002F42F0805203F1080040E8002161
:105598000029F3D1002030BDB4F5805F0E4A03D155
:1055A8000E4C002908BF2246426741B153E8002F3C
:1055B80042F4907243E800210029F7D1EAE753E862
:1055C800002F42F0200243E800210029F7D1E1E74B
:1055D8003D4D0008E54E0008AD4B0008794C000829
:1055E800D0F88C30202B30B415D1B9B1B2B100232A
:1055F8000468C3660A4B9C420AD063681B0207D53D
:1056080054E8003F43F0806344E80035002DF7D1AB
:1056180030BCFFF761BF022030BC70470120FBE7B8
:1056280000800040436E30B52BB90123A0F86A30E2
:10563800A0F8683030BD0368094D9A689968094C2C
:10564800490FC2F342626B5C615CDB00B3FBF1F3B0
:10565800A0F86A30AB5CA25CDB00B3FBF2F3E7E7CF
:1056680038EC000830EC00081FB504AB03E906006D
:1056780090F88430012B04463AD0012380F8843016
:105688002423C0F8883003681A6822F001021A60DF
:105698009A6822F440120A439A6071B95A68BDF8B0
:1056A8000C009DF80E1022F0100202435A605A684E
:1056B80022F07F4242EA01625A601A6842F001020F
:1056C8001A60FCF7CDF86FF07E42034600924FF463
:1056D800800100222046FFF735FE38B92023C4F8A0
:1056E8008830002384F8843004B010BD0320F8E724
:1056F8000220F9E790F88430012B0FD0012380F8BD
:105708008430016851E8002F42F0020241E800238A
:10571800002BF6D180F88430184670470220704775
:1057280010B590F88430012B044617D02423C0F814
:10573800883003681A68196821F00101196042F07D
:1057480000524FF0005141661A60FFF76BFF2023AB
:10575800C0F88830002084F8840010BD0220FCE7DF
:1057680070B590F88430012B044617D005682423BF
:10577800C0F888302E682B6823F001032B60AB68D3
:1057880023F060431943A960FFF74CFF20232E60E4
:10579800C0F88830002084F8840070BD0220FCE73F
:1057A80038B5084D052455F8043B2BB9013C14F0D5
:1057B800FF04F8D1204638BDDB6898470028F5D0AB
:1057C800F9E700BFAC050020034BD870034B1B68FA
:1057D8001B6C03B118477047940500209005002002
:1057E800034B1874034B1B685B6C03B11847704775
:1057F8009405002090050020F0B5314D314B95F906
:105808000420314E91B00C46012795F905108DF80A
:10581800047002288DF809208DF80A1010D18DF82F
:105828000800D8711C7202F063FD337803B114B11B
:1058380001A803F0C1F9254B059A1A6011B0F0BD13
:1058480059714FF480711A71D9801C7233788DF8B0
:10585800087053BB1F2306A88DF81C208DF818303C
:1058680002F024FF20238DF8183006A82B798DF834
:105878001C3002F01BFF22238DF8183006A86B7924
:105888008DF81C3002F012FF21238DF8183006A87D
:105898006B798DF81C3002F009FF29238DF8183038
:1058A80006A80B4B079302F001FF02F021FD01232C
:1058B80006A88DF818308DF81C3002F0F7FEB4E712
:1058C80094050020AC00002070040020640500202E
:1058D800000400017FB5092301A88DF8043003F006
:1058E8006BF90038044B059A1A6018BF0120404232
:1058F80007B05DF804FB00BF6405002070B50446DE
:105908000B46144962784A700020A2780A7208701F
:105918001A884A729A788A72DB780B746368CB604B
:105928000D4B1B68DA6A2AB1237803F0FB030A2BB4
:1059380000D09047094E002556F8043B1BB15B6A1E
:105948000BB1204698470135EBB2052B6DB2F3D168
:1059580070BD00BF7C00002090050020AC05002031
:1059680070B5044611480123037063784370A37827
:105978008372E368C360E378037623694376237907
:1059880043720B4B1B689B6A03B19847094E00256D
:1059980056F8043B1BB19B690BB12046984701356B
:1059A800EBB2052B6DB2F3D170BD00BF90000020A3
:1059B80090050020AC050020014B1868704700BF17
:1059C8006405002000B58BB0012368468DF80030CF
:1059D80002F046FD38B99DF80400003818BF0120D0
:1059E8000BB05DF804FB0020FAE7000008B501F0F1
:1059F80037FE40B9FFF7E6FF012806D0054B197AB4
:105A0800D879FFF7F9FE012008BDBDE80840FFF787
:105A1800C7BE00BFAC0000202DE9F04186B00546A6
:105A28000E46174601F01CFE002873D101F030FE27
:105A3800044640B9FFF7C6FF01280AD03D4B197A42
:105A4800D879FFF7D9FE6FF00204204606B0BDE80A
:105A5800F081DFF8E48088F80860003E18BF01266E
:105A68008DF80460354E687833798DF812306946C0
:105A780002F094FC00283FD08DF804400394ADF860
:105A880010406FF0060495E803002D4B83E80300EF
:105A9800337988F80A30394601A803F091F9294B7F
:105AA800059A1A6011283FD801A353F820F000BFC7
:105AB800235B00081D5B0008315B0008315B0008B0
:105AC800315B0008315B0008315B00084F5A000861
:105AD800315B0008315B0008315B0008175B000888
:105AE800315B0008315B00081D5B00081D5B000886
:105AF8001D5B0008375B00082B788DF808306B7841
:105B0800ADF810306B6803934FF0FF34BBE76FF0CC
:105B180005049AE76FF0010497E70B4B00221A700F
:105B2800E31D18BF144690E74FF0FF348DE76FF080
:105B380004048AE7AC0000209000002094050020AF
:105B4800A0000020640500206305002037B501F09F
:105B5800A9FD134D052455F8043B4BB11A693AB118
:105B68009B682BB1984718B155F8043C1B699847B6
:105B7800013C14F0FF04EED1FFF712FE68B9094D9D
:105B88002B7853B1084BADF80040D97801942246E0
:105B98006846FFF741FF00B92C7003B030BD00BF65
:105BA800AC050020630500209405002030B58BB0BB
:105BB800044601F055FD0546002835D1FFF702FFE0
:105BC800012834D168468DF8005002F049FC40BBEA
:105BD8009DF80430A34204D0012C22D0022C12D00C
:105BE80014B100200BB030BD002BFAD068468DF8F8
:105BF800044002F05BFDA0B90E4B1B681B6B002B29
:105C0800EFD09847EDE763B968468DF8044002F095
:105C18004DFD30B9074B1B681B6B002BE1D02046AC
:105C2800EFE74FF0FF30DDE76FF00100DAE76FF0E4
:105C38000200D7E79005002010B504468AB018B9CD
:105C48004FF0FF300AB010BD002368468DF80030D1
:105C580002F006FC0028F3D19DF804302370F1E728
:105C68007FB500220B4620498DF8072001220A70D3
:105C780042784A700446002A33D102790A721A8897
:105C88004A729A788A72DB780B740369CB60C3789E
:105C9800164D8DF80830037B8DF80930836803931F
:105CA8002B68DB6A0BB102A898472B689B6B13B172
:105CB800227E02B198470E4E052556F8043B1BB1CB
:105CC800DB690BB120469847013D15F0FF05F4D17B
:105CD8000DF10700FFF7B0FF637913B1054B0122FF
:105CE8001A7004B070BD00BF7C0000209005002031
:105CF800AC0500206305002010B504468AB018B929
:105D08004FF0FF300AB010BD202368468DF80030F0
:105D180002F0A6FB0028F3D1024A9DF90430237053
:105D28001371EFE79405002000B58BB02323019091
:105D380068468DF8003002F0B9FC003818BF012021
:105D480040420BB05DF804FB70B5654C01468EB05F
:105D58001822204606F0C0F8624B00221A70FCF7A1
:105D680073FA23784068012202FA03F1014004D152
:105D78005D4B084608F09CF8FEE75C495C481A460B
:105D880002F0F8F818B14FF0FF300EB070BD2723BD
:105D980004A88DF8103002F089FC564E564D0028A4
:105DA80070D1012333702B68DB690BB10020984751
:105DB800272304A88DF8103002F052FB059B93F8B6
:105DC8004820227093F8182193F81A316270A37052
:105DD800464BD3E9020105F06FFF05460028D2D1F2
:105DE800464E062304A88DF8103002F039FB059BB7
:105DF800736104A802F05AFC022304A88DF810303D
:105E0800059602F02DFB0836032304A88DF8103000
:105E1800059602F025FB0F2606F014F8012304A8C6
:105E28008DF814308DF8106002F040FC10230DEB53
:105E380003008DF810308DF8145002F037FC04235D
:105E48008DF8103004A8A3788DF8143002F02EFCD9
:105E58003A238DF8103004A86369059302F026FCF4
:105E680002A920788DF8086004F09CF8003818BF63
:105E78000120E0711420FFF757FFE07903F062F981
:105E8800284682E728238DF810302B681B6943B118
:105E980004A802F0E5FA2B6805981B6940F2C45182
:105EA8009847272304A88DF8103002F0FFFB50B95B
:105EB800012304A88DF8103002F0D2FA9DF81430AE
:105EC800002B7FF46EAF3378002B7FF46CAF052284
:105ED80004A88DF81020059302F0E8FB78E700BFCE
:105EE800940500206305002040EC000868050020A8
:105EF800800500207004002090050020D0050020B7
:105F080037B500230D4601930446D0B900F0A8FB2D
:105F18000190019BD3B10F4A42F824300E4A9A628D
:105F28000E4A1268916B1963916C596392690C4916
:105F3800D9625A6128465B680A49F22298470020CC
:105F480006E001A900F092FB0028E2D04FF0FF30F4
:105F580003B030BDAC0500200158000890050020B2
:105F6800DD58000871040020194B07B51860194B5B
:105F7800194A1A60194A5A60194A9A60194ADA6025
:105F8800194B02681A6042685A6082689A60C2684F
:105F9800DA60164A1A6182695A61154BC26B5A60F7
:105FA800144A019119609A601946134ADA60002070
:105FB800FFF7A6FF48B901A800F056FB003818BF44
:105FC8000120404203B05DF804FB4FF0FF30F9E7D1
:105FD800900500208005002069590008695C0008C8
:105FE8007D60000805590008680500205D9F0008CD
:105FF800C0050020D1570008E957000849B118B179
:10600800012804D000207047034B0B60FAE7034BCC
:10601800FBE74FF0FF307047000400010100010268
:1060280008B503F0ABF8002814BF6FF0010000209A
:1060380008BD08B502F084F9002814BF6FF001000C
:10604800002008BD10B504468AB018B94FF0FF30DB
:106058000AB010BD212368468DF8003002F000FA1E
:106068000028F3D1024A9DF9043023705371EFE7F9
:10607800940500202DE9F0412F4D304F00232B705F
:1060880043786B703B689B6A8AB004460BB128461C
:106098009847DFF8AC80002658F8043B1BB11B6A10
:1060A8000BB1204698470136F3B2052B76B2F3D1EF
:1060B8002378052B2FD00B2B35D0012B25D1214C44
:1060C800062368468DF8003002F0CAF90199E07994
:1060D80005F038FE10B91C4B019A5A611B48FFF7AE
:1060E8000BFE1B48FFF7AEFF6B788BB9A371194BFA
:1060F8005878FFF75BFD3B685B6A0BB1114898471E
:106108006B7813B9E07905F0AFFE0AB0BDE8F0810D
:10611800FF23A371EFE7104B01225A74227A9A7475
:10612800627ADA74F1E76378002BEED00AB0BDE842
:10613800F041FFF7CFBB00BF900000209005002082
:10614800AC050020AC000020D0050020B0000020E5
:10615800B1000020940500207C00002030B58BB0F1
:10616800FFF767FF0446F0B903F0FCFE831C1DD05F
:10617800F8B9134D2B685B69DBB1272368468DF8A6
:10618800003002F06DF92B6801985B694FF4B96132
:10619800984703F0F9FE78B92CB9094B1B68DB69FD
:1061A8000BB10120984720460BB030BD6FF00704B3
:1061B800EFE74FF0FF34ECE74FF0FF34F3E700BFB1
:1061C80090050020014B1878704700BF0406002096
:1061D800014B5878704700BF040600207047000044
:1061E800044B9A7A0AB101225A70034B5B6903B1D6
:1061F8001847704704060020B800002073B5224CE9
:106208006378002B33D008F03BF966680546FFF742
:10621800D3FB0644AE4214D2A37A93B1E0228DF8A0
:1062280000208DF80130217AE36801930122684645
:10623800FFF7F2FB08B1073010D100236370A37297
:10624800656094F83430EBB1002384F834300F4B98
:106258005B6BBBB102B0BDE87040184740F2DC513F
:106268000B4808F0D9F90A4808F09CF9E8E794F8CF
:106278003520002AE5D094F8360084F83530FFF749
:1062880095FCDEE702B070BD04060020B8000020CF
:10629800E805002037B5104D104CC8B1C1B1627285
:1062A800012300222860E16023700D480D4B009205
:1062B8004FF0FF3108F0CAF800250B48258220224C
:1062C800294605F01DFE6570A574A58603B030BD8E
:1062D80000232B602370EFE700060020040600204F
:1062E800E8050020E9610008180600202DE9F047BC
:1062F8008E4C23788CB0002B56D0C2780AB9837B99
:1063080013B1238A01332382437B002B4CD0E02A2C
:106318004AD10023A372876897F80080B8F1220F4A
:1063280027D8B8F1220F30D8DFE818F04100FB0079
:1063380052005A0061006E0075008E009D00B40086
:10634800C7002F002F002F002F002F002F002F0035
:106358002F002F002F002F002F002F002F002F00BD
:106368002F002F002F002F002F002F00C900D00072
:10637800D400B8F17E0F00F0CC80B8F17F0F00F0A8
:10638800DF80B8F17D0F00F0AB80A57A002D00F01A
:106398005B81674C637A3BB94FF47A71204608F009
:1063A8003BF9204608F0FEF80CB0BDE8F087E3683A
:1063B80001220021A2721970A37AE1689818A072CC
:1063C8000620C854A37AE1689818A072CA54DCE77A
:1063D800584B9B6A002BD8D0012102209847D4E75C
:1063E8007B7884F83630012384F83530CDE70423F0
:1063F8008DF804307B78003B18BF012301A88DF885
:10640800083002F053F9C0E77878003818BF012047
:1064180002F098FEB9E7484E0FCE01AD0FC50FCE7A
:106428000FC596E8070085E807007B780A2BACD8EB
:10643800424A12685268002AA7D00CA901EB8303CC
:1064480053F82C0C9047A0E77878431E012B9CD872
:106458003A4B01381B6818BF012020729B68002B3B
:1064680093D0984791E7E26801230821A37211703D
:10647800627A057BA17AAA4228BF2A46934284D22F
:1064880085685A1CEB5CE56801334E1CA6726B5498
:10649800D3B2EDE7E3680122A27209221A70A37A47
:1064A800E268218A581CA072D154A27A238AE16832
:1064B8001B0A501CA0728B5467E7238265E70523EB
:1064C8008DF8043001A802F077FB5EE7194BDB6A10
:1064D80098475AE7194B78781B686075DB68BEE700
:1064E800037B072B7FF451AF06238DF80430B7F8F0
:1064F8000130ADF808307B793A791B0443EA02236E
:10650800FA781343642253430393BB798DF8103010
:10651800D8E73B2201A88DF804208DF8083002F056
:10652800C5F8012384F834302FE700BF04060020A3
:10653800E8050020B80000209CEA000800060020BA
:106548002A2301A88DF8043001F08AFF94F80A90F4
:10655800E6689DF808009DF809509DF80A709DF8B6
:106568000BC09DF80D309DF80E209DF80F109DF87A
:106578000CE009F1010A84F80AA006F80980354EF2
:1065880094F80A903668D4F80C8009F1010A84F866
:106598000AA096F803A008F809A094F80A90D4F87D
:1065A8000C8009F1010A84F80AA096F802A008F8FC
:1065B80009A094F80A90D4F80C8009F1010A84F82B
:1065C8000AA096F801A008F809A094F80A9009F121
:1065D800010A84F80AA096F80080E66806F809809F
:1065E80094F80A80E66808F1010984F80A9006F828
:1065F80008C094F80AC0E6680CF1010884F80A801B
:1066080006F80C70A77AE66807F1010C84F80AC04E
:10661800F555A57AE6686F1CA7727055A07AE568EB
:10662800461CA6722954A17AE0684D1CA5724254F2
:10663800A27AE168501CA0728B54A37AE268591CB4
:10664800A17202F803E0A0E6034807F05DFF657059
:10665800AAE600BF00060020E805002070470000F9
:1066680000487047B8000020002070474FF0FF3006
:1066780070470000044B054A93F81831022B18BFE5
:10668800062382F890347047A80C00206C12002072
:10669800034BD3F8483313B15B6903B1184770470C
:1066A8006C120020034A137843F004031370FFF7B9
:1066B800EFBF00BF500600201FB50A4B8DF8090038
:1066C80093F87C208DF80A2093F88C2093F84800E2
:1066D8000D3202A98DF8082003F064FCC0B205B0A1
:1066E8005DF804FBA80C002008B5074807F00CFF6C
:1066F800064B93F81A2412B1012283F81924BDE835
:106708000840FFF7C5BF00BF6C1600206C120020C0
:1067180010B50C4CD4F8403343F08003C4F8403330
:1067280094F81A3413B10020FFF7DEFF94F891347F
:1067380023F0120343F0120384F89134BDE81040AB
:10674800FFF798BF6C1200202DE9F041DFF8AC800C
:1067580098F81831022B06460D4602D0284BDB6A02
:10676800984702F0A6FD044628B1022002F097FDE2
:10677800002002F099FD98F81831012B17D102F08A
:106788009AFD074630B1002002F08AFD002002F091
:106798008CFD3C4602F091FD48B1002002F081FDDD
:1067A800002002F083FDBDE8F041FFF763BF002C35
:1067B800F9D1144C94F8902494F81A34BAB90BB15E
:1067C80084F84164304602F017FFD8F82C0007F02F
:1067D80061FED4F8B4339842E5D30B4807F094FE31
:1067E80094F8913443F0100384F89134DBE70BB14B
:1067F80084F84154284602F0FFFEF1E7A80C002077
:10680800BCF300086C12002004160020074A10B5DB
:10681800137843F002031370FFF73AFFBDE8104006
:10682800034B01220021022007F042BB5006002042
:1068380089EC0008074A10B5137843F00803137071
:10684800FFF726FFBDE81040034B0122002102207C
:1068580007F02EBB5006002099EC00082DE9F04106
:106868000F4616461D46804607F00AFE0B4A0C4C9A
:106878001378278123F0110343F01103C4E90008BA
:10688800137066812573FFF703FFBDE8F041054BE0
:1068980001220021022007F00BBB00BF5006002098
:1068A8003C060020A9EC000813B507F0E9FD0D4BE4
:1068B8006C461860204607F037FD94E803000A4A42
:1068C8000A4B83E80300137843F020031370FFF7A3
:1068D800DFFE074B01220021022002B0BDE8104074
:1068E80007F0E6BA4C06002050060020A415002048
:1068F800B6EC00082DE9F04192B0064602F0D9FC4A
:10690800002840F05881AD4D95F81831012B09D079
:106918002B6BAB4C93B194F80431BBB1042B6FD003
:10692800032003E002F0C7FC18B10F2012B0BDE845
:10693800F08102F0C2FC0028EAD0F6E7B5F8203171
:10694800D4F81C24013B53432B63E4E79D4803F030
:1069580060FA002840F0128194F80C3123802B6BE8
:106968000C930DF1180895F839308DF838304046F9
:1069780095F81C318DF83A3007F0FCFCD5F8283131
:10698800009302AF98E80600D5F82431384607F09E
:1069980088FC97E803000FAB83E80300EB6A0D93CC
:1069A80000238DF844302388ADF8463095F830310F
:1069B80001228DF839201BB98DF844208DF8393023
:1069C800814B0093814B95F84800A3F179020CA9FB
:1069D80003F05DFBC0B10B28A8D1D4F8941499B189
:1069E800002EA3D0D4F84033794843F02003C4F8EC
:1069F800403307F011FE764807F0D4FD002095E7F4
:106A0800704803F03AFAA4E795F8487095F96930A8
:106A180095F9392095F87D106E4E384603F044FB01
:106A2800009641B2EB6C95F850203846183603F0C2
:106A3800DFFA0096EB6C95F8502095F9701095F8F0
:106A4800480003F0D5FAD4F8C413AB6DD4F8DC23AE
:106A58000B44C4F8B033EB6D1344C4F8B43394F862
:106A68000431042B07D02B6E0B44C4F8B0336B6E83
:106A78001344C4F8B4330023089395F83031002B3D
:106A880040D100238DF8133095F839308DF8213036
:106A980095F838308DF82230D5F880300993D5F83C
:106AA80084300A932388ADF82C3095F8303194F867
:106AB8001B648DF82E3095F84800474B8DF8206000
:106AC8000DF1130208A903F0A7FA012384F8413451
:106AD80095F8393084F842349DF8133084F84334FB
:106AE800D4F81C34C4F85064C4F84834C4F8583492
:106AF80002F0E5FBC8B1D4F81C0402F0F2FBA0B127
:106B0800102013E708A802F0A7FC60B995F939002E
:106B180094F837629DF82070FFF7CEFD3E44B042EE
:106B2800AFD2082002E7132000E795F81831012BAF
:106B380001D102F0D8FB02F0C5FB0023059394F8BD
:106B4800043195F9395094F81B649BB1042B7FF4F8
:106B5800E7AE05A802F0B4FE58BB94F8183413B198
:106B6800059B013B0593174B05983246E9B202F0A5
:106B78000DFF02E0134802F0DDFE08B11120D5E652
:106B8800D4F8403394F80C11218043F00203C4F880
:106B9800403394F8183411480133DBB284F81834C0
:106BA80084F845340E4B00259B6AC4F898549847DE
:106BB80024E71220BAE60E20B8E600BFA80C002091
:106BC8006C12002074130020D80C0020001700203D
:106BD800D415002024160020881600206E120020EC
:106BE800BCF3000873B5134D134E0096EB6C95F883
:106BF800502095F9781095F8480003F0F9F995F8C0
:106C08003031337595F8480040F2012306F13C0213
:106C18003146738203F0F8F950B196F83C3086F8A3
:106C28008230064B00205B6B9847F37C86F8A830CF
:106C380002B070BDA80C002054160020BCF3000858
:106C4800F8B5324C94F81831012B05460ED0022BBA
:106C58004ED0002B57D138B9D4E91B0104F1740385
:106C680083E803000020F8BD012806D102F02CFBC0
:106C78000028F8D184F81851F5E7022843D1244EAA
:106C880084F8180106F5747CBCE80F0006F57A77DD
:106C98000FC79CE8030094F8E92094F8003187E8CE
:106CA800030086F8FB53D2B1022B18D1D4F8043173
:106CB8006367C6F8EC3394F87D3094F8082186F8B9
:106CC800F83394F88C3084F8782086F8F93396F8FD
:106CD8001B2486F8E82340F20133A6F8FA33002390
:106CE80086F81A340B4BDB6A9847FFF77BFFB9E746
:106CF80048B9074B84F81801062283F89024054BFD
:106D0800DB6A9847AEE70320ADE700BFA80C002078
:106D18006C120020BCF30008F0B5504C504EB4F88B
:106D2800DC202287D4E92D0194F8B12084F8692069
:106D380004F16C0282E80300D4E92F0104F1740223
:106D480082E80300B4F8C420A4F87C2091B0D4F8F9
:106D5800CC20D4F8C810C4F884200025D4F8D0205A
:106D6800C4F888200123A4F82031C4F8801084F8DE
:106D78003051A56284F81B5184F83A5084F81D51AB
:106D880084F81E51C4F83451C6F89854A6F818541B
:106D980086F81A54A4F838518DF8183004F5097398
:106DA800039304F50A7394F84800049303A92D4B40
:106DB80084F84551C4E94F55A4F84651059303F0AA
:106DC800FFF8E36EC6F8D43394F87D3086F8E033E4
:106DD80094F88C3086F8E1334FF48073A6F8E233E8
:106DE80086F8D05394F8303186F8E43306F5747792
:106DF8000FCF06F57A740FC497E8030040F2012319
:106E080084E80300A6F8FA33D6F8483386F81B540A
:106E1800CDE901551BB15A685B6901920293124B87
:106E28000793A3F148020892A3F1140209920F4AAA
:106E38000B9229330A93A2F19C030C93A2F19803B5
:106E48000D93131D0E9301A902F14C0307A802F537
:106E580099620F9302F022FA11B0F0BDA80C00203D
:106E68006C12002054060020D41600208C0D00203F
:106E7800F8B50D4F0D4E0C4607F046FB3B6B984797
:106E88000B4A96F84800214603F0BEF850B1094D68
:106E9800706D95F8243485F86A347B6B9847E37CE9
:106EA80085F89034F8BD00BFBCF30008A80C00209A
:106EB800901600206C1200200F4890F81B3480F8C0
:106EC800B8330E4B93F8692080F8BB2393F87D20E4
:106ED80080F8C82393F88C2080F8C92393F83031C0
:106EE80080F8CC330022A0F8CA2300F56E7100F5B3
:106EF8006070FFF7BDBF00BF6C120020A80C002017
:106F0800114890F89034EBB190F81B3480F8D033E6
:106F18000E4BDA6EC0F8D42393F87D2080F8E02376
:106F280093F88C2080F8E12393F8303180F8E4332B
:106F38004FF48072A0F8E22300F5747100F56670D2
:106F4800FFF796BF704700BF6C120020A80C002006
:106F580070B5344C2421204604F0D4FF636A98426B
:106F680018BF60624FF01C012F4814BF012500258F
:106F780004F0C8FF636C984218BF60644FF48071D6
:106F88002A4818BF45F0020504F0BCFFD4F8483180
:106F9800984218BFC4F848014FF0D401244818BFDC
:106FA80045F0040504F0AEFFD4F82032984218BF2B
:106FB800C4F820024FF000011E4818BF45F008052C
:106FC80004F0A0FFD4F82432984218BFC4F8240271
:106FD8004FF46071184818BF45F0100504F092FF8F
:106FE800D4F8A835984218BFC4F8A8054FF0140182
:106FF800124818BF45F0200504F084FFD4F8C035C6
:1070080098420F4B18BFC4F8C005D3F8483318BFCF
:1070180045F040052BB11B691BB12846BDE87040FF
:10702800184770BDA80C0020D00C0020F00C0020E0
:10703800F40D0020CC0E0020D00E002054120020A9
:107048006C1200202DE9F04F8FB04FF00009012B92
:1070580006460F4690468DF80D90ADF8109002D870
:107068004C46BC4202D30FB0BDE8F08F305D02F051
:1070780033FA2044B842F6DC335D651C023BEDB2BE
:10708800112BF0D801A252F823F000BFDD700008E0
:1070980007710008057200082D720008AB7200081D
:1070A800D1720008377300085F730008E5730008A1
:1070B8006F7000086F700008397400086F7000085E
:1070C8006F700008E1740008097500084175000830
:1070D80075750008052002F0A7FA70B10521002097
:1070E80002F068FA725DBA4BE51C0234E4B283F828
:1070F8005C24325D83F85D24EDB22C46B1E70023B1
:107108008DF80E308DF80F308DF814308DF818305A
:10711800B9F1000F6DD1AF4C4FF0050994F87C2000
:107128008DF831206B1E94F839208DF833203344C4
:1071380094F838200B938DF8342094F81A3194F889
:1071480068208DF83520D4F82C218DF832300A9239
:1071580073B37B1C5B1BDBB28DF8303006AB01933D
:1071680005AB009394F848000DF10F030DF10E02E2
:107178000AA902F05DFF8DF80D0000F0070007284E
:1071880013D194F939209DF90E3084F839309A4298
:107198009DF80F3084F83830B8BF01229DF81430BC
:1071A800B8BF84F81D2184F868304FF0000A09E060
:1071B8000523D1E701220DF10D01032002F0A4F807
:1071C8000AF1010A5FFA8AF29DF81830B3FBF9F167
:1071D8009142EFD82B44DDB26B1EDBB29F420BD934
:1071E800F25C032A9AD0AF4288BF1D464FF00109CE
:1071F80083E70534E5B2F9E71D46F7E7735D75499E
:1072080003F00F03012281F81B31023402FA03F361
:10721800A1F82031E4B2002204A9042002F074F895
:1072280025466AE707238DF80D30735DC3F3021214
:1072380003F00F038DF82830E31CDBB28DF829200A
:10724800F25C231DDBB2651DF35C0234E4B21B045F
:1072580043EA0223325D5F4C13436422534394F89C
:1072680048000B930AA902F0F2FE00F00703072B6F
:10727800EDB28DF80D000CD19DF8283084F87030EF
:1072880084F878300B9BE36663679DF8293084F8AF
:1072980069308DF81000012204A9052002F034F8A5
:1072A8002BE74B4BD3F8483363B11B6853B198476E
:1072B80008F03F038DF810008DF81130022204A960
:1072C8000620EBE7FF20F3E703238DF80D30735D0D
:1072D8008DF81C300AAB0693E31CDBB2A51DF25CEB
:1072E800231DDBB206A9F35C1B0443EA0223A21C9C
:1072F800D2B20534B25C134364225343E4B20A9316
:1073080000230B93335D8DF83030324B93F84800EF
:1073180002F0A3FEC3B20028EDB28DF80D30FFF6DF
:10732800ECAE8DF81030012204A90720B6E7735D92
:1073380003F00F03012B4FF47A7238BF0123534334
:10734800244A0234936503F57A73D365E4B20022C4
:1073580004A9082062E7735D1E4DC3F340128DF83F
:10736800152095F84800C3F3001205A903F00F0390
:107378008DF814208DF8163002F075FE02340130B5
:10738800E4B23FF44DAFBDF81430134AA5F87C3091
:107398009DF816309DF814A0D05CF9F713FA022373
:1073A800C5F880000AA995F848008DF828308DF8AE
:1073B8002AA002F0F7FD95F93930069040B29842BC
:1073C800B8BF184685F83900002204A9092025E726
:1073D8006C120020A80C0020C3EC000803238DF8D1
:1073E8000D30735D8DF82830E31CDBB2651DF25C4F
:1073F800231DDBB20234F35CE4B21B0443EA02232C
:10740800325D1343642253430B93644B0AA993F8E8
:10741800480002F02EFEC3B20028EDB28DF80D3000
:10742800FFF66BAE8DF81030012204A90A2035E76B
:10743800092002F0F9F8DFF868B1002849D00921DD
:10744800002002F0B7F80023ADF81E30A31CDBB211
:10745800F25CE31CDBB216F803A0735D4FEA0A4A3C
:107468004AEA022A4AEA030A231DDBB2A51D0534AB
:10747800F35CE4B24AEA036A335D4FF47A72534329
:107488000AAC1B122046ADF81C3006F04DFF454BE8
:1074980053440693DBF83C3300930DF1180A9AE83D
:1074A8000600DBF8383308A806F0FBFE099B0093BA
:1074B80094E80600089B504606F0D8FE9AE80300B8
:1074C80006F00AFF01F00AFF0123EDB28BF8383409
:1074D80013E68BF8380410E60C2002F0A5F8002813
:1074E8003FF40BAE0C21002002F064F82C4B93F80B
:1074F8009034043B012B7FF600AE01F0EBFEFCE577
:10750800A31CDBB2725DF15CE31CDBB2651DF35CAE
:107518000434E4B21B04305D43EA012313436421BD
:10752800594300F00F0001F0D6FEEDB28DF81000BF
:10753800012204A91120B1E60D2002F075F80028F7
:107548003FF4DBAD0D21002002F034F8A31CDBB2C0
:10755800154AF05C735D1268251D0334E4B243EAF2
:107568000020315DEDB201F0B8FEC6E5725DA31CE6
:10757800251D0334DBB2E4B2F15C335D1B0443EA3E
:10758800012313436420584301F0A9FEEDB28DF89E
:107598001000012204A9132080E600BFA80C0020D7
:1075A8006C120020803DD5123C0600200E4B93F84B
:1075B8009124920703D593F88F24012A08D90B49FF
:1075C80091F81A2122B18A6A501C18BF01328A62C6
:1075D8000022A3F8182483F81A24D3F8402322F0B1
:1075E8000202C3F8402370476C120020A80C002048
:1075F80070B5184C1848194D06F086FFD4F840337A
:10760800D4F89804D5F8906023F02003C4F84033E8
:1076180038B106F03FFF864203D2002385F83A309E
:1076280070BD0120FFF766F90028F9D00B28F7D0C4
:1076380095F8393084F84234092094F8183484F8DD
:10764800453484F8410401F0D7FFBDE87040FFF7E6
:10765800ADBF00BF6C120020D4150020A80C00207C
:10766800094BD3F84023012A0AD008490978C907E9
:1076780008D43AB993F89204013818BF012070472A
:1076880000207047012070476C120020500600202F
:10769800034BD3F84003431E58425841704700BF7C
:1076A8006C1200202DE9F04FA9B0EFF3108272B6EA
:1076B800DFF8F0B20021DBF80030CBF8001082F3DD
:1076C8001088B94C002B00F0E180DAB29B060392D7
:1076D80064D5B64D95F81831022B02D0B44BDB6A4D
:1076E8009847EFF3108872B6B24F06F0C9FE3E68AD
:1076F800D4F8B013361A3144AF4806F08DFFAE48BF
:1077080006F050FFD4F8B413AC48314406F084FFB7
:10771800AA4806F047FF88F3108894F81A34002B1B
:1077280000F06B81152312A995F848008DF84830B0
:1077380002F038FCD4F8B4130F900144A04806F0C6
:107748006BFF9F4806F02EFF3B6894F81B24EB6202
:107758000DAF38468DF870201D9306F00BFED5F856
:107768002831009306AE97E80600D5F82431304654
:1077780006F097FD96E803001FAB83E80300D4F8F2
:107788001C341E9395F8303195F84800003B18BF1B
:1077980001231CA98DF8713002F00DFC039BDF0654
:1077A80048D5824DDFF81CA2D5F8E42004929BF856
:1077B8000020BAF90A809AF90C90A4F88C84002366
:1077C80063F300020A9384F84434A4F8223484F85A
:1077D8002534C4F82834A4F82C3484F82E34C4F89A
:1077E800303484F82034C4F8343484F83834C4F895
:1077F8003C346F4B8BF8002094F89024DB6A84F8B3
:107808008E9484F88F24DAF80470BAF808609847E0
:1078180094F88F3413B9694806F076FE3146384635
:1078280001F045FD8346002800F0EA80A4F87E8434
:1078380084F88094039B19071AD55C4B93F8183188
:10784800022B02D05A4BDB6A98470220FEF712FF40
:1078580084F8410401F0D0FE94F81A3413B10123DE
:1078680084F8193494F8913443F0100384F891346F
:10787800039B5A0703D506210520FEF765FF039BE6
:107888009B0703D504210320FEF75EFF01F02DFDC1
:1078980094F89124D7065FD5002384F89234D4F85D
:1078A80040331E0644BF23F08203C4F8403312F06D
:1078B800050F00F0FB820B2001F0B6FE002800F057
:1078C800F58294F89134DD0700F1F082580740F111
:1078D8000783D4F8403323F00203C4F84033D4F8C4
:1078E800402382BB94F8915415F001011EBF2B462A
:1078F80062F3000384F8913494F891345E0744BF2E
:107908006FF3820384F89134012384F8923421B10F
:10791800D4F844332C481B6898476D070BD52B487F
:1079280001F08EFE01F0BCFE28B194F8913443F0CA
:10793800040384F8913401F0C6FC94F891346FF391
:10794800041384F89134012384F8923494F8913420
:1079580043F0200384F8913494F8913418070AD539
:107968006FF3C3031A4984F89134D4F84433A1F16E
:107978002400DB68984794F8913499070AD56FF387
:107988004103134984F89134D4F84433A1F16C00CD
:107998005B68984794F89034022B1BD1FFF722F9C3
:1079A80018E000BF500600206C120020A80C002030
:1079B800BCF300084C060020EC150020041600203B
:1079C8006C1600203C060020AC160020C0160020D3
:1079D800F816002094F891349A0640F1C4826FF3A7
:1079E800451384F89134D4F84033002B40F0BB821F
:1079F80029B0BDE8F04FFFF7ABBA84F84134A3E6ED
:107A080095F81831012B0CD101F055FC804668B16E
:107A1800584601F045FC584601F047FC042384F819
:107A28008F347EB9012384F821344FE101F045FCFD
:107A38000028F6D0404601F034FC404601F036FC00
:107A48000523ECE73B7805935B09013B062B00F225
:107A58001782DFE813F0070015029500150292005F
:107A680015020602102EDDD995F830311297F6B2BC
:107A78008DF84C60002BD5D11CA804F055F912AA3A
:107A88001CA9FF2002F09EF89DF85830C3F30303A9
:107A980007468DF82C3095F8480095F87D308DF81C
:107AA8002D3007220BA902F090FA002F5DD1002893
:107AB8005BD09DF853309DF852201599C5F8E41015
:107AC8001B0443EA02239DF8512002201343C5F802
:107AD800E03004F037F99DF8583095F8480085F8FB
:107AE8002E71C3F30212C3F3030385F8703085F8CF
:107AF80078309DF8593085F86920012B38BF01236B
:107B08004FF47A725343AB651344EB650DF15A0396
:107B18004FF001081093113E94F81B348DF83C3057
:107B28000FA985F868808DF8446002F056FA0223A0
:107B3800404685F8303101F077FD18B141463846A6
:107B480001F038FD94F88F34012B00F2A78194F8E6
:107B58001A34002B40F09A8194F8913443F01003C2
:107B680084F89134FEF786FD64E6012001F05CFD9F
:107B78000028E7D001210720E2E7012384F8203418
:107B880095F87D308DF82E3094F824348DF82D300A
:107B980095F88C3095F848000D330BA98DF82C30EA
:107BA80002F000FAA6F10D031BB2099023EAE37371
:107BB80000B283423FF736AF0B2E7FF633AFBA4B96
:107BC80025931CA8FF231C978DF874608DF89830B6
:107BD80002F0C4F8074600287FF424AF95F818315E
:107BE800012B13D101F067FB002872D0384601F051
:107BF80057FB384601F059FB04239DF87C101E986A
:107C080084F88F34C1F3001101F06EFB9DF87C30CD
:107C18001E99C4F8341413F00F0203D09DF8900095
:107C2800002862D19DF89800002861D0002A7FF4CE
:107C3800F9AE9DF89020002A14BF4FF003084FF0CA
:107C4800020800220A92D5F8EC2095F8E900914242
:107C580051D100284FD0D5F80C1195F8EAB0096831
:107C68000A9195F81811022902D1032184F88F147A
:107C7800B8F1030F7FF4D6AE13F0600F7FF4D2AEE5
:107C88000492012795F82E31BBF1000F36D0BBF1D5
:107C9800010F13D1012B33D16FF0090646FA08F60C
:107CA80006F00106C6F10206F6B2BDF87E100AAA71
:107CB800304601F011FE38B3072823D0012384F899
:107CC80021340A9BC4F83034C4F86C34FEF720FD24
:107CD800B0E501F0F2FA002898D0384601F0E1FA50
:107CE800384601F0E3FA052387E74FF00008A8E7D4
:107CF8004FF00108A5E74FF0010BC3E70426D4E7CE
:107D08000326D2E70823DAE71CAB009304990A9B01
:107D18003246584601F0A2FE20B1022814BF0B23B8
:107D28000A2380E60A9BC4F83034C4F86C349DF802
:107D38007C3084F82104C3F3401384F82E3484F88B
:107D4800443494F88F3484F82274012B9EBF0122A6
:107D5800A86285F81E21012FC4F8280484F82C0491
:107D680084F8410438D1022284F8202495F83A2076
:107D7800002A4AD19DF87C20D60646D4012B94F8D7
:107D880040149DF87C2005D8012901D1900601D521
:107D980001F04CFBB8F1020F94F88F3443D0B8F1DE
:107DA800030F0AD09DF87C10B8F1010F4A4601F084
:107DB8000F0120A83BD0FFF745F99DF8903084F8D3
:107DC8002334259BC4F828349DF8983084F82C3443
:107DD800012384F82D3430E0059A02F0E002A02A4D
:107DE8001BD195F82E11012285F83A2009B9279957
:107DF8006963012B84F8202407D9D5F89020C4F8AA
:107E08003C24DAF80020C4F8982495F81821002AB0
:107E1800B4D1012284F82524B0E7002285F83A205D
:107E280084F82024A6E79DF8981025984A46FFF77D
:107E380009F99DF8903084F823349DF89020E02AC1
:107E480008D195F81F312BB984F82324C4F82834B5
:107E5800A4F82C3494F8913443F0020384F8913454
:107E680070E6114D013EB2B2791C284604F034F890
:107E78000323A4F82034C4F8285484F82C64E9E7D0
:107E8800012384F82134FEF743FC5BE694F844347C
:107E9800002B3FF461AE0020FEF726FC94F88F34E7
:107EA800022B3FF45FAE57E6A414002094F89134F7
:107EB800590715D5012001F0B7FB60B1012001F089
:107EC8008BFB08B984F81804D4F8403323F0020374
:107ED800C4F8403304E0062001F0A6FB0028F3D1E3
:107EE80094F89134DA077FF5FAAC94F840240AB193
:107EF800032A18D11D4A94F8181492F86820914260
:107F080005D29B0723D594F88F34012B1FD8184826
:107F180006F0FAFAD4F8403323F02003C4F84033CB
:107F2800FFF744FBDBE4012A11D194F81924002A55
:107F38003FF4D5AC0D4A94F8181492F86820914291
:107F4800E5D29F0703D594F84434002BDFD194F889
:107F5800913400206FF3041384F8913484F81904E1
:107F6800FFF746FBBBE429B0BDE8F08FA80C002062
:107F7800D41500202DE9F04F89468DB0904607466C
:107F8800002800F08F81002900F08C810368002B05
:107F980000F088814368002B00F084818368002BFF
:107FA80000F08081C368002B00F07C81104601F04E
:107FB800F5FF002800F07881BD4CBE4D384601F031
:107FC800AFFA40F2C4520021204603F099FF40F274
:107FD8001C520021284603F093FFB74BC4F82C31FC
:107FE80004F50973089304F50A73002640460993BB
:107FF80008A9B24B84F848800A9384F8186184F879
:108008008C608DF82C6001F0DBFF0F2306A994F833
:1080180048008DF8183001F0C5FF801B18BF0120FB
:108028004FF00A0B84F81C0106A994F848008DF853
:1080380018B001F0B7FF4FF0060A84F8DC0006A973
:1080480094F848008DF818A001F0ACFF102384F8CC
:10805800DD0006A994F848008DF8183001F0A2FF59
:108068001123C4F89C0006A994F848008DF818302C
:1080780001F098FF1223C4F8A00006A994F848005C
:108088008DF8183001F08EFF1323C4F8A40006A958
:1080980094F848008DF8183001F084FF1423C4F8D0
:1080A800A80006A994F848008DF8183001F07AFF66
:1080B8001623C4F8AC0006A994F848008DF81830C7
:1080C80001F070FF172384F8B10006A994F848005E
:1080D8008DF8183001F066FF18230DEB0301C4F882
:1080E800B400C4F8BC0094F848008DF8183001F0CA
:1080F80059FFC0B21D2384F8B80084F8C00006A94F
:1081080094F848008DF8183001F04CFF1E2384F8CD
:10811800C40006A994F848008DF8183001F042FF11
:108128001F2384F8C50006A994F848008DF8183074
:1081380001F038FF2023C4F8C80006A994F84800C5
:108148008DF8183001F02EFF0B23C4F8CC0006A9D7
:1081580094F848008DF8183001F024FF0C2306A984
:10816800A4F8D00094F848008DF8183001F01AFFF0
:10817800D4F89C306365D4F8A030A365D4F8A43053
:10818800E365D4F8A83023664FF00108D4F8AC3082
:108198000590A4F8D200636684F8B080C4F894B05F
:1081A80084F898A0C4F84CB084F850A084F868808B
:1081B80084F81F81C5F84893FEF7AEFDC5F84473EF
:1081C800C4E90B663E4B84F8198185F89164C5F8BB
:1081D800408332464FF0FF31009605F55A7006F09D
:1081E80035F9384B009632464FF0FF3105F560708F
:1081F80006F02CF9344B009632464FF0FF3105F566
:10820800667006F023F902AF304B009632464FF005
:10821800FF3105F5806006F019F9384606F0AAF82E
:1082280097E8030004F5927383E80300284B294F6D
:108238001E60294BC5F84C33284BC5F85433284BDE
:10824800C5F85C33274BC5F85033274BC5F858336E
:1082580005F553703B68984704F5A67003F080FB5A
:1082680020B1112630460DB0BDE8F08F204601F050
:1082780003FB0028F5D101F039F8B8B91B4801F023
:108288004DFB06460028ECD17B69984703F002FEB7
:10829800BB6D94F819019847FB6A9847012385F844
:1082A8009234DFE70326DDE70926DBE71326D9E763
:1082B800A80C00206C1200200004000154060020C5
:1082C800F9750008C16E0008096F0008F16600081A
:1082D80050060020BCF30008B16800086568000873
:1082E800AD6600083D68000815680008900D00207C
:1082F80008B5034B0020C3F84003FEF7BBF908BDDF
:108308006C12002010B5FFF7ABF90A4C60B90A4BA4
:1083180093F81831022B02D1084BDB6A98470123E6
:10832800C4F84033002010BDD4F84003013818BF0A
:108338000120F8E76C120020A80C0020BCF300080C
:1083480038B5124C204606F0DFF804F1180006F0A4
:10835800DBF804F1300006F0D7F804F1980006F0D5
:10836800D3F800F0AFFF0A4B0025DB6A984744F8C2
:10837800285CFEF7EDFD0749074840F2C45203F0B8
:10838800ABFD012344F8283C284638BDD41500200D
:10839800BCF30008A80C0020E406002070B52E4BA2
:1083A8008AB0054693F8DD008DF8090093F8DC00E3
:1083B8008DF80A0029489A6A90F818040392002652
:1083C8008DF80B0004960C46002940D00692D3F88D
:1083D800882007921A8F93F81A118DF8151052BA3F
:1083E800ADF8202093F87C2093F848308DF824309D
:1083F80003AB8DF822008DF8232000930DF10A02BB
:108408000DF10B030DF1090105A88DF8146000F0BA
:10841800D7FE9DF90900FEF74FF9607004A801F036
:108428001BF8B0B9049A0F2A0DD863789A420AD873
:108438001544AB42A3EB02012CBF002001202170A0
:10844800C0000AB070BD002323700820F9E703209C
:10845800F7E71320F5E700BFA80C00206C120020F6
:108468001FB50446002800F010810378412B00F264
:108478000781DFE813F0420049004D005100550024
:1084880059005E0005010501050105010501050109
:1084980005010501650069006D0078007F00820014
:1084A80085008A0088008C0090009300960099004F
:1084B8009C009F00AE00B200BA00B600BE00C1002A
:1084C800C500CE00CA00CC000501D2000501050197
:1084D8000501050105010501050105010501050164
:1084E80005010501050105010501DA00DE00E200CC
:1084F800E700EB00EF00F300FC00664B93F818313F
:108508002371002004B010BD624B93F83031F7E7B7
:10851800406803F0C3FBF4E7406803F005FCF0E7AC
:108528005C4B93F81A31EBE75A4BD3F8E0306360B1
:10853800E7E7584B011D93F8300103F00DFCE0E725
:10854800544B93F81931DBE7524B93F88C30D7E74B
:108558001C238DF808304F4B02A993F8480001F00E
:1085680021FD6060CDE74C4B043493E8030084E8B8
:108578000300C6E7494B0434F7E7494B0434F4E7F2
:10858800484B0434F1E71A23E3E71923E1E7414BA9
:1085980093F86830B4E73F4B5B6DC8E73D4B9B6D84
:1085A800C5E73C4BDB6DC2E73A4B1B6EBFE7394B67
:1085B8005B6EBCE702238DF80830364B02A993F8AE
:1085C8007C2093F848008DF80A2001F0EBFC20711C
:1085D80097E7304B93F8DD3092E72E4B93F839301C
:1085E8008EE72C4B93F8DC308AE72A4B93F8383027
:1085F80086E7284BDB6C9AE7264B93F850307FE7E9
:10860800244BD3F8843063607BE7224B8FE7264BFB
:108618008DE7204BD3F8CC30F5E71E4BD3F82C313F
:10862800436001F04DFDA0606BE71A4BD3F8903022
:108638007DE7184B93F81F3162E7164BB3F8883083
:10864800A3805EE7134BB3F88A30F9E7114BB3F810
:10865800D030F5E70F4BB3F8D230F1E70D4B93F874
:1086680048200AB1062A12D1B3F8A035E8E7094B29
:1086780093F848200AB1062A09D1D3F8A43556E759
:1086880004B0BDE8104000F021BE03203AE71820EE
:1086980038E700BFA80C0020140D00205C0D002056
:1086A8001C0D0020640D0020E40600207FB5044660
:1086B80010B9032004B070BDA34DD5F840339A0714
:1086C80000F16F820278412A00F26882DFE812F036
:1086D8004200470055005B005F00640069007600B7
:1086E800810087008D00930099009F00A500AB00D2
:1086F800B5006602BA00DC00EF0016013801290156
:1087080042014B014F01530157015B0166025F01B2
:10871800710199018701AB01B101B801BD01C20125
:10872800660228026602660266026602660266023F
:1087380066026602660266026602660266026602F1
:1087480066026602340239023E02430248024D02C2
:1087580052025C020079FEF773FA30B1AAE7037996
:10876800022BA6D0794A82F8303195F8913443F03B
:10877800200385F8913400209CE7406803F080FAD4
:108788000028F2D095E7406803F0BEFAF8E76F4B8F
:10879800027983F81A21E8E76C4B4268C3F8E020B5
:1087A800E3E76A4E416896F8300103F0CBFA0028F7
:1087B8007FF47FAF6368C6F8E430D6E741680029E4
:1087C8003FF477AF002001F0DDF90028CDD011206B
:1087D80070E7416800293FF46CAF0120F3E7416876
:1087E80000293FF466AF0820EDE7416800293FF40F
:1087F80060AF0920E7E7416800293FF45AAF0C2031
:10880800E1E7416800293FF454AF0D20DBE74168F8
:1088180000293FF44EAF0E20D5E7416800293FF408
:1088280048AF0F20CFE74A4C484B007983F819012D
:10883800A36D9847E36A984797E7444B027983F812
:108848008C2092E7414E037A8DF8043096F8480060
:1088580096F87D308DF80530072201A901F0B5FBA7
:1088680000283FF426AF636896F848000193002279
:1088780001A901F0AAFB00283FF41BAF6C36D4E92C
:10888800010186E8030070E7304E037A8DF8043062
:1088980096F8480096F87D308DF80530072201A932
:1088A80001F093FB00283FF404AFB436E7E7274E06
:1088B800037A8DF8043096F8480096F87D308DF8E4
:1088C8000530072201A901F080FB00283FF4F1AE32
:1088D800D4E9010106F1740383E8030096F818311E
:1088E800022B7FF442AF96F83031002B3FF43DAFB6
:1088F800174BDB6A9847FEF775F936E7134E037A8C
:108908008DF8043096F8480096F87D308DF80530DB
:10891800072201A901F059FB00283FF4CAAEBC3672
:10892800ADE74368029301238DF80C30074B02A989
:1089380093F8480001F056FB00287FF416AFB8E61C
:10894800436802930023EFE76C120020A80C002074
:10895800BCF3000803795A1E0E2A3FF6AAAE934AC2
:1089680082F8683001E7914B42685A65FDE68F4B03
:1089780042689A65F9E68D4B4268DA65F5E68B4BF5
:1089880042681A66F1E6894B42685A66EDE6874CFA
:10899800037994F848008DF80430062201A901F003
:1089A80014FB00283FF485AE9DF8043084F8DD30D0
:1089B800DBE67E4C03798DF8043094F8480094F88F
:1089C8007C308DF80630052201A901F0FEFA002856
:1089D8003FF46FAE9DF8043084F83930C5E6734C27
:1089E800037994F848008DF804300A2201A901F0AF
:1089F800ECFA00283FF45DAE9DF8043084F8DC30D2
:108A0800B3E66A4C037994F848008DF804300922DB
:108A180001A901F0DAFA00283FF44BAE9DF80430C2
:108A280084F83830A1E6614B4268C3F89420DA64D0
:108A38009BE65E4B027983F8982083F8502094E6F1
:108A48005A4B4268C3F884208FE6584B4268C3F8F3
:108A5800CC208AE6012B40F0A480554C24212046E6
:108A680003F050FA636A984201D0172022E61C21CD
:108A780004F1280003F046FA636C9842F5D14FF4EC
:108A8800807104F1480003F03DFAD4F84831984267
:108A9800EBD1D42104F5A67003F034FAD4F82032CF
:108AA8009842E2D1002104F5097003F02BFAD4F8BA
:108AB80024329842D9D14FF4607104F50A7003F05A
:108AC80021FAD4F8A8359842CFD1142104F2AC5039
:108AD80003F018FAD4F8C0359842C6D1334E21466F
:108AE800304640F2C45203F0F7F9204640F2C4522F
:108AF800002103F005FA95F81B3485F8E833736F05
:108B0800C5F8EC3396F87D3085F8F83340F2012348
:108B1800A5F8FA33274B96F819019B6D984724E678
:108B28008379012B3FF6C5AD204B42684068C3F8F6
:108B38002C2100F0BDFE48E61C4B4268C3F890208B
:108B480013E61A4B027983F81F210EE6174B828829
:108B5800A3F8882009E6154B8288A3F88A2004E642
:108B6800124B8288A3F8D020FFE5104B8288A3F827
:108B7800D220FAE50D4B93F848200AB1062A12D103
:108B8800A288A3F8A025F0E5084B93F848200AB17D
:108B9800062A08D16268C3F8A425E6E500F098FB28
:108BA800DBE5012086E5182084E500BFA80C00203D
:108BB800E4060020BCF300082DE9F04387B0002349
:108BC800ADF800300646002800F0EE800361FEF79D
:108BD80047FD20B10124204607B0BDE8F08300F02E
:108BE80065FD0028F6D100F05BFD014618B96F4815
:108BF800142203F085F96E4D95F89134012243F063
:108C0800040385F8552485F8913433788DF80430B9
:108C18000021013B8DF80520ADF806100C2B00F261
:108C2800BB80DFE803F007B9B9B97982B9B990B95F
:108C3800AD9AA900D5F8407317F02007CAD196F865
:108C48000480B8F1020F46D1DFF868815A4CFEF76C
:108C580063F896F9051098F848003A4601F00FFABB
:108C680088F83900B37988F83830384607238DF802
:108C78000530FDF7E5FFFF2304F58670A5F80C31F4
:108C8800C5F8084185F8047103F04EF804F58A70B8
:108C980003F004F83846FDF72DFE0446002839D0C5
:108CA80096F9051098F84800012201F0E8F988F8CB
:108CB8003900D5F894343361002C71D000F0F0FC01
:108CC800002888D195F8913485F81A0460F3820356
:108CD80085F891347FE7B8F1010F4FF00204E8D12D
:108CE800DFF8D0908DF8144099F8480089F81D7184
:108CF80002A901F065F9337989F830318DF80570EA
:108D08008DF80680FDF7C4FC95F8913443F0100304
:108D180085F891340024CCE700226946022000F04F
:108D2800F3FA0028F6D01324C3E7244BB288DB6B90
:108D380096F90C10B0689847D5F8403343F0020311
:108D4800C5F84033E6E702A90D2000F053FB0028E0
:108D5800E0D0002269460D20E1E7164B93F8183160
:108D6800D3B9347904F0070000F0ABFA8DF800406D
:108D7800012269461020D2E7002269461220CEE778
:108D88008DF8072000F08EFA044638B900F087FA0B
:108D9800204600F089FABDE702248AE7012488E723
:108DA80001A800F0D1FB16E7032414E7C016002041
:108DB8006C120020A80C00206E120020BCF30008E2
:108DC8002DE9F04F99B08046059118B9032019B0E4
:108DD800BDE8F08F00230361FEF742FC044600283B
:108DE80040F0A58046460FCE0EAD0FC5142252485E
:108DF80098F800A0B8F80C7098F90EB04F4E2146BC
:108E080003F07EF84E4B012283F8412496F8302176
:108E1800022A25460BD196F81821022A07D196F87E
:108E28001E2122B9BAF1010F38BF4FF0010ABAF179
:108E3800010F2BD0BAF1030F2AD0BAF1000F33D1AA
:108E480002229DF83C30DDF84090029362F347150A
:108E5800012496F87C108DF8321002220CA996F89D
:108E680048008DF8302001F09DF896F81A3196F8F0
:108E780030C196F81D1140B2002B63D0BCF1010F30
:108E880057D1002955D1002C61D153E00422D8E7ED
:108E98000023DDF83C90BDF840709DF942B0029384
:108EA80065F01F050124D4E74FF0000BD946CDF833
:108EB80008B0CEE74FF0010084F81A04D2E005F2BA
:108EC8009A420BA900F0D4FA002800F0158113206B
:108ED800049B33871A4B002283F81A2423E105F2F6
:108EE8009A452A460BA900F0C3FA0028EFD10B9B3C
:108EF80084F82801C4F82C5184F83031FCE0B9F129
:108F0800000F00F0F980002A00F0F6804946E01CC6
:108F180002F0E2FF94F8373201332380ECE01220AC
:108F2800D6E70220D4E70720D4E71320D2E70120B0
:108F38004DE7FCB90220F6E0AC160020A80C002092
:108F48006C120020002CF5D05845B8BF584696F84A
:108F58007C308DF82000052296F848008DF82230E4
:108F680008A901F032F800283FF430AF9DF820300E
:108F780086F839306F4A704BD2F89804D3F890408D
:108F880038B105F087FA6C4B84423CBF002283F865
:108F98003A20198F1A8F93F830010491996A099130
:108FA80052BA0028BFD093F81B0100B9186393F890
:108FB8001801ADF85820013893F87C2093F81A412D
:108FC8001491D0F1000BD3F888108DF85B204BEB8F
:108FD800000B93F8482093F83A0093F868308DF81E
:108FE8005A3009AB0093554B03904FF001008DF8B0
:108FF8004C0015918DF85C20A3F12F01A3F13002EC
:1090080013A88DF84D4000F0DBF8039B4FEA0B1BCB
:109018004BEA431B00264BEA801B4BEAC413B145BD
:10902800444C039308BF37463A46494604F59C70BA
:10903800CDE90A669B46268084F81A6402F04CFF44
:10904800E9B2A570C5F34215FAB2042D3A4E039B56
:1090580084F837223FF42EAF072D3FF450AF022D8E
:109068007FF45FAF364D84F80D110420029984F81F
:109078000401FF2084F80C0184F8281184F81431C5
:10908800D6F8E410C4F8085105F59B730AA8C4F88B
:10909800101184F83021C4F82C3100F011FC00289C
:1090A8007FF43DAF0A9BA4F844040BA8A4F816313A
:1090B800C4F84C3400F0D0F900287FF408AF0B9BBB
:1090C800D3B196F93900FDF7F7FA94F83732002B47
:1090D8003FF405AF0B9B0F2B3FF6F1AE05F58B72F6
:1090E8000BA90F2000F0C4F900287FF4F0AE0B9B09
:1090F80063F3030B84F814B10598FDF7FBFB002814
:109108007FF4E6AE099B86F83A00B36200F080F976
:1091180000287FF40AAF94F8913484F840A443F00F
:10912800010384F89134034BD3F89434C8F8103011
:109138004DE600BF6C120020A80C0020100D002086
:109148006E12002037B50B4D8DF8040004460F222F
:1091580095F8480001A900F038FF40B1064A85F8A3
:109168001C4192F8913443F0200382F8913403B003
:1091780030BD00BFA80C00206C12002010B5FFF70E
:10918800C1F8044688B90A4805F0BEF9094805F04F
:10919800BBF9094805F0B8F900F094F8FDF7BCFDF3
:1091A800064BDB6A9847204610BD0124FBE700BF49
:1091B800D4150020EC15002004160020BCF300088C
:1091C8002DE9F04F8BB047780093149B90F90C80F1
:1091D80090F90D6090F80EB08A464168196004460F
:1091E8009146002F58D002238DF8103004A9C37B74
:1091F800007C8DF8123000F0D5FEB4F808C0618903
:1092080043B26068984545466144B8BF1D4660450D
:1092180034BF00270127884209D30A218DF810108E
:10922800207C019304A900F0BDFE019B46B2B4F86E
:1092380008C0608961680CEB400E714519D3A1EB39
:109248000C01B1FBF0FC00FB1C1191B9984503DC43
:109258002378CBB94FF0010B21238DF81030207CF7
:10926800E37B8DF8115004A98DF8123000F09AFEB6
:1092780045B2009B8AF80050384689F8006083F8A8
:1092880000B00BB0BDE8F08F0223207C8DF82430AD
:1092980006A900F095FEDDE74546EAE77047704706
:1092A800704770470020704770477047704700202C
:1092B800704700207047002070470020704700204A
:1092C8007047704770477047022070470220704708
:1092D8000220704770470020704770477047002091
:1092E80070470020704770477047704710B5054CAD
:1092F8004FF403722046002102F002FE0020C4E968
:10930800000010BD881700202DE9F84381469046DB
:1093180000293CD01F4C2023224604F1100012F8EB
:10932800017F6FBB8242FAD11B4E3368013403B907
:109338003460736803B11C6000252560C4F8088098
:1093480074601FFA88F284F80490601D02F0C4FD6E
:10935800B9F1110F4FF0000398BF104D6373D6F8A1
:10936800083298BF25FA09F503F1010398BF05F003
:10937800010543442573C6F808323846BDE8F8832A
:10938800013B13F0FF030446C6D10227F5E7012786
:10939800F3E700BF8F17002088170020200702007E
:1093A80010B518B3124A1368984204D103681360C1
:1093B800002305E00B46002BFAD019688842F9D142
:1093C8005168884208BF53600BB101681960D2F830
:1093D80008328168013B00245B1A04602146C2F808
:1093E8000832102202F08CFD204610BD0120FCE757
:1093F80088170020054B1B6813B11A798242FAD1ED
:10940800002B0B600CBF032000207047881700203A
:1094180010B5054B186800B910BD037B04680BB97B
:10942800FFF7BEFF2046F6E78817002038B5084B3F
:10943800084C186800B938BD03790568112B05D8A0
:1094480024FA03F3DB0701D5FFF7AAFF2846F1E763
:10945800881700202007020028B1044BD3F80832EF
:109468000360002070470120704700BF8817002064
:109478002DE9F04107460E46154642B339B3154B60
:109488001C6800232CB93046FFF7E6FF0020BDE832
:10949800F081A268F91A0132914215D32279EA546F
:1094A800581C22895FFA80F8611D55FA80F002F095
:1094B80013FDA368246898445FFA88F3E2E720461E
:1094C8002568FFF76DFF2C46002CF8D1DBE701205B
:1094D800DDE700BF881700200238C0B211289ABF04
:1094E800014B185C00207047D3EC000830B50B4BDB
:1094F80093F820200446084672B100211C330578F1
:10950800A54208D001319842CDB214BF04301038BA
:10951800AA42F4D8002030BD1046FCE79419002078
:1095280010B5084C00232060142204F10C00FF2120
:1095380084F82030C4E9010002F0E2FC012384F839
:10954800213010BD9419002010B50E4A92F8201051
:10955800042915D8936804781C7044785C70C47822
:10956800807898700131DC7082F8201002F11C01BB
:109578008B4214BF043302F10C039360012010BD29
:109588000020FCE794190020094B93F8200068B1EB
:109598005A6803F11C018A4200F1FF3014BF0432FB
:1095A80003F10C0283F820005A600120704700BFC5
:1095B8009419002010B5074B93F82020044608465C
:1095C80032B15968FFF792FF10B1012344708370DC
:1095D80010BD00BF9419002008B5064B93F8202051
:1095E8002AB15968FFF782FF08B1407808BD012009
:1095F800FCE700BF9419002030B50A4A92F8201001
:10960800536882F8210061B1916801241C32DD7829
:10961800587005B99C70934214BF0433103B9942AB
:10962800F5D130BD9419002008B5044B5968FFF7EF
:109638005DFF003818BF012008BD00BF9419002045
:10964800F7B50422154E044600210DEB020096F8EA
:10965800207002F055FC0025EBB29F4201D803B000
:10966800F0BD7368197821705A786270987838B1AB
:10967800336820469B689847FFF786FF0135EBE77C
:10968800DB788DF804108DF805208DF80730FFF78A
:109698007BFF01A8FFF758FFF0E700BF94190020EF
:1096A800014B93F82000704794190020034B93F85E
:1096B8002000042894BF002001207047941900203E
:1096C8001FB50024CDE90244C41F8DF800408DF871
:1096D80001100C0AADF80420090C120C8DF80310C7
:1096E8008DF806208DF8073002461B0A01216846CE
:1096F8008DF802408DF8083002F05DFA002818BF96
:109708000E2004B010BD2DE9F04188B090460D46FA
:109718000F9A0746002847D000240121CDE90444C8
:109728008DF810109DF838108DF81510ADF816301A
:10973800190CCDE900441B0ECDE902448DF819300F
:10974800ADF81A20130C120E07948DF818108DF826
:109758001C308DF81D20E3B21E01002DF6B203DC8B
:10976800002008B0BDE8F081013310218DF81F30CA
:1097780042466B460DEB010002F0B3F90346A8B967
:10978800102D28463E44A8BF10206946327811F8AB
:1097980001CB013382EA0C02984206F8012BF5DC72
:1097A800103D2DB20134D6E70920DAE70E20D8E7BC
:1097B8000138032815D8DFE800F002080C100A4B1E
:1097C8001B681B690B6000207047074B1B685B69AF
:1097D800F8E7054B1B689B69F4E7034B1B68DB69DB
:1097E800F0E70520704700BFB81900202DE9F041C7
:1097F800C4B00C464A9E17461D468046B8B3B1F51C
:10980800807F36D84FF488720021684602F078FBD2
:10981800492300934FF48073ADF804302B0C8DF876
:109828000830330CADF80650ADF80A608DF80C30EE
:1098380022460023414604A82D0E360E8DF80E3020
:109848008DF809508DF80D608DF80F4002F044FB3B
:1098580004F110014B9A3B4689B2684602F02BF995
:1098680010B1012818BF0E2044B0BDE8F0810920CE
:10987800FAE70D20F8E7000010B590B10A4C28224D
:109888000021206002F03CFB2368084A1A6000208F
:109898004FF0FF32C3E90302C3E90522C3E90722F7
:1098A80010BD0820FCE700BFB81900200001010125
:1098B800024B1B6818600020704700BFB8190020D1
:1098C80030B1044B1B68DB6801330360002070472C
:1098D80009207047B819002013B500230C460193DE
:1098E800CAB101A9FFF764FF18B9019B591C02D13D
:1098F800146002B010BD99B2611A002901DD5C182C
:10990800F6E702D113600720F3E71B0C1B0403F5ED
:1099180080331C44ECE70920EBE7000028B1044B36
:109928001B681C334362002070470920704700BF42
:10993800B81900201FB5044600B3002303A80393F9
:1099480002F090F9104ABDF80C3012682046938056
:10995800E38200F05EFA98B904F1180300932168D5
:109968000123132202F09CF860B9204600F051FA56
:10997800003818BF0120000104B010BD0920FBE722
:109988001020F9E70E20F7E7B8190020F0B50546D2
:1099980087B01C4613B9092007B0F0BD2E4E3368B6
:1099A800DB68834255D894F82020002A0CBF08228F
:1099B8000922834205D3204600F05FFA68B11020DF
:1099C800EAE7002301900093A36894F82810606ADE
:1099D800FFF799FE0028EED0DEE723792168B4F876
:1099E80008C0A768043B9AB20029D4D0B2F5807F9A
:1099F8002DD8ADF80EC08DF817304FEA174C04F18A
:109A08002C033F0E8DF8117000932F0C08234FF094
:109A1800490EADF80C008DF814708DF816002F0E55
:109A28000DEB0300CDF808E08DF810C0ADF812502A
:109A38008DF8157002F034F808B10E20ACE7204616
:109A480000F01BFA0028BAD13368DD60A4E70D20C6
:109A5800A2E70620A0E700BFB81900202DE9FF41C2
:109A68000A9D80460F4616461C46002D5AD00023F4
:109A780003A910460393FFF79BFE18B1062004B014
:109A8800BDE8F081039B9C4201D80133F6D12846FA
:109A980000F064F9002847D1264B1A78424503D0D4
:109AA8001A79424542D10120AA68BA4240D103EB53
:109AB8008002EB6A92F801802979CDE900430439E4
:109AC800927828683B4689B2FFF790FE0028D6D1E5
:109AD80095F820300194002B4FF00103009314BF38
:109AE8004246082295F82810686A3B46FFF70BFEA5
:109AF8000028C4D1013E032EC1D8DFE806F00207D2
:109B08000B0F0D4B1B681C611C62B8E70A4B1B68E6
:109B18005C61F9E7084B1B689C61F5E7064B1B681D
:109B2800DC61ACE70920AAE70F20A8E70B20A6E72D
:109B38000220A4E7F0000020B81900201FB50B2967
:109B48004FF00003CDE90033CDE902330A4607D0D0
:109B58000C2914D00A2910D00A2005B05DF804FB9E
:109B6800012802D120238DF800300021684602F038
:109B780022F8002818BF0E20EFE73023F3E70B2167
:109B8800F4E7000038B5054602F010F8044610B1B5
:109B98000E24204638BD002DFBD1094B1B680B2134
:109BA8009878FFF7CBFF0028F2D10C21FFF7C6FF0A
:109BB8000028EDD10A21FFF7C1FF0028E9D0E7E727
:109BC800B81900202DE9F04380468FB00C4617469F
:109BD800002A6BD0002969D0002529461D2206A835
:109BE800059504F097FE8DF81350344D2B680DF150
:109BF80014099E88CDF804900DF1130302933B7964
:109C080000933B6832462146404601F0F0FF0028A9
:109C18004ED138683A79494602F05EF9384600F084
:109C28004FF8002846D13C7AFA79BB79240444EAF3
:109C380002241C432B689A6894423DD99C609DF885
:109C480013000B21FFF77AFF034658BB0C21FFF7DF
:109C580075FF034630BB0A21FFF770FF034608BBB8
:109C68007B7ABA7AFF7A3F0447EA02271F433A46CB
:109C7800334621460920FFF723FD034690B93346B2
:109C88003A4621460820FFF71BFD034650B92A68CB
:109C98009DF8131091700021D1604FF0FF31C2E997
:109CA8000411916118460FB0BDE8F0830923F9E764
:109CB8000E23F7E70F23F5E70323F3E7B81900208E
:109CC80010B50446002845D00168002942D011F893
:109CD800013B43710322063002F0FEF820460322BE
:109CE80050F8091B043102F0F7F82168CB79E360DA
:109CF8000A7A43EA0223E3604A7A43EA0243E360CA
:109D08008A7A43EA0263E360CB7A23740B7B637439
:109D18002379212B1AD110220D3104F1120002F0FF
:109D2800DBF81D222168501C8B5C6362085C43EAE7
:109D38000023901C6362085C033243EA00436362B9
:109D48008A5C43EA02636362002010BD112B03DCC6
:109D58000D22E7E70220F8E70120F6E710B50446F0
:109D6800002854D00168002951D00B7843714B78F2
:109D780083608A7843EA02238360CA7843EA02430D
:109D880083600A7943EA026383604B7903738B79B2
:109D9800C381CA7943EA0223027BC38102F00F021E
:109DA8000831103002F098F8237B002203F00F03EB
:109DB80084F8202084F82820227903F10800111A59
:109DC80004290DDD21680933043AD21A085C84F8A5
:109DD8002000D2B2606A84F82820194402F07CF886
:109DE800237922681A44002012F8043CE36212F82E
:109DF800031C43EA0123E36212F8021C43EA01430D
:109E0800E36212F8012C43EA0263E36210BD022008
:109E1800FCE710B5044660B3036853B30279162A09
:109E280029D942791A700146082251F8060B0130E7
:109E380002F05CF82146082251F80E0B093002F0B6
:109E480055F82368E28A5A74E38A22681B0A9374D5
:109E58002368A269DA74A36922681B0A1375236848
:109E6800628B5A752368E27E9A7517232371002046
:109E780010BD0120FCE70220FAE738B504460028A7
:109E880063D00168002960D0037B90F8282003F094
:109E98000F03002A57D1083320790432134498421B
:109EA80055D363790B702368A2685A70A368226837
:109EB8001B0A937023686289DA702368E27A1A7140
:109EC8002368227B5A712368E2899A71E3892268A0
:109ED8001B0A2146D371227B51F8100B02F00F02A6
:109EE800083001F0F9FF237B94F8282003F00F03D2
:109EF80003F108052AB1226894F82010515503F19E
:109F08000905206894F82820616A284401F0E4FFD4
:109F180094F828302268E16A2B44D1545A1CE16A2B
:109F2800206892B2090A81549A1C2168E08D92B285
:109F38008854DA1C216894F82F0092B204338854AC
:109F48002371002038BD0933A6E70120FAE7022073
:109F5800F8E70000024B1A8810431880704700BFCA
:109F6800BC19002008B5074B1B883BB1FEF7CAF99E
:109F7800002814BF6FF00200002008BD6FF0010038
:109F8800FBE700BFBC19002010B5034B00241C8060
:109F9800FEF7AEF9204610BDBC190020B0FA80F0DB
:109FA8004009704782B018B9084602B000F0CAB834
:109FB800002002B0704710B9084600F077B9704722
:109FC80010B9084600F08EB9704703460846114696
:109FD8000BB900F0E5B90020704710B9084600F049
:109FE8006DBD704710B9084600F006BA00207047EA
:109FF80010B40446084611461A46019B14B910BC11
:10A0080000F014BA10BC70470346084611460BB955
:10A0180000F03EBA0020704710B4044608461146C6
:10A028001A4614B910BC00F0ABBA002010BC704737
:10A0380030B40546084611461A46DDE902341DB912
:10A04800029430BC00F02ABB002030BC704710B925
:10A05800084600F0DBBB0020704710B9084600F046
:10A068006BBD0020704710B9084600F0EABB00201D
:10A07800704710B9084600F0E7BB00207047034658
:10A08800084611460BB900F001BC0020704710B417
:10A098000446084611461A46019B14B910BC00F044
:10A0A800F7BB092010BC704710B404460846114697
:10A0B8001A4614B910BC00F061BDC8B210BC704794
:10A0C8000048704701000102064B10B51B6A0446A0
:10A0D800984730B10448054B204498428CBF002073
:10A0E800012010BDBCF3000840C220C980B92A0075
:10A0F800F0B5114B85B00C4610491F56054601F0C6
:10A108004BF80F4BE4B25E6A072D4FF00103CDE91F
:10A11800024301460AD105220023CDE900234FF46A
:10A128007A727A431846B04705B0F0BD082200207D
:10A13800CDE900203A46F5E7A0ED000880ED0008DB
:10A14800BCF300081FB5002300930378013B372BAD
:10A1580021D8DFE803F01C242020201E2020202006
:10A168004143454E2055585B5E6164206C1E6E73FA
:10A17800787A20207D812620202020202020202061
:10A188002020202083858A2020838A208C90C378F1
:10A198000BB102230093009805B05DF804FB8378A7
:10A1A800F6E743788DF8043005238DF80530837879
:10A1B800003B18BF01235B008DF8063010238DF893
:10A1C8000730304B1B6801A803F55872CDE902230C
:10A1D80000F0C2FF0090DEE74023DBE72023D9E749
:10A1E800827890F9013012B9274AD35CD2E7274A1E
:10A1F800FBE7827890F90130002AF8D1244AF4E785
:10A2080040F6B833C6E74FF47A73C3E74FF4FA63FE
:10A21800C0E741F28833BDE741F27073BAE71D48E1
:10A228004FF47A7101F03CFE00F5FA60D2E71A4B60
:10A23800B0E7144B1B6803F55873ABE7114B1B6869
:10A2480003F55B73A6E71023A4E70E4B1B68A1E791
:10A258004FF0834300939EE7104BFBE7104B99E7C1
:10A2680040F21113ADF8003095E7032392E790F917
:10A2780001300C4AB9E70C4990F9010000F08CFF55
:10A28800A8E700BFC419002075ED000865ED0008B7
:10A298006DED000818FCFFFF00EA06379A9909409F
:10A2A80040F70937A0ED000880ED000837B50B4BE3
:10A2B80002781B680C2101FB02335B7A03EB430431
:10A2C800074B1D6803690093C3684278816805EBF2
:10A2D800C40000F0DDFC03B030BD00BFC41900208D
:10A2E800C019002070B586B0027B6423ADF8003039
:10A2F800012A4FF00003CDE90133CDE903338DF88E
:10A3080002308DF8143030D0022A39D05ABB036895
:10A318004BB343683BB31F4D80682B601E4B18221C
:10A328006946186001F0D8FD1C4B2C6893E80700BB
:10A338000C3384E8070093E8070004F10C060323B4
:10A3480086E80700A4F86C33012204F55B7104F574
:10A35800587000F08EFC2B684FF6B072A3F8782383
:10A368000522C3F87C2306B070BD0A49086843601B
:10A37800036100F55B7100F5587000F07AFCF2E7B4
:10A38800044B1B68B3F86023B3F86C130A43A3F8B3
:10A398006023E8E7C4190020C0190020C8EA0008B3
:10A3A80008B503460A2924D8DFE801F00623232349
:10A3B800230B161B23212100BDE808400068FFF786
:10A3C80083BE90F900009978052271B900F011FC5C
:10A3D800003818BF012008BD052293F900000021AC
:10A3E800F4E790F900005978EEE70221EEE707223A
:10A3F800F3E70020EFE7000008B502791AB1012A57
:10A408000BD0002008BD084B01681B68012203F52A
:10A41800587000F02EFC0120F4E7034B01681B681C
:10A4280003F55B70F5E700BFC4190020F7B50528F0
:10A43800144D1C46A8BF052058700E4629461746DD
:10A4480000F0AAFE94F90130A070072B13D1322036
:10A4580000F0A2FD0C4BDB6D0546984704F10C0299
:10A4680008340346019200943A463146284600F0E3
:10A4780098FD03B0F0BD054A55F82310D05C00F0F4
:10A4880083FDE7E780ED0008BCF30008A0ED0008B5
:10A498002DE9F04F344F90F901607B68D0F80490B3
:10A4A8008BB00446884698470546002859D1E37C76
:10A4B80073B92E4A2378126803EB4303990002EB21
:10A4C8008303D3F80490B9F1000F01D152F8019039
:10A4D800274B484613F906B0FB689847A37C2289A6
:10A4E800D7F818A00993072E28D100230121CDE918
:10A4F8000223204A0693CDE90431CDE9073305212B
:10A50800CDE900214FF47A7202FB0BF24CF2503184
:10A518001846D047637C13B3174B995D7B6D0D319B
:10A52800C9B228469847E07C3246494600F046FEC4
:10A5380088F8006001200BB0BDE8F08F00210125EC
:10A548000823CDE90013CDE90715CDE90511CDE9BB
:10A5580003110292A1782B465A462846D9E7074BA1
:10A56800DBE70020E7E700BFBCF30008C4190020C0
:10A57800A0ED0008854501006DED000875ED0008A7
:10A588002DE9F04F8DB090F90130DFF8FCA0DFF82D
:10A59800FC90CDE90A123E4A12F903B00278DAF8C3
:10A5A80000300C2505FB02333A4A5B7A126803EB4C
:10A5B800430302EBC303044693F9021090F9020027
:10A5C80000F0E5FD3449064694F9010000F0E4FD89
:10A5D800A26861688046304600F00BFD2178DAF801
:10A5E8000020D9F80C306943074650589847D9F8E5
:10A5F8001C309C4694F901300025072B4FF47A63F0
:10A60800CDE90753CDE905552DD10123CDE90353F4
:10A618000523CDE901534FF47A7303FB0BF3009341
:10A628003946434646F2A81228466746B847237873
:10A63800DAF800200C214B4394F90110D05800F0AF
:10A64800DFFDA18994F90100FFF752FD0B9B217BE7
:10A658001860D9F85430284698470A9B01201E7084
:10A668000DB0BDE8F08F01200823CDE90350CDE9F6
:10A6780001032A46CDF800B0654643463946A84747
:10A6880001200546D3E700BFC4190020BCF3000829
:10A69800A0ED0008C019002080ED00082DE9F04F5A
:10A6A8008FB0002405468A46914698460494ADF832
:10A6B8001440ADF8024007264FF0010B2B7AA34255
:10A6C80006D9686804A9204400F0F6FB00285ED18A
:10A6D80002238DF8083002A86B7A8DF80A30FFF74C
:10A6E80031FDAB7A8DF81D309DF811308DF81E3094
:10A6F8009DF812308DF81F309DF810308DF82030FD
:10A70800EB7A8DF821302B7B8DF822306B7B8DF81E
:10A71800233010238DF81C608DF824303A4E8DF8C4
:10A728002C000DF102030A9305238DF82D303368B0
:10A738000C930723ADF834302B6806930DF1120201
:10A7480004AB0DF1110106A800F0D0FB072805465F
:10A758000BD130680C22002100F5587001F0D0FBB5
:10A768003368BDF80220A3F860239DF811308AF8F9
:10A7780000309DF8123089F800309DF8103088F8C4
:10A788000030189B28461C700FB0BDE8F08F9DF86C
:10A798001330BDF81470ADF802702044C4B2F3B998
:10A7A80017B3194A00201168072602464FF00C0C0F
:10A7B800062B1BD10CFB00FE51F80EE0BEF1000F7A
:10A7C80004D00BFA00F23A4397B201220130102864
:10A7D800EED1002A3FF472AFADF802706EE75A1E50
:10A7E800042A01D9062BDCD0062667E747FA00FEC3
:10A7F8001EF0010FEAD00CFB00FE51F80EE0BEF18E
:10A80800000F08BF0626E1E7C419002038B5054641
:10A818004068FFF759FC0522841D002195F90000C6
:10A82800E4B200F0E6F908B904F0FD0495F9010076
:10A838000722002100F0DDF908B904F0FB042046E6
:10A8480038BD00207047000010B503780F2B044670
:10A8580018D84068FFF738FC22780B4902EB42020F
:10A868000968831C01EB820051F82220DBB21AB977
:10A8780003F0FD0358B210BD032B06BF62684260A7
:10A888000223F7E70020F6E7C419002002207047EA
:10A898002DE9F04FDFF838810446D8F8000099B068
:10A8A8008946174600211E460122032300F55870E9
:10A8B800CDE90611CDE908118DF814108DF81510A1
:10A8C800ADF8163000F0B7F938B9D8F80020B2F86A
:10A8D800603343F00303A2F86033D8F80020637AAA
:10A8E8008DF8283002F55871CDE90B12394A94F9E0
:10A8F800083012680D920DF116020F92226810921C
:10A9080062681192D4E90301A27A8DF848200122E5
:10A918008DF8492013AA82E803001025227DE18AD8
:10A928008DF8293018468DF85420ADF83850FFF7C7
:10A93800DFFB0AAB17930DF1150316900093314610
:10A94800019705AB06AA10A800F0C2FB064698BB03
:10A958009DF81410204F013901F0A2FA1F4B1B6912
:10A968000393C4B24FF00C0B04F160036B44D8F8A6
:10A97800000013F848AC9DF814300BFB0AFC0134B6
:10A988003946B4FBF3F203FB1244D0F87C33B0F938
:10A99800782350F80C00DDF80CC0E4B2E04728B189
:10A9A80089F800A0304619B0BDE8F08F013D15F0D8
:10A9B800FF05D9D10D26F5E70C2801BFD8F80020EE
:10A9C800B2F8603343F00303A2F86033EAE700BF4C
:10A9D800C4190020C0190020400D0300BCF3000872
:10A9E800F8B50679012E054648D90F2E48D80368D0
:10A9F800187A40F303000522002140B200F0F9F86C
:10AA08002B680446187A40F303100522002140B24F
:10AA180000F0EFF8B8B1B4FA84F4640929680B7A45
:10AA2800086843F3030243F303135BB252B29A423A
:10AA3800C8BF0124FFF748FB80F00103DBB224B153
:10AA48000533D8B2F8BD0124E8E7DBB90E4F296811
:10AA58003B6806EB460003EB80000C2201F03CFA51
:10AA68003A680C2303FB062320465C72B2F8601395
:10AA78000123B3400B43A2F86033E3E70620E1E784
:10AA88000320DFE70420DDE7C419002010B40178B3
:10AA980001290ED9084B18680C234B43C41800220F
:10AAA800C250C4E9012200F5587010BC102200F011
:10AAB800A9B8002010BC7047C41900202DE9F04146
:10AAC80086B050238DF81430037A102B074630D106
:10AAD8004368DD7B6DBB0224A8466426062C14D887
:10AAE8007A68535D03932A44517843EA0123039318
:10AAF800927843EA02437343CDE9033863B9684661
:10AB08008DF80040FFF7C2FF0DE0CDF80C808DF8FE
:10AB18001480CDF81080F2E703AB01A801938DF8FB
:10AB28000840FFF75DFF0134E4B2102C05F103057E
:10AB3800D4D106B0BDE8F0811FB502680379116869
:10AB480049B901A88DF80430FFF7A0FF78B10320B8
:10AB580005B05DF804FB02A802928DF80C30FFF7EF
:10AB68003FFF042805D0052805D00028EFD0002095
:10AB7800EEE70220ECE70120EAE70000C90020B96F
:10AB8800034B0B449856C0B27047024BF9E700BF1D
:10AB980025ED0008E5EC0008F0B59A42069D03DBB8
:10ABA8009DF914309A4220DD0020F0BD03EB4303E9
:10ABB80031F814C005EB830300264CFA06F7FF07AB
:10ABC80007D51F7A07F00F0E964502DCB2EB171F68
:10ABD8000DDD0136102E03F10C03EED10134E4B281
:10ABE8002301DBB29842E1D8DEE70024F8E7012030
:10ABF800DBE7884204DB9042CCBF0020012070478D
:10AC08000020704710B51409B4EB111F03464FEA32
:10AC180011100ED391420CD202B201F00F0133F899
:10AC28001240012000FA01F124EA010123F8121070
:10AC380010BD0020FCE7F0B528B100EB4105012765
:10AC48000020914200D3F0BD002435F802CB234602
:10AC580007FA04F636EA0C0608BF013304F10104CA
:10AC680008BFDBB2102CF3D118440131C0B2C9B20D
:10AC7800E7E710B500B149B910BD31F8134020F825
:10AC880013400133DCB2A242F7D8F5E70023F9E715
:10AC980082B030B504880493D2B9B3F5616F15D387
:10ACA80049F6AF2542F21072AB4298BF4FF47A7260
:10ACB800944238BF14466143BDE83040C3688B42B4
:10ACC8008CBF5B1A0023C36002B070476422EFE7B1
:10ACD800012C38BF0124EEE72DE9F04F8FB015465F
:10ACE800199F03939DF8603007930C46804603F044
:10ACF800C7FB6A4A0590A7F5F633303BB3FBF2F37E
:10AD0800534303F5F63B0493182313FB05430BF158
:10AD1800300B069300254FF0FF3A069B9C4207D163
:10AD2800002D14BF50464FF0FF300FB0BDE8F08F34
:10AD3800BDF96830ADF82430099919973846089755
:10AD480003F02EFB2688B8F1000F5FD1B7F5616FCD
:10AD58005AD349F6AF2242F21073974298BF4FF484
:10AD68007A739E4238BF1E46642E59D1DFF830915F
:10AD7800A060A1680CA803F035FB0D9B0093DDE9EA
:10AD880008120C9B0AA803F08CFA039A0A9B0AB9CA
:10AD9800079A2AB122694A4502D1424A93420ED9FA
:10ADA800414BC4F80C909F4209D90023ADF82C30D0
:10ADB8000B99CDF828B0584603F0F2FAA060606805
:10ADC80008B9C4F80C90C4F81090B8F1000F04D07A
:10ADD80003F060FBE3680344E360D4E90332934281
:10ADE800059B88BFE26063601B9BE16873439942DF
:10ADF80004D20398E8B9B8F1000F1AD001231D4412
:10AE08002375EDB2183488E76423AAE7039B0BB9CE
:10AE1800234BE360012EDFF8889038BF0126CEE788
:10AE2800B6F57A7F0ABFDFF88490DFF88490A060D7
:10AE38009FE700209342207506D85B1A9A4505F1D2
:10AE4800010528BF9A46EDB2B8F1000FDAD1642E99
:10AE5800184AADF82C801DD049F6B023B6F57A7F94
:10AE680018BF1346974281BF049A02F5A83202F52B
:10AE7800C0729B180A931A9B00930AAE96E80600C4
:10AE8800199B304603F00DFA96E8030003F088FAA0
:10AE98008246B7E74FF46163E4E700BF80510100E1
:10AEA80040771B007F5101002FEC010080A81201A0
:10AEB800002E930230EC01000378032B14D1437861
:10AEC80003F00F021B098A704B7083788B80C2785D
:10AED80043EA02238B800379C3F3021203F00F03C2
:10AEE800CA700B7005207047002070472DE9F347A2
:10AEF8009A464379057990F907609146044690F996
:10AF080006208846D3B190F90870002D37D00F2A53
:10AF18001BD194F909200F2E27D194F90A00072D87
:10AF280002D1002F08BF012788F8002089F8000007
:10AF380028468AF8007002B0BDE8F08790F90B70D7
:10AF480090F9092090F90A60DFE7A369019394F961
:10AF58001530009394F914302169207BFFF71CFE0B
:10AF68000028D8D105F0FD05D5E794F91D00B042B9
:10AF7800D5DC94F91C30B34203DA05F0FB05304602
:10AF8800D2E73046CBE70000024B03FA00F0B0FBF3
:10AF9800F1F0704740420F004FF4FA53B3FBF0F062
:10AFA800704730B54FF47A750C1F6A4300FB0422D2
:10AFB80052001EBF00F1FF341219B2FBF0F29142A9
:10AFC80038BF1146039A1160820048431CBF013004
:10AFD80040084FF47A71121A01FB1323002BCABFE1
:10AFE80003F2E73393FBF1F1B3FBF1F1049B196032
:10AFF80030BD38B5400014460D46F5F7E3FB014671
:10B008002846F5F72DFB2146F5F72AFBF5F71CFA3C
:10B0180003F0AEFCF5F7F8FA40B238BD2DE9F74F6A
:10B02800019300239C469E46048A1E01F6B2B44250
:10B0380046D906EB46054FEA4309AD0000244768A8
:10B0480037F809702741FF0729D5876807EB050AF4
:10B058007F5927B3077837B9476927B137F8097097
:10B068002741FF071BD59AF8087090F901B047F3FC
:10B0780003084FFA88F8D84511DC47F303177FB265
:10B088005F450CDB9AF8097007EB4708C76807EBC0
:10B09800C8073F7D5FB90CF1010C5FFA8CFC0134E5
:10B0A800102C05F10C05CAD10133DBB2BCE70EF157
:10B0B800010706EB040801F80E805FFA87FEEEE749
:10B0C800019B82F800E083F800C003B0BDE8F08F70
:10B0D8002DE9FF4704464068DDE90C671D468A46AE
:10B0E800914603F0D7F923681B1A3B604FF000081C
:10B0F8000123337085F80080636813B123688342A5
:10B1080024D8D4F81CC0CAF80080A3699CF800E0D1
:10B118000393D4E9030101AB83E80300237D009383
:10B12800DCF80C10237A627A7046FFF7D5FD3346B7
:10B1380038602A46E0694946FFF770FF2B782BB143
:10B14800C7F80080002004B0BDE8F0873378002BF2
:10B158000CBF0C200B20F6E737B590F9002090F9CA
:10B168000250954204460FD0013A52B295420BD094
:10B17800A368019394F9013000936168E0782B4645
:10B18800FFF70AFD0028EFD0104603B030BD884213
:10B19800B8BF08467047000051F82000054B984298
:10B1A80005D0054BC31A584258414000704701204A
:10B1B800704700BF90D0030020A1070005281FB5E5
:10B1C8000ED80C4B53F820300093CDE901120A4BEE
:10B1D80001220021022002F06BFE05B05DF804FB9D
:10B1E800CDE90012054B01220021022002F060FE89
:10B1F800F3E700BF14EE0008A8ED0008C7ED00084B
:10B2080007B5054BCDE9000101220021022002F01B
:10B218004FFE03B05DF804FBE3ED000810B5102203
:10B2280004460021F13000F06BFE0021C4F814112F
:10B238002046F022BDE8104000F062BE02460846F3
:10B24800102100F0A5B92DE9F0430446D0F8140107
:10B2580085B00E46154604F2011988B3C0F11008EE
:10B268009045474628BF1746BAB2484400F034FE16
:10B27800D4F814313B440F2BC4F814312DD9A84508
:10B288002BD204F1F00304F5807113F8012F187C18
:10B298008B4282EA00021A70F7D104F1F1081022F9
:10B2A8004146684600F018FE22466946684600F0A6
:10B2B800F1F910226946404600F00EFE3E44ED1BAF
:10B2C80004F5807804F1F107102D09D8AAB23146A7
:10B2D800484600F001FEC4F8145105B0BDE8F083FB
:10B2E80004F1F003711E13F8012F11F8010F434503
:10B2F80082EA00021A70F6D110223946684600F038
:10B30800EBFD22466946684600F0C4F910226946FA
:10B31800384600F0E1FD1036103DD5E7F0B589B0AC
:10B328000C46102200210546684600F0E9FD224639
:10B338006946684600F0AEF99DF90030002B6A4670
:10B348004FF0000143DA137812F8010F01315B0066
:10B3580043EAD0130F2902F8013CF4D19DF80F30CD
:10B368005B0083F08703D4F81401DBB210288DF852
:10B378000F303BD104F58073694604F5887013F8E3
:10B38800016F11F8012B984282EA06021A70F6D171
:10B3980004F1F00304F5807113F8012F187C8B4237
:10B3A80082EA00021A70F7D110220DEB020004F1B4
:10B3B800F10100F091FD2246294604A800F06AF93F
:10B3C80010220021684600F09BFD09B0F0BD1378FB
:10B3D80012F8010F01315B0043EAD0130F2902F87C
:10B3E800013CF4D19DF80F305B00BCE79DF90030BB
:10B3F800002B6A464FF0000137DA137812F8016F14
:10B4080001315B0043EAD6130F2902F8013CF4D15D
:10B418009DF80F305B0083F08703471CDBB28DF883
:10B428000F30102F04EB0003C0F10F064FF080021D
:10B4380088BF002600F5817083F80121002132467B
:10B4480020443E4403F066FAC4F8146104F580739E
:10B45800694604F5887013F8016F11F8012B9842BA
:10B4680082EA06021A70F6D192E7137812F8016F91
:10B4780001315B0043EAD6130F2902F8013CF4D1ED
:10B488009DF80F305B00C8E70A78037853400370D3
:10B498004A784378534043708A788378534083705E
:10B4A800CA78C3785340C3700A790379534003714B
:10B4B8004A794379534043718A7983795340837138
:10B4C800CA79C3795340C3710A7A037A5340037225
:10B4D8004A7A437A534043728A7A837A5340837212
:10B4E800CA7AC37A5340C3720A7B037B53400373FF
:10B4F8004A7B437B534043738A7B837B53408373EC
:10B50800CA7BC37B5340C373704710B50B7814785C
:10B518006340037054784B786340437094788B7819
:10B5280063408370D478CB786340C37014790B7907
:10B538006340037154794B796340437194798B79F3
:10B5480063408371D479CB796340C371147A0B7AE1
:10B5580063400372547A4B7A634043728B7A947ACD
:10B5680063408372D47ACB7A6340C372147B0B7BBB
:10B5780063400373547B4B7B63404373947B8B7BA7
:10B5880063408373CB7BD27B5340C37310BD0000F1
:10B59800A1F11003DBB2102B2DE9F047044604D8C3
:10B5A8003A4820FA03F3DB0705D4002382F8F03089
:10B5B800FF20BDE8F087561E254615F8013B06F822
:10B5C800013F631B0B4413F0FF00F6D101F11C038C
:10B5D8009B005FFA83FCC3F30313013BDFF8B090D1
:10B5E80082F8F030884653184FF0010EB8FBF1FA94
:10B5F80001FB1A8A1AF0FF0A13F8047C13F8036C8B
:10B6080013F8025C13F8014C30D119F806A019F8A8
:10B61800056019F8045019F807404FEADE1707EBE0
:10B6280047078EEA0A0A07EBC7074FEA4E0EFFB232
:10B638005FFA8EFE87EA0E0E574692F800A087EA58
:10B648000A071F7057787E405E70967875409D7027
:10B65800D57808F104085FFA88F86C40C445DC70B6
:10B6680002F1040203F10403C0D8A2E71829E4D9BF
:10B67800BAF1100FE1D1DFF818A01AF807701AF81C
:10B6880006601AF805501AF80440D6E701010100CF
:10B698002CF000082DE9F04FA3B092F8F0301D917E
:10B6A8001B920193002B00F0538101461EA8FFF75F
:10B6B8002CFF1B9BA74CA84DA84E103302930023C8
:10B6C80003939DF87C0004909DF886000590205C0B
:10B6D80006909DF87B000790205C089004989DF8E0
:10B6E80081C0205C099014F80C000A909DF8800035
:10B6F8000B909DF885009DF878809DF87DE09DF879
:10B7080082A09DF887900C909DF87A00029B1C936C
:10B7180014F80A2014F8093014F8081014F80E70F8
:10B728000D90205C0E909DF87F000F90205C10908B
:10B738000B98205C11900C98205C12909DF8840066
:10B7480013909DF8790014909DF87E001590205C68
:10B7580016909DF883001790205C18901398205C31
:10B7680019901498205C1A9003980130039002985D
:10B77800DDF804B0103002909DF80C00834536D8EF
:10B788008DF878108DF87A2009990E9A8DF87C102A
:10B798008DF882201199069A8DF880108DF87E20F8
:10B7A8001999169A8DF884108DF886200A99189A96
:10B7B8008DF87D108DF887201299109A8DF87B30BE
:10B7C8001B9B8DF881108DF883201A99089A1D9873
:10B7D8008DF885108DF87F201EA903EB0B128DF8CC
:10B7E8007970FFF792FE002023B0BDE8F08F15F8BE
:10B7F80008B082EA03008BEA000016F80EB080EA6F
:10B808000B008DF8780015F80E004B40434016F8F1
:10B818000A0043408DF8793081EA070315F80A10C9
:10B82800594016F80930594016F808308DF87A1042
:10B838007A40534015F8092053408DF87B30089A18
:10B84800069B5340049AAA5C534016F80C205340B8
:10B858008DF87C30DDE908325A4015F80C30534039
:10B86800059AB25C53408DF87D30DDE909325A40C3
:10B87800059BEB5C5340079AB25C53408DF87E30D1
:10B88800069B0A9A5340049AB25C5A40079BEB5CA9
:10B898005A408DF87F200E9B109A53400B9AAA5C51
:10B8A80053400C9AB25C53408DF88030DDE9103279
:10B8B8005A400C9BEB5C53400D9AB25C53408DF898
:10B8C8008130DDE911325A400D9BEB5C53400F9AF1
:10B8D800B25C53408DF88230129A0E9B53400B9AFB
:10B8E800B25C5A400F9BEB5C1C995A408DF8832040
:10B8F800169B189A5340139AAA5C5340149AB25C48
:10B9080053408DF88430DDE918325A40149BEB5CC3
:10B918005340159AB25C53408DF88530DDE91932F1
:10B928005A40159BEB5C5340179AB25C53408DF814
:10B9380086301A9A169B5340139AB25C5340179A52
:10B94800AA5C1EA853408DF88730FFF79DFDB8E626
:10B95800FF2049E72CF000082CEF00082CEE000827
:10B9680008B538B1044A05491060D82200F0B4FA85
:10B97800002008BD0220FCE7C81900205CF500087B
:10B988000A4B1A6870B5002302F1180503EB03147B
:10B998002E5D864204D1183422440A60002070BD0E
:10B9A80001330B2BF2D10320F9E700BFC81900209F
:10B9B8002DE9F041CCB00646DDF8488117461C4613
:10B9C8000D4631B3B8F1000F23D006A8FFF726FCC7
:10B9D800204601A9FFF7D4FF0446B0B9019906A88B
:10B9E8000131FFF72BFC26B11022314606A8FFF7DC
:10B9F8002AFC3A46294606A8FFF725FC06A902A80C
:10BA0800FFF78CFC029BC8F8003020464CB0BDE81C
:10BA1800F0810224F9E7000030B595B013A9044677
:10BA2800FFF7AEFF002830D11B4B0C2101FB00F2C1
:10BA3800D5189A5CA2422AD1139B1A7C1092DA7B01
:10BA48000F929A7B0E925A7B0D921A7B0C92DA7A9D
:10BA58000B929A7A0A925A7A09921A7A0892DA79A1
:10BA680007929A7906925A7905921A790492DA78A5
:10BA780003929A7802925B7801930022AB68009354
:10BA88001146064B022002F013FA15B030BD013002
:10BA98000B28CBD1F9E700BFA4F200082CF100086D
:10BAA80010B40B2B019C03D8019410BCFFF780BF86
:10BAB800032010BC704730B50D4685B014460146CA
:10BAC80068B103AA002000922A460390FFF770FF8E
:10BAD80018B90398001B18BF012005B030BD02201B
:10BAE800FBE72DE9F0430D46BFB014469946804662
:10BAF80020B31BB311F00F0122D1F02201A800F0EE
:10BB0800FFF920466946FFF73BFF044648B900980D
:10BB180001AA10210130FFF73BFD2E46AF1BFFB2F3
:10BB28001EB920463FB0BDE8F08301AA09EB070122
:10BB380008EB0700FFF7AEFD103EEFE70224F0E741
:10BB48000524EEE7F0B5184E3468024685B008467D
:10BB5800002304F1180103EB03154F5D97421ED132
:10BB68000D2A05F1190513D10023CDE90033CDE9DC
:10BB780002330C2210216B46FFF7B3FF04463068EE
:10BB880010226946284400F0A7F9204605B0F0BD08
:10BB980001461022601900F09FF90024F5E70133EF
:10BBA8000B2BD8D10324F0E7C819002009B1FFF7FF
:10BBB800C9BF022070471FB51446A0B10C2A01D195
:10BBC8000B2912D10023CDE90033CDE902330A460F
:10BBD8006B461021FFF785FF18B969462046FFF725
:10BBE800B1FF04B010BD0220FBE70320F9E7F8B568
:10BBF8001E46DDE907479DF818505BB354B34FB3B1
:10BC0800212D29D819462A46204600F065F9012237
:10BC1800631C691EB018FFF764FFF8B9E37ADB0903
:10BC28003B70EBB96319204613F8012C13F8021C7A
:10BC3800120642EA014213F8041C0A4313F8031CD3
:10BC4800012342EA0122291FFFF735FF003818BFF8
:10BC58000120F8BD0220FCE70520FAE70720F8E7F5
:10BC68000420F6E710B5044628B1044B5B699847F1
:10BC78002060002010BD0220FCE700BFBCF30008D4
:10BC880008B5014630B1044B0822186800F024F9C1
:10BC9800002008BD0220FCE7C819002008B530B113
:10BCA800044B0822196800F017F9002008BD02208B
:10BCB800FCE700BFC81900207FB5124E00230446D8
:10BCC80002A801930D46FFF7E9FF33685B6901930A
:10BCD8006CB102AA082312F8011B41B9013B13F009
:10BCE800FF03F8D102A8A04702A8FFF7C9FF35B1A2
:10BCF800019B23B901A8A8473368019A5A6100201B
:10BD080004B070BDC819002008B5014638B1054B0C
:10BD180018680822104400F0DFF8002008BD02204F
:10BD2800FCE700BFC819002008B538B1044B1968F2
:10BD38000822114400F0D0F8002008BD0220FCE7DA
:10BD4800C8190020034B1B6802280CBF19615961F0
:10BD580000207047C819002049B1064B1B68D3E979
:10BD68000423022808BF13460B60002070470220F6
:10BD7800704700BFC819002030B58FB000240546B1
:10BD88000CA80994FFF78AFF9DF8373007939DF8B0
:10BD9800363006939DF8353005939DF8343004937A
:10BDA8009DF8333003939DF8323002939DF831307B
:10BDB80001939DF830300093224621461E4B022005
:10BDC80002F076F80AA8FFF7AFFF9DF82F30079327
:10BDD8009DF82E3006939DF82D3005939DF82C3054
:10BDE80004939DF82B3003939DF82A3002939DF815
:10BDF800293001939DF82830009322460F4B2146A5
:10BE0800022002F055F809A92846FFF7A5FF9DF87A
:10BE1800243003939DF8253002939DF82630019332
:10BE28009DF8273000932246054B2146022002F058
:10BE38003FF80FB030BD00BF88F10008C6F1000818
:10BE480004F2000808B50020FFF7E6FD0120FFF71F
:10BE5800E3FD0920FFF7E0FD0820FFF7DDFD0020E6
:10BE6800FFF78AFF002008BD10B504460B20FFF736
:10BE7800D3FD0C20FFF7D0FD0920FFF7CDFD0820EA
:10BE8800FFF7CAFD0A20FFF7C7FD2046FFF774FF3A
:10BE9800002010BD014B1860704700BFF80000205B
:10BEA8000B4A30B514680B4D43F2390305FB0433D4
:10BEB8001360091A6FF00042B3FBF2F2C2EBC272D0
:10BEC80001319B1A93FBF1F201FB1233184430BD88
:10BED800F80000206D4EC64101380A44914200D155
:10BEE800704711F8013B00F8013FF7E710440A4496
:10BEF800914200D1704711F8013B00F8013DF7E786
:10BF080002F008BD30B530B10A4D01444FF0FF339F
:10BF1800814201D1D84330BD10F8012B534008228B
:10BF280043F30004013A2C4092B284EA5303002AF6
:10BF3800F6D1EDE72083B8ED01207047054B4FF4AB
:10BF480000529A62044B1B6813B15B6803B118472F
:10BF5800704700BF00040048581A0020054B4FF4F2
:10BF680080529A62044B1B6813B1DB6803B118470F
:10BF7800704700BF00040048581A0020012070478D
:10BF88000120704701F03EB901F02CB910B501F05D
:10BF98000FFE0E21044640F61F1001F023F920463B
:10BFA800012101F0EFFDBDE8104001F0CDBA00001D
:10BFB80070B50C4E01EB40030D46B3654FF6FF71AB
:10BFC800002304461A46084601F054FB96F856002A
:10BFD800002101F0D7FD29462046BDE8704001F058
:10BFE8008BBA00BFFC19002010B5044601F0A0FE72
:10BFF80001281CD101F0A4FE34B11248214602F0F8
:10C008000BFB104802F0CEFA0F4C104B00214FF4F6
:10C018008052A1659A6194F8560001F0B3FD6378E7
:10C028006BB16FF07F40BDE8104001F049BA0023C2
:10C0380040F262211A46084601F01CFBDCE7A068C2
:10C048008001F0E7CC190020FC190020000400480A
:10C05800002001F0B5B9000008B501F0BDF80438BA
:10C06800C0B2032896BF024B0020185C08BD00BF71
:10C0780086F3000808B501F0B0FD033008BD01F0F3
:10C088003FB901F0FFB808B501F0F6FC08BD0000A3
:10C0980038B50D46144601F053FB284601F088FDDB
:10C0A8000E21054640F61F1001F09CF82846012194
:10C0B800074D01F067FD01F047FA4FF47A716143CB
:10C0C800284602F0A9FA2846BDE8384002F06ABAC4
:10C0D800E419002001F034BB08B5084B002193F89F
:10C0E800560001F04FFD00234FF4C0711A46084670
:10C0F80001F0C0FABDE8084001F01ABAFC190020A6
:10C1080010B5044601F014FE01281CD101F018FEF8
:10C1180034B11248214602F07FFA104802F042FA80
:10C128000F4C104B00214FF48052A1659A6194F88E
:10C13800560001F027FD63786BB16FF07F40BDE8D2
:10C14800104001F073B9002340F262211A460846F4
:10C1580001F090FADCE7A0688001F0E7CC19002034
:10C16800FC1900200004004808B54FF0040001F055
:10C178000DF9BDE808400220F5F77ABB08B50023A1
:10C188001A461946184601F075FABDE8084001F04C
:10C1980063B900001D4B73B51D4D186000241D4880
:10C1A8006C70C5E90144AC6501F08EFAAC8101F010
:10C1B800F9F92146204601F041FC214604220120DC
:10C1C80001F0F2FA144E154D4FF6FF712346224640
:10C1D800084601F04FFAFFF7C7FF2246104B0094BC
:10C1E8004FF0FF31304602F031F90E4B00942246F1
:10C1F8004FF0FF31284602F029F9304602F084F961
:10C20800284602B0BDE8704002F07EB9581A0020F6
:10C21800FC190020D1D10008E4190020CC19002015
:10C2280045BF000865BF00080128084805D1084B2C
:10C23800C17719700E3001F09DBB437D012B03D1EE
:10C24800034B81751970F5E7704700BFFC19002092
:10C25800FC0000200D4B10B50446187358730120DC
:10C2680000F016F85CB134214FF4E86000F0BAFF32
:10C278004421BDE8104040F2417000F0B3BF1421E2
:10C288004FF4E86000F0AEFF2421F2E7FC1900202B
:10C2980038B5114C0546207001F057FD052D04D81E
:10C2A800DFE805F0090B03171709032001F066FA08
:10C2B8000023637338BD0020F8E7012001F05EFA1F
:10C2C800207B637B8342F5D06073BDE83840FFF77D
:10C2D800C1BF0220EAE700BFFC1900202DE9F043A6
:10C2E8001E4687B000230546CDE901330C461746A4
:10C2F80001F01DFD032D5BD8DFE815F07A00C100C1
:10C308000C010400A27C082A69D8A16801A801F0E0
:10C31800D5FE2168002962D042F210729142E37C76
:10C32800874D50D80322AA7385F83820E96385F829
:10C3380044304FF002086368A17DDB002B820423A0
:10C34800AB74A37CDB00EB7402294FF000032B7560
:10C35800637D02D0227D022A46D103F10F02D2B2B8
:10C36800012A01D9012B3AD1764B774A19680394EF
:10C378004FF0010903A88DF8149001F0D5FC70BBAB
:10C38800287685F817906875FFF762FE4046FFF734
:10C398007FFF6E4801F082FA6D4801F0EBFA01A8C0
:10C3A80000F080FF208A00F051FFA08900F096FF7E
:10C3B800384601F0FDFB624C84F8560001F0BCFCE5
:10C3C800666000200DE04FF00008E963890885F8F1
:10C3D8000E8085F8388085F844302964ABE74FF043
:10C3E800FF3007B0BDE8F083EB7529766A75CBE7B7
:10C3F8002368002BF3D0A27C082AF0D8504DA168FE
:10C4080001A801F05BFE002385F838302268EA6352
:10C41800E27C85F84420A269AB732A646268D20082
:10C428002A820422AA74A27C2B75D200EA74A27D07
:10C43800022A02D0237D022B1CD1627D02F10F0358
:10C44800DBB2012B01D9012AC9D13E4B3E4A1968FA
:10C4580003944FF0010803A88DF8148001F064FCE0
:10C468000028BCD1287685F817806875FFF7F0FD9D
:10C4780000208CE7617DE9752A766B75F6E7304D0B
:10C48800012185F83810227885F85020637885F8DE
:10C498005130A37885F85230E3788B4202D0022BD2
:10C4A80003D03BB985F8533004E00B3A012A29D868
:10C4B80085F853104FF0010885F80E80A388AB83E8
:10C4C800A379AB77E37985F82030237A85F8213092
:10C4D800FFF7BEFD4046FFF7DBFE1C4801F0DEF922
:10C4E8001B4801F047FA95F85130062B40F68900B1
:10C4F8000AD100F087FE00F0FB0140F6890000F049
:10C5080071FE55E70023CDE700F07CFE40F0040102
:10C51800C9B2F2E72368013BB3F57A7FBFF45FAF96
:10C528000320FFF7B5FE0648022380F83830236859
:10C538008364162380F84C30383001F0AFF937E7C0
:10C54800FC190020581A0020E4190020341A002091
:10C558000A1A0020F0B51E4687B00023CDE9013342
:10C56800144607460D4601F0E2FB002C724C16BF3C
:10C57800012300230026637027B1012F7AD0002001
:10C5880007B0F0BDAB68002B00F0D280EB68002B41
:10C5980000F0CE80AA7F082A00F2CA80296901A883
:10C5A80001F08CFD2868003818BF012000F0D6FF84
:10C5B80084F83870AB68E36395F8203084F8443029
:10C5C800686801F057FBA77384F84500EB68DB0047
:10C5D8002382EB7FA374AB7FDB00E37495F82130F3
:10C5E800237595F82230002B3ED12A7D95F824102A
:10C5F800A275022995F8232001D0022B36D102F129
:10C608000F03DBB2012B02D9012A40F091800023ED
:10C618008DF81430494B4A4A1968049503A801F06B
:10C6280083FB002840F0848001232076E375607541
:10C63800FFF70EFD0020FFF72BFE424801F02EF910
:10C64800414801F097F901A800F02CFEA88B00F0F2
:10C65800FDFD288B00F042FE4FF4FA53AA6873439D
:10C66800B3FBF2F3A3608AE7FF22BFE7E275217606
:10C678006375DDE72B8E002B5AD095F83230A86A07
:10C68800012B0CBF2F7DFF27003818BF012000F0B9
:10C6980065FFF0B200F06EFF012184F8381095F8BC
:10C6A8002C2084F8502095F82D3084F8513095F8D6
:10C6B8002E3084F8523095F82F308B4202D0022B5E
:10C6C80003D03BB984F8533004E00B3A012A27D849
:10C6D80084F853102B8EA38395F83230A377012664
:10C6E800AB8E2384A673E777FFF7B2FC3046FFF7DB
:10C6F800CFFD144801F0D2F8134801F03BF994F843
:10C708002130B34240F236700CD100F07BFD00F0CE
:10C71800FB0140F2367000F065FD4FF6FF73A1E7AC
:10C728000023CFE700F06EFD40F00401C9B2F0E746
:10C738004FF0FF3024E700BFFC190020581A0020F2
:10C74800CC190020341A00200A1A00202DE9F04FD5
:10C7580085B082460E9DBDF840809DF844709DF8D6
:10C768004890019193461E4601F0E1FABAF1010F93
:10C77800524C54D0BAF1040F00F09180BAF1000F76
:10C788003AD10B22304684F8442084F838A0E56377
:10C7980001F070FA4FEAC803B9F1000F238241F69D
:10C7A800040363820CBF0123F223E37587F00107BA
:10C7B8000123237684F84500C4F840B084F80EA01D
:10C7C80084F814A06775FFF743FC5046FFF760FD37
:10C7D80004F1380001F062F804F10E0001F0CAF823
:10C7E800374A1068516802AB03C302A800F05AFD2B
:10C7F80040F2FF1000F02AFD019801F0D9F90E214E
:10C8080084F8560040F61F1000F0ECFC94F856002F
:10C8180001F092FA169B636005B0BDE8F08F2949D4
:10C8280084F838A0EAB2895D84F8502076BB0B3DC5
:10C83800012D8CBF00250125053A012A04D8B8F13D
:10C848000C0F38BF4FF00C081F4B9DF83C201B788D
:10C8580084F85350E37701259DF8543084F851103B
:10C8680084F8522084F82130A573A4F81C80A77797
:10C8780084F82090FFF7ECFB2846FFF709FD1348E2
:10C8880001F00CF8124801F075F8B5E7012E04D153
:10C89800A5F10C035D425D41CEE70025CCE750468B
:10C8A800FFF7F6FC022384F8383004F13800162329
:10C8B800A56484F84C3000F0F1FF9DE7FC190020D6
:10C8C800E0EA0008B8F30008FC000020341A002051
:10C8D8000A1A00202DE9F04F87B0DFF8B4B29DF8AE
:10C8E80064A09DF84C90029314469DF854309DF82E
:10C8F8005020BDF84880039205468BF801A0BDF88A
:10C90800446001930F4601F012FABAF1000F18BF04
:10C918004FF00008DFF87CA2039AB9F1000F08BFB6
:10C92800FF22012D8AF8002000F0C880052D48D08C
:10C93800002D40F0C080284600F010FE0B2238463B
:10C948008BF844208BF83850CBF83C4001F092F932
:10C95800019B8BF8450041F60402002BABF812202E
:10C968009AF800208BF816200CBF0122F2228BF8CF
:10C978001720F600012289F001098BF818208BF89E
:10C988000E50ABF810608BF814508BF81590FFF729
:10C998005FFB2846FFF77CFC0BF1380000F07EFFB8
:10C9A8000BF10E0000F0E6FF7B490868496804AA0D
:10C9B80003C204A800F076FC40F2FF1000F046FC29
:10C9C80071E0012000F0CAFD09224FF000098BF840
:10C9D800442038464FF44872CBF840208BF8389002
:10C9E800CBF83C4001F046F94FF48052ABF81220E6
:10C9F8009AF800208BF845008BF81620284601226B
:10CA0800F6008BF817208BF80E90ABF81060ABF897
:10CA180014908BF81890FFF73BFC0BF1380000F0EE
:10CA28003DFF0BF10E0000F0A5FF5B498868C9685F
:10CA380004AA03C204A800F035FC40F2FF1000F07D
:10CA480005FC40F6B80000F0DDFB00F0EF0140F611
:10CA5800B80000F0C7FB042140F6B90000F0C2FBA3
:10CA680040F69B0000F0CEFB00F0E30141F0080126
:10CA780040F69B0000F0B6FB40F2D16000F0C2FB2C
:10CA880040F01801C9B240F2D16000F0ABFB40F2AF
:10CA9800AC6000F0B7FB00F08F0141F0500140F2AC
:10CAA800AC6000F09FFB4FF4FA5202FB08F2B2FBB5
:10CAB800F4F2CBF8082007B0BDE8F08F002000F0B2
:10CAC8004DFD36498BF83850E2B2C95D8BF85020DD
:10CAD800002F4DD10B3C012C8CBF00240124053ABA
:10CAE800012A02D80C2E38BF0C26029B9AF8002087
:10CAF8008BF852308BF85340019B8BF81F20012490
:10CB08009DF860208BF821208BF851108BF820308D
:10CB18008BF80E40ABF81C608BF81E90FFF798FA64
:10CB28002046FFF7B5FB1E4800F0B8FE1D4800F090
:10CB380021FF5FFA88F000F01DFD40F6A30000F029
:10CB480061FB00EA040140F6A30000F04BFB9BF8F0
:10CB58002120A24240F2367013D100F053FB00F0BE
:10CB6800FB0140F2367000F03DFB4FF6FF72A0E784
:10CB7800012F04D1A4F10C035C425C41AFE700240F
:10CB8800ADE700F03FFB40F00401C9B2E9E700BFA0
:10CB9800FC190020FC000020E0EA0008B8F30008B7
:10CBA800341A00200A1A0020F0B58BB00D4604464E
:10CBB80017461E46FFF74CFA0020FFF769FB204690
:10CBC80000F0BEFD00240123CDE9084303234FF400
:10CBD800167229462046CDE90644CDE90444CDE93C
:10CBE8000244CDE900532346FFF774FE2046FFF7C1
:10CBF80087FAFFF73FFAF4F73BFE01F041FC0446E1
:10CC0800204601F047FCB04205D30124FFF720FA83
:10CC180020460BB0F0BD00F02FFF8742F0DA002469
:10CC2800F4E70000F7B500230C4640F201211A464C
:10CC38000646084600F01EFD644B654D4FF4005251
:10CC48009A6195F85600012100F09CFF2B78012B82
:10CC580040F6890013D195F85130062B0FD100F01A
:10CC6800D1FA00F0FB0140F6890000F0BBFA2B78FE
:10CC7800042B6CD8DFE803F0524B527F090000F018
:10CC8800C1FA40F00401C9B2EDE7524A731E1046DA
:10CC9800C6F101074FF0000CF9188C426FDC002236
:10CCA800E7001346BA4271D19A0142EAC3125B0106
:10CCB80083F020031343661C0355F6B2022346484B
:10CCC800AB73AE7600F056FE0021F12000F08AFA30
:10CCD8000021F02000F086FAAB6C642B70D1702133
:10CCE800F32000F07FFA1D21F22000F07BFAE1002A
:10CCF8008C1CF420090A00F075FA04F0FE01F520F6
:10CD080000F070FA33486FF07F4231461DE0EC774F
:10CD1800314800F02FFE0022214615E001F008F806
:10CD28000128074625D121460DF10702304601F0BA
:10CD380004F80446A0B99DF807302748AB7500F001
:10CD480019FE9DF807102246304600F065FB696819
:10CD5800224801F061FC214801F024FC002006E093
:10CD68001F4B3A460021022001F0A2F8032003B02D
:10CD7800F0BDAC75CCE70223AB73AC76C8E713F80B
:10CD8800011FC943197002F801CB85E7D1106FEA7A
:10CD9800020C715C0CF0070C013241FA0CF101F045
:10CDA80001014FEAE20C4B40D14310F80CE001F0CE
:10CDB800070103FA01F141EA0E0100F80C1071E7CE
:10CDC800E121F32000F00EFA04218DE70004004869
:10CDD800FC1900205C1A00200A1A0020E41900201F
:10CDE80028F30008F0B5BDF814409DF818709DF8B8
:10CDF8001CE09DF8205040B1012814D001220023E6
:10CE080098180138B0FBF2F0F0BD87F00107E30095
:10CE180003EBC70318330EEB450503EBC5034FF4CB
:10CE28007A714B43ECE7501F012803F1040302D841
:10CE38000C2C38BF0C24D1B9A2F10B0CBCF1010F9A
:10CE48008CBF4FF0000C4FF0010C2801002F00EBB5
:10CE5800CE000CBF14250025A0EB8200062A4FEA5D
:10CE680082062844A2F102070DD8354610E00129B0
:10CE780006D1A2F10C00D0F1000C4CEB000CE4E759
:10CE88004FF0000CE1E70830BCF1000FEDD0BD0019
:10CE98000028ACBF2E182E1C701E90FBF5F003FB6B
:10CEA8000044094B062A5A5C8CBF0C340E340A2AFB
:10CEB80009D8A30001334FF47A71BB404B430349AF
:10CEC80051F822209CE7FFDEB8F300088CF3000835
:10CED80008B5094B012193F8560000F053FE4FF4B2
:10CEE800D7602D2100F07EF900F033FBBDE8084043
:10CEF800024800F07BBA00BFFC190020FFFF0F00BA
:10CF080073B5A44CB4F854300025202B8DF8035089
:10CF1800019500F01B8114D8082B0DD87BB1013B7B
:10CF2800072B0CD8DFE813F042005B000B00CD00A4
:10CF38000B000B000B00FD00102B00F0008102B06D
:10CF480070BDB3F5807F00F0988011D8402B00F0B9
:10CF58001081802BF3D1284600F032FA8E4B1B68E3
:10CF6800002BECD09B69002BE9D028469847E6E7D0
:10CF7800B3F5007FE3D1894B01222946022000F056
:10CF880097FF00F029F9042840F08580844B8548F4
:10CF98004FF400529A6201F0B7FA284600F010FAEE
:10CFA8007D4B1B68002BCAD05B6814E07C4B7D4826
:10CFB8004FF400529A6201F0A7FA002000F000FA3C
:10CFC80000F0B8FE012801D100F0BDFE724B1B68CD
:10CFD800002BB4D01B68002BB1D09847AFE7704B3B
:10CFE80071484FF480529A6201F08EFA657895B9CB
:10CFF800284600F0E5F9294640F6021000F0F2F85C
:10D0080040F6441000F0FEF840F00201C9B240F6C4
:10D01800441000F0E7F8FF220DF1030163485E4D6C
:10D0280000F05AFD624800F071FD2B68002B86D095
:10D038009E68002E83D094F82430012B08D194F9EF
:10D04800313094F930209DF803105848B04776E7FE
:10D05800E06B01A900F022FE019B9DF803105348E4
:10D068004FF47A7203F5FA7393FBF2F32A685BB212
:10D07800956894F92920A84761E7284600F0A0F9A7
:10D08800454B1B68002B3FF45AAF9B69002B3FF4BC
:10D0980056AF01206AE700F09FF805287FF44FAFEC
:10D0A8003F4B41484FF480529A6201F02DFA2846CE
:10D0B80000F086F9384B1B68002B3FF440AFDB6863
:10D0C80089E700213B4B0122022000F0F1FEA16D0F
:10D0D80000293FF434AFC1F3074140F6031000F0D4
:10D0E80081F894F8591040F6041000F07BF894F891
:10D0F800581040F6051000F075F840F6021000F0E0
:10D1080081F840F00101C9B240F6021000F06AF857
:10D11800002340F262211A460846A36500F0AAFAE5
:10D128000DE7254B01220021022000F0C1FE00F08E
:10D13800FFFD01287FF403AF00F006FEFFE61F4B5A
:10D1480001220021022000F0B3FEF8E6164801F0A3
:10D15800DBF9607808B900F033F90F4B1B68002B36
:10D168003FF4EDAEDB68002B3FF4E9AE9847144B73
:10D17800E6E7144B01222946022000F099FE607868
:10D1880008B900F01DF9044B1B68002B3FF4D7AE1B
:10D198001B6920E7FC190020581A00203DF30008FD
:10D1A80000040048E4190020CC1900205C1A002073
:10D1B800201A002051F300085AF3000864F300080D
:10D1C8006DF3000876F30008024BA3F85400FFF74C
:10D1D80097BE00BFFC190020014B1878704700BFAC
:10D1E8006A1B002007B501238DF807100DF107020F
:10D1F80001460348F7F748FA03B05DF804FB00BF9F
:10D20800C401002007B5012301460DF107020448B7
:10D21800F7F773FA9DF8070003B05DF804FB00BF49
:10D22800C401002010B50446F5F778F801280CD1A0
:10D2380040F62310FFF7E6FF00F0F901214340F61E
:10D248002310BDE81040FFF7CDBF10BD10B50C4B43
:10D258001B7804469BB94FF4D760FFF7D3FFC4F39C
:10D26800002100F0FE0001434FF4D760FFF7BAFF3A
:10D27800E1B240F2B960BDE81040FFF7B3BF10BD9E
:10D28800691B002010B51346EFF3108472B60A46E6
:10D2980001460348F7F7F8F984F3108810BD00BF7A
:10D2A800C401002008B5014608224FF4D860FFF7F2
:10D2B800E9FF002008BD000007B5074B1B7840BAFE
:10D2C800ADF804002BB9022201A940F2BC60FFF7B7
:10D2D800D9FF03B05DF804FB691B002007B5074BB5
:10D2E8001B7840BAADF804002BB9022201A940F21C
:10D2F800BE60FFF7C7FF03B05DF804FB691B0020A1
:10D3080010B51346EFF3108472B60A460146034877
:10D31800F7F7F3F984F3108810BD00BFC4010020AB
:10D3280010B51346EFF3108472B60A460146034857
:10D33800F7F7D5FA84F3108810BD00BFC4010020A8
:10D348000A4601460020FFF7EBBF000010B5134660
:10D35800EFF3108472B60A4601460348F7F7F2FA6B
:10D3680084F3108810BD00BFC401002010B5134617
:10D37800EFF3108472B60A4601460348F7F7F8F946
:10D3880084F3108810BD00BFC401002013B5044603
:10D398000020F4F79DFF0220FFF744FF04F0070484
:10D3A80001220DF1070184208DF80740FFF7DEFF09
:10D3B800024B00221A7002B010BD00BF6A1B002089
:10D3C80007B501228DF807000DF107018020FFF74E
:10D3D800CDFF9DF80730002B034B14BF022201221A
:10D3E8001A7003B05DF804FB6A1B002007B5094BEF
:10D3F8008DF8060004221A70030C8DF804300322FD
:10D40800030A01A983208DF80530FFF7AFFF03B0A9
:10D418005DF804FB6A1B002010B51446FFF790FF67
:10D428002046BDE81040FFF7E1BF000007B5094BF3
:10D438008DF8060005221A70030C8DF804300322BB
:10D44800030A01A982208DF80530FFF78FFF03B08A
:10D458005DF804FB6A1B002073B5002640F6E20065
:10D468000196FFF7CFFE00F0FE01054640F6E20008
:10D47800FFF7B8FE40F6E500FFF7C4FE00F07F01B5
:10D48800044640F6E500FFF7ADFE6FF07F40FFF77A
:10D49800CDFF04220DEB020140F61900FFF730FF23
:10D4A8003046FFF78DFF294640F6E200FFF79AFE67
:10D4B800214640F6E500FFF795FE019802B070BDE1
:10D4C80013B50C4B04460522972140F6AC001A70A0
:10D4D800FFF788FE230C8DF804300322230A01A9E4
:10D4E80082208DF805308DF80640FFF73FFF02B027
:10D4F80010BD00BF6A1B002007B5030C8DF8003073
:10D50800030A8DF801300B0C49BA8DF80200ADF80A
:10D5180004100622694694208DF80330FFF726FF91
:10D52800024B06221A7003B05DF804FB6A1B002048
:10D53800002208B51146C520FFF718FF014B072246
:10D548001A7008BD6A1B002000221146D120FFF77F
:10D558000DBF00221146D220FFF708BF07B50122F0
:10D568008DF807000DF107019F20FFF7FFFE03B0BC
:10D578005DF804FB07B501228DF807000DF10701DE
:10D58800A020FFF7F3FE9DF807103F2907D901F007
:10D59800F8010131C9B240F20670FFF723FE03B06B
:10D5A8005DF804FB07B5F4F7B9FE431E584258412D
:10D5B8008DF8070001220DF107019620FFF7D6FE2E
:10D5C80003B05DF804FB07B500F07F008DF8070095
:10D5D80001220DF107018920FFF7C8FE03B05DF8AD
:10D5E80004FB0000154B984207B51BD8144B984212
:10D5F8001BD8144B98421BD8134B98421BD8134B7B
:10D6080098428BBF6B2229226F232B238DF804208D
:10D6180001A9022298208DF80530FFF7A7FE03B074
:10D628005DF804FBE122E923F0E7D722DB23EDE7ED
:10D63800C122C523EAE775228123E7E700E9A4357B
:10D6480080F8A9328044E52D000B6B1B40FC54196F
:10D6580007B58DF8062004228DF804008DF8051012
:10D6680095200DEB02018DF80730FFF77FFE03B020
:10D678005DF804FB07B552BAADF8042040BA082299
:10D6880049BAADF80000ADF802105BBA6946104619
:10D69800ADF80630FFF76AFE03B05DF804FB07B586
:10D6A8000B0C042200F0070049BA8DF80400ADF80D
:10D6B800061097200DEB02018DF80530FFF756FE96
:10D6C80003B05DF804FB000010B508B1194B1860F1
:10D6D800F3F7D2FF0220FFF7A5FD0024164B2046E2
:10D6E8001C70FFF76DFEF4F717FE012817D14FF4F1
:10D6F8002071FFF7D4FF40F611102146FFF772FDA5
:10D708004FF07F00FFF75FFF0E2140F61F10FFF775
:10D7180069FDF4F7A9FD094B01221A7010BD10210B
:10D7280040F61110FFF75EFD102140F61210FFF7CA
:10D7380059FDE9E75C1B0020601B00206A1B0020E4
:10D7480037B50C4D2B7804461BB9FFF74BFF012367
:10D758002B700023084A6006E109F3F721FA042236
:10D7680000BA01900DEB02018620FFF7FFFD03B020
:10D7780030BD00BF601B00200048E80107B5094B19
:10D788008DF807000146187018B940F2AC60FFF731
:10D7980029FD01220DF107018A20FFF7E7FD03B0FB
:10D7A8005DF804FB691B0020012873B50C4616467A
:10D7B80037D10020F4F7B4FDA042B8BF44B20E2818
:10D7C80005461AD101231A4600210420FFF740FF1D
:10D7D8006FF010039C42B8BF1C46182140F6E700C2
:10D7E800FFF700FD022201A98E208DF804408DF874
:10D7F8000560FFF7BBFD02B070BD01230A28E4B243
:10D808001A464FF0000105D11846FFF721FF0334EF
:10D8180064B2DDE70720C5F10E05FFF719FF2C44B8
:10D82800F6E740F6D800FFF7EDFC40F01E01C9B25C
:10D8380040F6D800FFF7D6FC0120F4F771FDA042AE
:10D84800B8BF44B2142805464FF001034FF0000258
:10D858000CD105210320FFF7FBFE023464B26FF000
:10D8680008039C42B8BF1C463821B7E7112805D1E8
:10D8780003210220FFF7ECFE0534EFE70E2804D160
:10D8880002210846FFF7E4FEE9E7C5F1160507217E
:10D8980004202544FFF7DCFE6CB2E0E713B5314AFB
:10D8A8000446516810686B4603C32F4B20781B78D9
:10D8B800834201D0FFF762FF2378032B27D8DFE8E4
:10D8C80003F00239283C6268284BB3FBF2F31A0CC8
:10D8D800A1688DF800208DF802301A0A237B8DF894
:10D8E8000330637B8DF801208DF80430204A002333
:10D8F8004806C909F3F754F9030C40BA8DF8053006
:10D90800ADF80600082269468B20FFF72FFD02B00C
:10D9180010BD2269154BB3FBF2F31A0C8DF80020E9
:10D928008DF802301A0A237D8DF801208DF8033016
:10D938000422E8E7A3690093FAE762680B4BB3FB9C
:10D94800F2F31A0C8DF800208DF802301A0A237BA6
:10D958008DF80330637B8DF801208DF804300522A3
:10D96800D1E700BFF0EA0008691B00200000093D6C
:10D978000048E8011FB52E4A0446D1689068127C19
:10D9880001AB03C31A702B4B20781B78834201D05C
:10D99800FFF7F4FE2378032B26D8DFE803F00238DC
:10D9A8003302637AF12B21D14FF6FF70FFF784FC25
:10D9B80048F20500FFF792FC02236288A188ADF8BF
:10D9C800061052BAE188ADF804208DF80B30227A9F
:10D9D800A37A8DF80A20ADF808108DF80C300922CA
:10D9E80001A98C20FFF7C2FC04B010BDF22BE4D1D2
:10D9F80041F60F50FFF760FC41F22100FFF76EFC83
:10DA08000623DAE7237B8DF804300122E8E7E3896F
:10DA1800094A5BBAADF80430237C13708DF80630E0
:10DA2800637C8DF80730638AADF808300622D7E7A3
:10DA3800F0EA0008691B0020681B002007B50222D5
:10DA48008DF804008DF805108F2001A9FFF78EFCD2
:10DA580003B05DF804FB000010B51346EFF3108423
:10DA680072B60A4601460348F6F7BAFE84F31088F0
:10DA780010BD00BFC401002007B5012201A915206F
:10DA8800FFF7EAFF9DF804004042401003B05DF83C
:10DA980004FB000037B505460C46022201A91320F5
:10DAA800FFF7DAFF0A4B1B78012B0DD1094B1B78C6
:10DAB800012B09D140F20270FFF7A4FB9DF8053055
:10DAC8002870237003B030BD9DF80400F6E700BF4E
:10DAD800691B0020681B0020F7B50D460646002488
:10DAE8000DF10701284617468DF80740FFF7D2FFCA
:10DAF8002A78BA4207D89DF807003146FFF726FC76
:10DB0800204603B0F0BD0120FBE7000013B5032257
:10DB1800044601A91420FFF79FFF184B1A782270BA
:10DB28004AB1012A17D014220021204600F0D0FA69
:10DB38000F2323700DE09DF8043023719DF8053004
:10DB4800A2605B425B10A3719DF806305B425B10DC
:10DB5800637102B010BD9DF804305B425B10237303
:10DB68009DF9053002339B1063739DF806305B42C4
:10DB78005B10A373024B1B682361EAE7691B002053
:10DB8800641B0020012908B5034608460ED1012B65
:10DB980007D10420FFF746FB0220BDE80840F4F750
:10DBA80097BB022B14BF08460320F6E70120F4E7D1
:10DBB80038B50446F4F7AEFB50B102280CBF022575
:10DBC8000125284602222146FFF7EEFD284638BDEA
:10DBD800102CB4BF01250225F3E70A207047000086
:10DBE800014B01201B6818475C1B0020014B0220D9
:10DBF8001B6818475C1B0020014B40201B68184716
:10DC08005C1B002011B1012904D07047044B1B682C
:10DC180080201847024B4FF480701B68F9E700BF5B
:10DC28005C1B0020024B4FF400701B68184700BFB4
:10DC38005C1B0020014B20201B6818475C1B002040
:10DC4800014B04201B6818475C1B0020014B08206F
:10DC58001B6818475C1B0020014B10201B681847E5
:10DC68005C1B0020024B4FF480401B68184700BF24
:10DC78005C1B002010B568B1074A002352F83340F6
:10DC8800844202EBC30101D9087910BD0133162B78
:10DC9800F4D1FEE71F20F8E748F4000873B51D4BE0
:10DCA8000193044640F607000D46FFF7ABFAC0F3B0
:10DCB800C10308336B4413F8042C00F00703013345
:10DCC80002FA03F3144AB2FBF3F2B2FBF4F00728AA
:10DCD8001ED84000042834BF042302234FF4D66022
:10DCE80002FB03F4FFF78EFA060240F2B160FFF779
:10DCF80089FA06F470663043030544BF6FEA0050A2
:10DD08006FEA105063094343DB112B6002B070BD0A
:10DD18000123E3E704080A0C0048E8014FF0FF304C
:10DD280070474FF0FF3070474FF0FF307047704733
:10DD3800002070470020704770474FF0FF30704751
:10DD48004FF0FF30704770477047704770B5EFF37A
:10DD5800108672B6144B5C8A1A8A944213D1C4F5A1
:10DD6800806292B2904206D3844218D901229A70F6
:10DD780000221C805A825A8A0A800244C2F309028D
:10DD88005A8200200DE006D9C4F58065ADB28542FF
:10DD9800F1D88242E9E7121B92B28242EBD84FF0E7
:10DDA800FF3086F3108870BD6C210020EFF31081DE
:10DDB80072B6034AD38A0133D38281F3108870473D
:10DDC8006C210020EFF3108172B6034AD38A013B1D
:10DDD800D38281F3108870476C21002010B5084861
:10DDE8001822002100F074F906484FF480620021DF
:10DDF80000F06EF9044B05481B68BDE81040184751
:10DE08006C2100206B1D002068EB000881DF0008F2
:10DE1800014B5860704700BF6C210020014B1872FD
:10DE2800704700BF6C21002073B5EFF3108572B600
:10DE38001C4CE08A00282FD1FFF7B8FF218A628A9C
:10DE4800914227D0A378012B12D1238820805B1A16
:10DE58009BB20221A382A17063B9A3702382238A93
:10DE68009A428BBFD21AC3F58063A282A38201E0D3
:10DE7800002BF4D0268A0C4B1E4485F31088F3F748
:10DE8800E5FC0A4BA18ADB680193304602B0BDE885
:10DE980070401847FFF796FF85F31088002002B0FE
:10DEA80070BD00BF6C2100206B1D002068EB0008CE
:10DEB80008B4F0B586B00023ADF800302B4B0B9CAE
:10DEC8001D7A85424CD3D86881434CD15B681BB11D
:10DED80012B1694602A898470CAB22464FF400716C
:10DEE8002348019300F0F4FBFFF760FFBDF8003012
:10DEF80018440DF1020180B2FFF728FF01302AD043
:10DF08000023BDF80020BDF802601A480DF1080C86
:10DF18001F4699B216FA83F58A42ADB215D817B1E1
:10DF28003244ADF80220BDF80250019B22464FF45E
:10DF38000071284400F0CCFBFFF744FFFFF774FFA3
:10DF480006B0BDE8F04001B070471CF8011B415510
:10DF580001330127DDE7FFF735FF6FF00200EFE738
:10DF68006FF00400ECE76FF00500E9E76C21002092
:10DF78006B1B00206B1D002013B5EFF3108472B6E5
:10DF8800204B9A78588A022A1DBF1A8A998A5218F1
:10DF9800002214BFC2F309029A7090421A8228D054
:10DFA800D98A012925D19978012913D119888A1A82
:10DFB800022192B2997000219A82198062B99A70EE
:10DFC8001A821A8A90428BBF801AC2F580629882A0
:10DFD8009A8201E00029F4D0188A0B4A104484F38D
:10DFE80010880A4A998AD368019302B0BDE81040A4
:10DFF800184784F31088F3F72DFC02B0BDE81040F1
:10E00800FFF7E0BE6C2100206B1D002068EB0008C4
:10E01800024A00231360024A1360704788210020D7
:10E028008421002010B5EFF3108472B641B10129A4
:10E0380003D1064A13680343136084F3108810BDA4
:10E04800024A136823EA0003F6E700BF882100208C
:10E0580010B5EFF3108472B641B1012903D1064A15
:10E0680013680343136084F3108810BD024A1368D1
:10E0780023EA0003F6E700BF8421002038B5EFF358
:10E08800108572B60A4B0B4C1B6833B1236898474E
:10E098006368984785F3108838BD074B1B681BB128
:10E0A800A3689847E368F4E7236998476369F0E74A
:10E0B8008821002004EB00088421002001380A444C
:10E0C800914200D1704711F8013B00F8013FF7E792
:10E0D80000F020BC10B5EFF3108472B6064A13683E
:10E0E80003431360054A52F83130034342F8313094
:10E0F80084F3108810BD00BFB02100208C210020BF
:10E1080070477047B0F5803F3ABF000410230023E2
:10E11800B0F1807F3EBF08330002DBB2B0F1805F10
:10E1280038BF00014FEA1070054A38BF0433125C4B
:10E1380038BFDBB2C3F11F03981AC0B2704700BFE3
:10E14800F8F400082DE9F84F384D394ED5F800801D
:10E15800DFF8E0B0DFF8E0A0DFF8E090D6F800C024
:10E16800374FDBF80010374CDAF80020D9F80030C8
:10E1780008EA00002860286800EA020E1EEA0C0F70
:10E1880001D019421ED04FF0FF333B60FFF7B8FFB4
:10E19800EFF3108472B63368DBF80020DAF8001069
:10E1A8000B4029680B4205D1D9F80030134201D140
:10E1B800F3F7DAFA84F31088FFF7A3FFC5F80080B5
:10E1C800BDE8F88F236823680340134062681A4249
:10E1D80004BF4FF0FF32626060681840FFF792FF9B
:10E1E80062683860012303FA00F022EA00026260E4
:10E1F800EFF3108172B63A689340326822EA03025C
:10E208003260226822EA0303236081F310880E4AF1
:10E218003B6852F823309847D6F800C0DBF8001066
:10E22800DAF80020D9F80030A5E700BF0001002087
:10E23800B0210020AC21002004010020A8210020EA
:10E24800A42100208C2100209421002010B5114623
:10E25800EFF3108472B6FFF755FF034B43F8201015
:10E2680084F3108810BD00BF9421002082B082B0D2
:10E278000DF1080C0CE90600BDF8042003930B44CB
:10E28800BDF810100A4491B212B2B2F57A7FA2BF5B
:10E29800A1F57A72013312B20360828002B002B033
:10E2A800704782B082B00DF1080C0CE90600BDF889
:10E2B80004200393CB1ABDF81010521A91B212B26F
:10E2C800002ABEBF01F57A7203F1FF3312B2036070
:10E2D800828002B002B0704730B585B0114D6B46F0
:10E2E80083E8030000230293ADF80C3003A82B69E0
:10E2F8009847009BBDF804400290181ABDF80C30EE
:10E30800E41AA3B224B2002CBEBF03F57A731CB280
:10E3180000F1FF302B689847AB682046984705B056
:10E3280030BD00BF28EB000873B5114E0023054629
:10E338000093ADF8043001A833699847F36800905A
:10E348009847736804469847009B1844BDF8043002
:10E3580023449AB21BB2B3F57A7FA2BF0130A2F56B
:10E368007A731BB228602846AB8002B070BD00BF2C
:10E3780028EB000837B500230093ADF80430074BAD
:10E3880004461B6901A898476D46009095E803006C
:10E3980084E80300204603B030BD00BF28EB000826
:10E3A80037B50F4D02AB03E90300EB6898476B687C
:10E3B80004469847BDF80430009A1B1B99B21BB25B
:10E3C800002BA2EB0002BEBF01F57A7102F1FF3209
:10E3D8000BB24FF47A7000FB023003B030BD00BFBF
:10E3E80028EB00082DE9F0414FF47A75B1FBF5F5FB
:10E3F800C5EB4513DFF83C8005EB8303A1EBC303B2
:10E408009CB2D8F80C3006469847D8F8043007462E
:10E418009847E31999B21BB2B3F57A7F2844A2BF93
:10E42800A1F57A7301301BB23060B3803046BDE885
:10E43800F08100BF28EB0008024B00221A60024B53
:10E448001B681847B42100203CEB0008F8B50446C7
:10E45800174608461E467CB173B1084B00255B6A17
:10E4680025609847069B60602581A572E660236158
:10E47800E77265612846F8BD0120FCE73CEB00081F
:10E4880010B5034CE3699847A36ABDE810401847E4
:10E498003CEB000870B5064DEB69064698476B6A79
:10E4A800044630469847AB6A201ABDE870401847C2
:10E4B8003CEB0008054B1B680BB9184670478342B4
:10E4C80001D05B69F8E70120704700BFB421002044
:10E4D8002DE9F3410B4E336A044698470123B76987
:10E4E8002372D4F800800546B8472844804502D2F4
:10E4F800B84728442060B3682068019302B0BDE89B
:10E50800F04118473CEB000870B520B3EFF31086D4
:10E5180072B6124D2B680122827253B100224272E8
:10E5280098425C690ED102723CB120462C60FFF71C
:10E53800CFFF86F31088002070BD094BDB68984731
:10E548002C60F6E71A465B69002BF2D09842F9D1A5
:10E5580043695361EDE70120EEE700BFB4210020D5
:10E568003CEB0008084B10B51A685369516911B99A
:10E578005061416110BD046819688C4202D91A467D
:10E588005B69F3E71946F3E7B4210020044A1368EE
:10E598000BB10021197243611060FFF799BF00BFEA
:10E5A800B42100202DE9F041044600282DD0FFF7C2
:10E5B80081FF50BB657A45BBEFF3108872B6144EE5
:10E5C8006768336A984787422CBF27602060114FDD
:10E5D800A5724FF4807323813B684BB93369984720
:10E5E8002046FFF7D3FF88F310882846BDE8F0815E
:10E5F800B3699847236818443B6820601B689842B1
:10E608002046EED3FFF7AEFFEDE70125EDE700BFAB
:10E618003CEB0008B421002010B5044608467CB144
:10E62800084B5B6A984760602046FFF743FF40B19C
:10E638002046FFF769FF2046BDE81040FFF7B2BF4C
:10E64800012010BD3CEB00082DE9F041EFF31087E5
:10E6580072B61D4E1D4D7369984733690446984735
:10E668002B684BB94FF000082B688BB9286828BB7A
:10E6780087F31088BDE8F081011B241A1A688A42C2
:10E688008CBF121900221A605B69002BF6D1E9E7EA
:10E698001C681CB1B36998478442E7D22C68636947
:10E6A8002B60A4F80880D4E9033098476389B3F550
:10E6B800807FD9D12046FFF775FFD5E7037A002B75
:10E6C800D6D1FFF705FFD3E73CEB0008B4210020C3
:10E6D8002DE9F04F002997B081461E4640F311817D
:10E6E80004464F1E1378A4EB090023B900232370B6
:10E6F80017B0BDE8F08FB842F8DA252B05D004F83A
:10E70800013B904608F10102ECE792F801E0AEF116
:10E71800300102F10108AEF130034A424A41092BA7
:10E728002BD8414600250A20884611F8013BA3F161
:10E73800300CBCF1090F1BD998F80030692B00F098
:10E748009E801DD8632B29D0642B00F09880582B0D
:10E758005AD0252B1AD198F80030002B00F093805E
:10E7680004F8013BA4EB0903BB4280F28A80C9E7A5
:10E7780000FB0533A3F13005D6E74FF0FF35DBE7A3
:10E78800752B7ED0782B41D0732B1CD0252304F811
:10E79800013BA4EB0903BB4273DADCE7002D05F16A
:10E7A800FF3AD8BF4FF0000A52462046202100F019
:10E7B800B1F8A244002D56F8043B8AF80030D8BFBF
:10E7C80001252C449EE7504B56F804BBBBF1000FC3
:10E7D80008BF9B465846F1F7CBFC2A1A8542B8BFBA
:10E7E8000022824620212046019200F093F8019AE7
:10E7F80000232244534502DB02EB0A0482E71BF89C
:10E808000310D1540133F5E742F040021021DFF83C
:10E81800FCB0DFF8FCA056F804CB12F0400F18BF8C
:10E82800DA46BEF1300FCDF808A0A4EB09030CBFFF
:10E838004FF0300A4FF0200A9207A7EB0303604617
:10E84800CDF80CA022D5002820DA4042013D4FF037
:10E858002D0C05AA019200228246B0FBF1F001FBC3
:10E8680010AB029810F80BB0019800F801BB5145A5
:10E87800019002F10102BAFBF1F0EDD910E042F08B
:10E8880002020A21C3E708F1FF386BE7BCF1000F69
:10E8980002D04FF0000CDCE730228DF81420012262
:10E8A800BEF1300FA5EB020504D02020002D05F1A4
:10E8B800FF350ADCBCF1000F05D02D21013B04F81F
:10E8C800011B3FF41FAF25440AE0013B04F8010B8C
:10E8D800ECD117E7039904F8011B013B3FF412AF91
:10E8E800291B0029F6DC05A9114423442244A2422D
:10E8F8003FF408AF11F8010D04F8010B9C42F6D162
:10E9080000E70020F4E600BF08F5000834F5000829
:10E918000FF5000802440346934200D1704703F8FC
:10E92800011BF9E770B50D4D0D4C641BA4100026B2
:10E93800A64209D10B4D0C4C00F09AF8641BA410A8
:10E948000026A64205D170BD55F8043B984701360C
:10E95800EEE755F8043B98470136F2E73CF6000825
:10E968003CF600083CF6000840F6000800000000ED
:10E978002DE9F041C1F30A57A7F2FF36132E0246DC
:10E988000B460C460546804635DC002E17DA34A3C4
:10E99800D3E90023F1F7FAFB00220023F1F72AFE5E
:10E9A80050B1002C57DA24F000442C430025AC4227
:10E9B8002D4C08BF4FF0004423462A4624E02B4F35
:10E9C800374101EA070C5CEA000C1DD024A3D3E907
:10E9D8000023F1F7DBFB00220023F1F70BFE0028F0
:10E9E800EAD0002CBEBF4FF480133341E41824EA68
:10E9F80007040025E0E7332E0ADDB6F5806F03D162
:10EA0800F1F7C4FB02460B4610461946BDE8F081F3
:10EA1800A7F213474FF0FF3C2CFA07F70742F3D051
:10EA28000FA3D3E90023F1F7B1FB00220023F1F78C
:10EA3800E1FD0028C0D0002C0ADA142E01D10134DF
:10EA480006E0C6F134060123B3401D444545F6D31C
:10EA580025EA0705B0E700252C46ADE7AFF30080AF
:10EA68009C7500883CE4377E0000F0BFFFFF0F0074
:10EA7800F8B500BFF8BC08BC9E467047F8B500BFA3
:08EA8800F8BC08BC9E46704773
:10EA90000000000001000000020000000000000073
:10EAA0008813000010270000204E00003075000081
:10EAB000409C000050C3000060EA0000C0D4010088
:10EAC00080A903000053070000EA06370000000099
:10EAD0005000000040F7093700000000500000001F
:10EAE000C194C10000000000B22700000000000037
:10EAF0000000000000000000000000000000000016
:10EB0000000000003116000845160008DD15000859
:10EB10002D160008D9150008431600082564732532
:10EB20003033643A0000000065190008051A000837
:10EB300075190008111A0008D51900081D1A0008D7
:10EB400000000000851900083D1900080919000897
:10EB5000C1180008191900082D190008CD1800085F
:10EB6000D1180008E51800088D1C0008B51C000825
:10EB7000391C0008251C0008A0860100400D030078
:10EB8000801A060000350C0040420F0080841E00F1
:10EB900000093D0000127A000024F40000366E01E6
:10EBA0000048E801006CDC020000000000000000EA
:10EBB0000000000000000000000000000000000055
:10EBC0000000000000000000010000000200000042
:10EBD000030000000400000001000000030000002A
:10EBE0000500000001000000010000000600000018
:10EBF0000A000000200000000200000004000000E5
:10EC0000080000001000000040000000800000002C
:10EC100000010000000200000100020004000600E4
:10EC200008000A000C0010002000400080000001D5
:10EC300008040204080101010101010307010000A9
:10EC40006572726F723A20526567696F6E206973E0
:10EC5000206E6F7420646566696E656420696E203D
:10EC6000746865204D573A20736574206C6F72612B
:10EC700077616E5F636F6E662E68206163636F728B
:10EC800064696E676C790D0A004D414320727854B7
:10EC9000696D654F75740D0A004D414320747854B9
:10ECA000696D654F75740D0A004D414320727844BB
:10ECB0006F6E650D0A004D4143207478446F6E6598
:10ECC0000D0A00080A0C0D0E10121415181A1B1D3F
:10ECD0001E212403050205010602020500000600AC
:10ECE0000001050404020202020202020202020200
:10ECF00002020202030202020202020304030202EF
:10ED000002020204050403020202020506050403CE
:10ED100002020206070605040302020707070605AA
:10ED200004030207070000000000000102010000C8
:10ED300000000002030201000000000304030201BE
:10ED40000000000405040302010000050605040399
:10ED5000020100060706050403020107070706056E
:10ED6000040302070700000B357DF2F2F233337320
:10ED700073DEDEDEDE33337373F2F2F2F200000094
:10ED800048E8010048E8010048E8010048E80100BF
:10ED900048E8010048E8010090D0030000000000AE
:10EDA0000C0B0A090807073252585F2573206F6E53
:10EDB000206672657120256420487A2061742044A1
:10EDC000522025640D0A005258206F6E206672652D
:10EDD0007120256420487A206174204452202564E3
:10EDE0000D0A005458206F6E2066726571202564EC
:10EDF00020487A2061742044522025640D0A003195
:10EE00000032004D756C74695F43004D756C746918
:10EE10005F500000FFED000801EE000809EE000859
:10EE200003EE000811EE00080BEE0008A584998D92
:10EE30000DBDB1545003A97D1962E69A459D4087E6
:10EE400015EBC90BEC67FDEABFF7965BC21CAE6A17
:10EE50005A41024F5CF434089373533F0C52655E81
:10EE600028A10FB509369B3D2669CD9F1B9E742EA8
:10EE70002DB2EEFBF64D61CE7B3E7197F568002C0E
:10EE8000601FC8EDBE46D94BDED4E84A6B2AE516B2
:10EE9000C5D75594CF100681F044BAE3F3FEC08A7B
:10EEA000ADBC4804DFC17563301A0E6D4C14352FAC
:10EEB000E1A2CC3957F28247ACE72B95A098D17FDD
:10EEC000667EAB83CA29D33C79E21D763B564E1E43
:10EED000DB0A6CE45D6EEFA6A8A4378B324359B70A
:10EEE0008C64D2E0B4FA0725AF8EE918D5886F722A
:10EEF00024F1C751237C9C21DDDC86859042C4AA85
:10EF0000D8050112A35FF9D0915827B93813B3334C
:10EF1000BB7089A7B622922049FF787A8FF88017B4
:10EF2000DA31C6B8C3B07711CBFCD63AC6F8EEF6E4
:10EF3000FFD6DE916002CE56E7B54DEC8F1F89FA01
:10EF4000EFB28EFB41B35F452353E49B75E13D4C2B
:10EF50006C7EF5836851D1F9E2AB622A0895469D33
:10EF600030370A2F0E241BDFCD4E7FEA121D583496
:10EF700036DCB45BA476B77D52DD5E13A6B900C162
:10EF800040E379B6D48D67729498B085BBC54FEDD8
:10EF9000869A66118AE904FEA078254BA25D800559
:10EFA0003F2170F16377AF4220E5FDBF811826C392
:10EFB000BE35882E9355FC7AC8BA32E6C0199EA396
:10EFC00044543B0B8CC76B28A7BC16ADDB64741490
:10EFD000920C48B89FBD43C43931D3F2D58B6EDA59
:10EFE00001B19C49D8ACF3CFCAF447106FF04A5C2A
:10EFF00038577397CBA1E83E96610D0FE07C71CC3A
:10F000009006F71CC26AAE6917993A27D9EB2B22F2
:10F01000D2A907332D3C15C987AA50A50359091A4F
:10F0200065D784D082295A1E7BA86D2C637C777BA0
:10F03000F26B6FC53001672BFED7AB76CA82C97DF4
:10F04000FA5947F0ADD4A2AF9CA472C0B7FD932685
:10F05000363FF7CC34A5E5F171D8311504C723C389
:10F060001896059A071280E2EB27B27509832C1ACD
:10F070001B6E5AA0523BD6B329E32F8453D100ED27
:10F0800020FCB15B6ACBBE394A4C58CFD0EFAAFB0B
:10F09000434D338545F9027F503C9FA851A3408FD3
:10F0A000929D38F5BCB6DA2110FFF3D2CD0C13ECEB
:10F0B0005F974417C4A77E3D645D197360814FDC80
:10F0C000222A908846EEB814DE5E0BDBE0323A0A64
:10F0D0004906245CC2D3AC629195E479E7C8376DE8
:10F0E0008DD54EA96C56F4EA657AAE08BA78252E0D
:10F0F0001CA6B4C6E8DD741F4BBD8B8A703EB56696
:10F100004803F60E613557B986C11D9EE1F8981186
:10F1100069D98E949B1E87E9CE5528DF8CA1890D75
:10F12000BFE6426841992D0FB054BB162323232319
:10F13000232320257320253032583A253032583A7F
:10F14000253032583A253032583A253032583A254F
:10F150003032583A253032583A253032583A253034
:10F1600032583A253032583A253032583A25303222
:10F17000583A253032583A253032583A25303258EC
:10F180003A253032580D0A00232323232323204419
:10F1900065764555493A20202020202025303258D8
:10F1A0003A253032583A253032583A253032583ADA
:10F1B000253032583A253032583A253032583A25DF
:10F1C0003032580D0A00232323232323204170705B
:10F1D0004555493A202020202020253032583A2514
:10F1E0003032583A253032583A253032583A2530A4
:10F1F00032583A253032583A253032583A25303292
:10F20000580D0A00232323232323204465764164D9
:10F2100064723A2020202020253032583A2530329E
:10F22000583A253032583A253032580D0A0041708C
:10F23000704B65793A2020202020004E776B4B657B
:10F24000793A2020202020004E776B534B65793A85
:10F250002020202000417070534B65793A202020F7
:10F2600020004442496E744B65793A202020004DBD
:10F2700043526F6F744B65793A2020004D434B45E4
:10F280004B65793A20202020004D43417070534B4C
:10F2900065795F303A004D434E776B534B65795F2C
:10F2A000303A0000000000004150505F2EF200088C
:10F2B000010000004E574B5F3BF2000808000000C1
:10F2C0004E574B5348F2000809000000415050537C
:10F2D00055F200080A0000004442495F62F200084B
:10F2E0000B0000004D4352546FF200080C00000068
:10F2F0004D434B457CF200080D0000004D434B3060
:10F3000089F200080E0000004D41533089F20008D8
:10F310000F0000004D4E533096F200081000000020
:10F320005A45524F63F30008526164696F53656E2A
:10F3300064204F76657273697A650D0A00495251EF
:10F340005F52585F54585F54494D454F55540D0A0C
:10F3500000505245204F4B0D0A0053594E43204F49
:10F360004B0D0A00484452204F4B0D0A00484452AE
:10F37000204B4F0D0A004952515F4352435F4552A3
:10F38000524F520D0A00020100030000841E0000CB
:10F39000093D0000127A000024F4000048E8010052
:10F3A00090D0030020A1070000000000B128000059
:10F3B00061510000C3A20000040506009DC10008C1
:10F3C00061C0000899C20008DDC00008B1CB000888
:10F3D00085C10008DDC8000855C7000841BF000806
:10F3E000EDCD00082DCC000871C1000859C00008FF
:10F3F00009C10008E1C0000899C000088FC00008DA
:10F4000091BF00088DBF00088BC0000887C00008AE
:10F4100031C200085DC200087DC0000809CF0008A5
:10F42000F1BF0008B9BF0008D9CE000895BF000899
:10F430005DC50008E5C2000825DD00082BDD0008D9
:10F4400085BF000889BF0008C01200001F0000002F
:10F45000A816000017000000841C00000F00000028
:10F46000E42500001E000000B42D0000160000007E
:10F47000083900000E0000002C4C00001D000000A8
:10F48000685B000015000000747200000D000000B1
:10F49000589800001C00000034B700001400000061
:10F4A000E8E400000C000000783101001B000000BF
:10F4B000686E01001300000034CA01000B00000058
:10F4C000286202001A00000040DB02001200000067
:10F4D0003C9303000A000000C0C2040019000000B1
:10F4E00060B305001100000038200700090000008B
:10F4F00020A1070000000000040302020101010135
:10F5000000000000000000003C4E554C4C3E003016
:10F510003132333435363738396162636465666752
:10F5200068696A6B6C6D6E6F7071727374757677E3
:10F5300078797A00303132333435363738394142D0
:10F54000434445464748494A4B4C4D4E4F50515213
:0CF55000535455565758595A00000000FB
:10F55C00000000000000000000000000000000009F
:10F56C000000000000000000002B7E151628AED213
:10F57C00A6ABF7158809CF4F3C012B7E151628AE8C
:10F58C00D2A6ABF7158809CF4F3C082B7E15162851
:10F59C00AED2A6ABF7158809CF4F3C092B7E1516BA
:10F5AC0028AED2A6ABF7158809CF4F3C0A00000055
:10F5BC00000000000000000000000000000B000034
:10F5CC0000000000000000000000000000000C0023
:10F5DC000000000000000000000000000000000D12
:10F5EC00000000000000000000000000000000000F
:10F5FC000E000000000000000000000000000000F1
:10F60C00000F0000000000000000000000000000DF
:10F61C0000001000000000000000000000000000CE
:08F62C000000000000000000D6
:08F63400440BFF7F0100000000
:04F63C005D01000864
:04F640003901000884
:10F644000000000025030020102700000000010036
:10F6540000000000000000000000000004000000A2
:10F66400401F000075170008A5170008BD17000803
:10F6740029180008211E0008FD200008851D000827
:10F68400252100080000000059200008312000084E
:10F6940085200008531D00084F1D0008511D000857
:10F6A4008D1D0008551D0008611D0008FD1F000880
:10F6B4000200000000093D001000000000000000EE
:10F6C400D00500200000000000000000FF00000042
:10F6D40000000000D0050020000000000000000031
:10F6E400000000000000000000000000D005002021
:10F6F4000000FF0000000000E00000009D62000820
:10F70400CD610008D961000805620008000000000E
:10F7140000000000F5620008E56100086566000865
:10F7240000000000000000000000000000000000D5
:10F73400000E0F0D0109081101000000FF00000078
:08F74400FFFFFFFFFFFFFFFFC5
:040000050800233597
:00000001FF
